:020000040000fa
:080000002801040000000000cb
:020000040000fa
:10020000de8304000000000036420400000000000d
:100210005e830400000000002a400400000000008b
:1002200006810400000000002a8504000000000090
:10023000fe850400000000007e880400000000002d
:10024000c401040000000000ee01040000000000f2
:10025000ef5c22008079220000018800000000008d
:10026000050007000c000700723c020000000000bf
:100270000040da000000fe004440a90040fc2000dd
:100280000000e0000300320010002000a001880000
:100290004440a80000000600203723001100200081
:1002a0001600370062004000e0804800910188009d
:1002b0009001ba0062004000e0804800910188008f
:1002c0009002ba0062004000e08048000002eb00ab
:1002d0006028e10005003a008301e90007003300cf
:1002e000038009000059eb00040037006128e10099
:1002f000010032000082eb00050007009101880038
:100300001001ba000200e000e6ff3a00000005001c
:10031000910188008002780062004000e08048007f
:100320003559ba008301e900080032002559ba00a6
:100330008301e900050032000400e000f4ff320010
:1003400015d9ba008301e900f1ff3a000000060068
:10035000800078001106b100030035009101b10062
:1003600001003c000050a100000006008000780061
:10037000010037000000e8001004e000fdff3a0033
:100380000100500000000600900178000200e0002b
:1003900002003a000308e900050037008080eb0006
:1003a0001304e000020032000308e8009300fb00a1
:1003b00001007800000006000200fa00f0bf9f0074
:1003c0003fb99700ea8157008f80e900401c200068
:1003d0004c0107000080fa0000000600881f78002a
:1003e000020478003e010700080040004f04780036
:1003f000000006000000fa00881f78000004780062
:100400003fb99700ea81570080007800e01e200085
:1004100004020700800078000000e00002003500c0
:100420000040eb0080707c00010078004f047800f1
:100430000080fa0000000600ec874700889fbe009d
:100440008a9fbe008c9fbe008e1f7800f0b79f0071
:1004500081bf9f008204780000047800010037000b
:100460000804e800184778000e00fb00a50207000a
:100470000000e000faff3a00d0c2b300804f5700fe
:100480000500320000c0e900804f57000200320032
:1004900000477800010037000804e8000900e00088
:1004a00045003500e18f5400430032004002200037
:1004b000808f540040003c000900e0000e00340032
:1004c000f08f54001a003a0000c3b300984f100098
:1004d00016003a009840900080c7b30080cf5000cb
:1004e0000300320080c5b30080cf50000f003a00f7
:1004f0000884e8000e003700a900200000c3b30004
:10050000984f10000a003a009840900080c7b3004e
:1005100080cf5000040032008900200080c5b30065
:1005200080cf500002003a000884e8000901200052
:1005300008057800010037000a05e80000c3b30091
:100540009a4f1000fcff32008a0578006066b80000
:100550000e00370030fc200000425200c4ef9f0024
:100560006149b9000c00be00e30f07004fea970095
:100570000401fb00cf91de008b05e800ccb79f00a3
:10058000ddb79f0000064100818649001b00fb008b
:1005900064020700800078000901780030fc200028
:1005a00067020700000278000000e000e9ff3a005f
:1005b0008b0f540006003a000fb897000000e000cf
:1005c00029003200ffb097000108780026003700ac
:1005d0008a805500e0f92000694078000000fb00a7
:1005e00000805000160033004240a9000f003c007c
:1005f0004fe997000200fb00cf80de0000005600ac
:1006000081805e00800f5600818f5e0007003900f8
:100610006149b900be0f07004fb19700dfb19700e5
:10062000820f5000838f5800050032002002200006
:10063000909088000086eb008086eb000500370074
:10064000d0c2b300804f570002003a006006160087
:10065000e0861e008fb997000300e000030032001f
:100660008b097800010037006066b8000c00be00fe
:100670004f0778004f06be004f05be004f04be0076
:10068000cf00b10000000600889fbe00e3044000d8
:100690000900a100808f540049003600e38f540008
:1006a00001003e0049002000109080000000e000a2
:1006b00002003200800078000c0037004120210049
:1006c00003003700908f5400230036008080e8003c
:1006d000110078001100e000faff3a000f00370027
:1006e000928f54001c0036008280e80011017800cf
:1006f0001100e000faff3a001001780041202100cb
:1007000003003700908f5400130036008080e8000b
:1007100011007800820f5000faff3a000890800024
:10072000890f5400010031000904780008007800a6
:10073000130207000000e00004003a00890f540093
:100740001f0032000804d100f5ff370008187800b8
:1007500030000700d4ff37001101780092017800c3
:1007600064805100890f5000030031001200900096
:1007700080087800070037000900410080087800f1
:100780009201900013009800110078001288140064
:1007900009097800910178001100e000040032009e
:1007a000130090008380e8000000e00001003a00a0
:1007b0008000eb00119088000280e8000100370003
:1007c0000000eb004f04be000000060000047800ab
:1007d000060037008200410040908000e100780070
:1007e0000200e80030908800010001003290800093
:1007f00050908000800f5100f6ff3900201021003a
:100800004090880020022000509088000800780066
:10081000b20d07000000e000300032008080e900e7
:1008200091027800e38f52002c0036000508a300e7
:100830002a003a00229080000200e000020032000c
:10084000828f500004003100020878002190880057
:100850001600370003017800920190000300e000c9
:1008600002003200818f5100faff39001202780035
:1008700004004100808f500018003900810f5000a3
:1008800003003a00050942008200780007003700a3
:100890000300e0000300320005804000808f51001b
:1008a0000e0039009300980011019800110190008a
:1008b0000200e0000900320011804000820f500069
:1008c00006003a000232ef0011009000110178009a
:1008d0009008410010009000900098000000060071
:1008e000000278008001780001003700b1597800db
:1008f00002004200808f5100fcff3a0004007800a3
:10090000000006001200fa00889fbe008a9fbe0009
:100910008c1f780002047800a0b79f00b1b79f0039
:1009200083007800788057009c0107000000eb00ee
:10093000e0b79f00d8b79f0000067800dfb49700ab
:10094000194578000a80fb000000ea00cf05de00b0
:100950000a00fb006b0107000000e0001a003200f3
:100960006fb097000000e800e0b79f001200200081
:100970008000eb003fb09700afb19700030001008b
:10098000000478005f010700000178000000e0002b
:10099000f3ff3a006fb09700e10f44000700320008
:1009a0000000e900e0b79f00880078003fb09700a2
:1009b000afb1970003000100220037000000e900fa
:1009c000e0b79f001f0037000b04e90050c2b300de
:1009d000804f5500190032000b04780017003700d3
:1009e0006fb097000000e800e0b79f001200200001
:1009f0008000eb003fb09700afb19700030001000b
:100a0000800078001900fb00808f50000a0032003f
:100a1000e18f40007d0032006fb097000000e900d8
:100a2000e0b79f000001eb003fb09700afb1970027
:100a300003000100750037008904e8000804e9009c
:100a4000e7ff3b005fb097008b004000d1b79f00ed
:100a500050c2b300804f5500030032000a04e0008a
:100a6000b6ff3a0069003700114178008041eb0081
:100a7000a0c2b300804f510003003a000100e8001b
:100a8000d0b79f0082417800a3f79f000000eb00e1
:100a900080bf9f000b0037008fb89700f0ff270042
:100aa000808f5000040032006a08b9000000410045
:100ab0000300400080bf9f005fb097000000e80087
:100ac000d0b79f00dfb49700194478000801fb00fd
:100ad00003fd2f0003004100e90f5000eeff360038
:100ae0008800fb00e0572200310107000000e00011
:100af00002003a0000447800020037000900e800d4
:100b0000d0b79f00b8f79f0080c6b300804f540055
:100b100005003a00dfb0970066405000914f140086
:100b2000080032000a003700c0c6b300804f5400ee
:100b300007003a00dfb09700914f140004003a001c
:100b400065404000b0f79f000100e800d0b79f006b
:100b50005fb097009000fb0050582200140107007e
:100b60000000e00019003a006fb097000000e800b4
:100b7000e0b79f00120020008000eb003fb097001c
:100b8000afb197000300010000047800dd0007000a
:100b9000000178000000e000f3ff3a006fb097001a
:100ba000e10f4400070032000000e900e0b79f00b9
:100bb000880078003fb09700afb1970003000100b4
:100bc000020037000000e900e0b79f007c8057007a
:100bd000c90107000000e00003003c000c00e00039
:100be00009003200090037004ff097000004e000d0
:100bf000010032000c06e8005fb097000000e8003a
:100c0000d0b79f004dff3700000678000c00780039
:100c10004f0678004f05be004f04be000080fa006a
:100c2000000006006200fa00889fbe008a9fbe0096
:100c30000004be00020578008300780060f92f00f0
:100c40000f004000d500070088979f0099979f00ec
:100c50000000eb00a09f9f009a4578000b80fb00ee
:100c60000000ea00cf04de000904e90050c2b3002e
:100c700080cf550001003200090478000800e00030
:100c80000b003400080178008a0078001f9097005c
:100c90008f9197000300010090979f000000e000f3
:100ca000930032002f98970008004000a09f9f00fb
:100cb0000905450050c2b30080cf55000400320042
:100cc0000b04e000e4ff3a002f98970089003700fa
:100cd0000000eb00809f9f00f0979f00e0979f002f
:100ce000d0979f00c0979f00b0979f00c09f9f0024
:100cf00009003700201b2100008050000000400048
:100d0000611a2100e08078004f9897000100700080
:100d1000c09f9f000a05e8001a4478008800fb0085
:100d2000201b2100a2000700800078000000e000e6
:100d3000f0ff3a00a0c2b300804f54000e003a000a
:100d4000bf8897000180e900b08f9f009000780075
:100d5000b19f9f000100e00005003d000100ea0096
:100d6000b09f9f004f9897000020a000c09f9f0059
:100d70000a05e80010003700b19f9f000900370006
:100d8000bf989700f0ff2700808f500004003200ca
:100d90006a08b9000000410003004000b09f9f00b6
:100da0000a05e8001a01fb0003fd2f0003004100c3
:100db000e90f5000f2ff3600e0c2b3009a4f100076
:100dc000040032000080eb00909f9f008a047800ae
:100dd0001c0037008a04e800a0c2b300994f10003d
:100de00007003a00bf8897000180e900b08f9f009c
:100df00010007800909f9f008a84e800110037005f
:100e00000000eb00909f9f00090037009f9897001b
:100e1000f0ff2700808f5000040032006a08b900fc
:100e20000000410003004000909f9f008904e800fb
:100e30001901fb0003fd2f0003004100e90f5000e2
:100e4000f2ff3600194478008800fb00a058220009
:100e5000570007000000e00002003a00004478005c
:100e6000010037008904e800a87f9f0080c6b30016
:100e7000804f540004003a0066405000994f14001f
:100e80000700320008003700c0c6b300804f54008e
:100e900005003a00994f140003003a0065404000f5
:100ea000a07f9f008904e8000905e800c8fb2f0027
:100eb0000f04440060f92f000f0040008085e80017
:100ec0008801780019417800800078000b007800d4
:100ed000a00107000000e00005003a00880078004b
:100ee0000b0078003a0007000000e0005aff3d00c8
:100ef0000080eb004f05be004f04be000080fa00ea
:100f0000000006006900e100040035006d00e1000a
:100f1000030034000002b1000100320000000500af
:100f200010000500800078001104b10003003500b6
:100f30009101b10001003c000050a000000006003b
:100f4000820178000400370090cf100005003200c5
:100f50000000e8008301e9000300e000faff3a0026
:100f60000000eb0000000600809080000000e00020
:100f700001003200000001002021210000000600d5
:100f80000000e00003003400dc0b0700e10f40002c
:100f900001003a000000eb00000006000200fa0029
:100fa000f1bf9f00010878000080fa0000000600f1
:100fb000040037001004e00001003a0000000500c2
:100fc0000000e80090cf1000faff3a000000060091
:100fd0000400fa00889fbe008a9fbe008c1f780024
:100fe000000478000106780070089000f800900076
:100ff00001005000880890000100500098089000ff
:1010000001005000a808900001005000b8089000ae
:1010100001005000c8089000810550000002220025
:10102000a0bf9f000003230090bf9f000810900006
:101030000028a30018003a000b00e000160034005e
:101040008b04780009057800e28f54000200360016
:101050002a002000020037000900e0000b003400e5
:10106000c80190000a017800ec80570058009000f9
:1010700003000100500498000000e00096003200d8
:10108000680890000a004000600c98008a845400b0
:101090004240a900ebff3c00780190000200e00014
:1010a0000b003400c80190008c00780058009000bc
:1010b00003000100500498000000e00086003200a8
:1010c00068089000f800900001004000600c980053
:1010d000880c90000900e000150034000905780034
:1010e000e28f5400020036002a0020000200370080
:1010f0000900e0000b003400c80190000a017800ec
:10110000ee80570058009000030001005004980042
:101110000000e00070003200680890000a00400003
:10112000600c98008a8454004240a900ebff3c0008
:10113000180990000200e0000b003400c801900084
:10114000e80090005800900003000100500498004f
:101150000000e000600032006808900098089000ed
:1011600001004000600c9800a80c90000900e0000d
:101170001500340009057800e28f540002003600a3
:101180002a002000020037000900e0000b003400b4
:10119000c80190000a017800ee80570058009000c6
:1011a00003000100500498000000e0004a003200f3
:1011b000680890000a004000600c98008a8454007f
:1011c0004240a900ebff3c00380990000200e0001b
:1011d0000d003400e8009000180890008080400066
:1011e000c8019000580090000300010050049800ce
:1011f0000000e0003800320068089000b808900055
:1012000001004000600c9800c80c90000900e0004c
:101210001500340009057800e28f54000200360002
:101220002a002000020037000900e0000b00340013
:10123000c80190000a017800ee8057005800900025
:1012400003000100500498000000e000220032007a
:10125000680890000a004000600c98008a845400de
:101260004240a900ebff3c00081090000028a300ba
:101270001b0032000b00e000190034008b047800e2
:1012800009057800e28f5400020036002a00200091
:10129000020037000900e0000b003400c801900094
:1012a0000a017800ec80570058009000030001000c
:1012b000500498000000e000070032006808900029
:1012c0000a004000600c98008a8454004240a90043
:1012d00003003400eaff37000080eb000100370014
:1012e0000000eb004f0678004f05be004f04be0023
:1012f0000080fa0000000600881f780000047800d3
:101300000040eb00005498003800900090407800b6
:1013100090c6b30080cf50002a00320013003c007a
:101320007140500080cf50002600320005003c0084
:1013300050c2b30080cf50006400320030c5b3000b
:101340001b00370030c6b30080cf50001b003200b6
:101350000040e80080cf50001a0032006940500081
:1013600080cf50006e003a007300370000c7b30012
:1013700080cf500007003c000040e90080cf5000c3
:1013800010003d000040e90080cf500064003a00aa
:101390000f00370050c7b30080cf50000900320063
:1013a0006340400080cf500006003200654050008e
:1013b00080cf500043003200590037008000eb001e
:1013c0005e003700080078009a0207005f003700cf
:1013d000684890000004e0005b003a00f848900084
:1013e000c0c6b30080cf5000270032000a003c0086
:1013f0006440500080cf50002b00320000c0e80055
:1014000080cf5000150032006840500080cf50005f
:1014100025003a000a00370040c7b30080cf5000d3
:10142000210032006640400080cf50001e00320094
:101430006940500080cf50001b003a000700370081
:10144000280090000080e900200498001000780037
:10145000084c9000084878003b00370028009000b6
:101460000080e900200498001002780048009000f5
:10147000cf80de000101780082017800009abe0072
:101480000292be0030003700280090000080e90082
:10149000200498001001780048009000cf80de0002
:1014a0000089be0028003700280090000080e90075
:1014b0002004980010007800480490000808780084
:1014c00021003700110020001c0037004800900068
:1014d0000000e80040049800980178001200200005
:1014e0008000eb00180090000300010080007800ed
:1014f00050022000808f50001300320048009000fe
:10150000e18f4000080032000000e900400498002c
:10151000980178000001eb00180090000300010022
:101520000000eb00090037000000e90040049800cb
:1015300001007800050037008080eb00080078008b
:101540009603070001003700100020004f047800c8
:1015500000000600889fbe008a1f78000004780003
:1015600001027800824478000305780070c6b30059
:10157000804f510021003c0000c0e900804f510025
:10158000e5003d0072405000804f51005101320093
:101590000d003c006c405000804f510066013c0043
:1015a00000c0e900804f5100db003d0050c2b30095
:1015b000804f51005d0132007c404000804f51005f
:1015c0005d013a00d400370010c6b300804f5100cf
:1015d000d100320004003c0069405000804f5100af
:1015e00055013a007500370030c6b300804f5100f6
:1015f000180032000040e8000900370000c7b300bf
:10160000804f51002401320008003c0000c0e90076
:10161000804f5100ea00320068003c0065405000f5
:1016200080cf540044013a000f00370050c7b30088
:10163000804f51006100320063404000804f5100f4
:101640005e00320065405000804f51003a013a0080
:10165000200137009180e900010a780078009000ad
:1016600011f079003a013700a8609000c0c6b300bd
:1016700080cf50000a003a00140078006401500046
:10168000020a78001200be004f88de00cf80de0024
:101690001202be00000378008003780016003700b5
:1016a00010c7b30080cf500003003a0094007800c8
:1016b000688050000500370014017800a0c6b30010
:1016c00080cf500005003a0068005100000a780001
:1016d0003002be002003be00070037000280e90090
:1016e000000a78001000780000027800cfa2de0027
:1016f0000503780086037800049cbe000694be00b3
:10170000a860900080c6b30080cf50000e00320069
:1017100020c6b30080cf500005003a000400fb0053
:10172000cf80de0001017800820178000a003700d6
:1017300040c7b30080cf5000030032006640400035
:1017400080cf500006003a0004007800cf80de0011
:101750000101780082017800009cbe000294be0066
:101760003800be002801be00e00f5000e08f580096
:10177000e00f5900e08f590003003d007800900011
:10178000d1c2b3000a003700081090000018a3006f
:101790000300320078009000b1c2b30004003700ab
:1017a0000008a300570032007800900001c2b30087
:1017b00001707d000000e80051003700a860900033
:1017c000c0c6b30080cf500007003a0094007800f4
:1017d00064805000000a78001002be000003eb0095
:1017e000860378001600370010c7b30080cf500082
:1017f00003003a009400780068805000050037002c
:1018000014017800a0c6b30080cf500005003a0054
:1018100068005100000a78003002be002003be00bc
:10182000070037000280e900000a78001000780005
:1018300000027800050020000600200007002000bc
:10184000049cbe000694be00a860900080c6b30051
:1018500080cf50000e00320020c6b30080cf500071
:1018600005003a000480fb00010020000200200077
:10187000030020000a00370040c7b30080cf5000ab
:10188000030032006640400080cf500006003a005e
:101890000400780001002000020020000300200066
:1018a000009cbe000294be00081090000038a30007
:1018b000140032003800be002801be00e00f5000c6
:1018c000e08f5800e00f5900e08f59000d00320002
:1018d00080c7b30080cf54000300320080c5b3003e
:1018e00080cf540007003a007800900001c3b30095
:1018f00001707d008000e80089707d000080e800b4
:101900007004980078009000000045006004980082
:10191000894078006c003700a860900014017800be
:10192000c0c4b30080cf500005003a0068005100e9
:10193000000a78005001be004000be0004003700dd
:1019400064005100000a78001000be00000b070080
:10195000009cbe000294be00380090000000e00031
:1019600003003d0078009000d1c2b3000a003700a8
:10197000081090000018a3000300320078009000c7
:10198000b1c2b300040037000008a3000500320014
:101990007800900001c2b30001707d000000e800f3
:1019a00070049800780090000000450060049800e2
:1019b0008940780008007800680307006600370057
:1019c000a8609000c0c6b30080cf50002500320050
:1019d0000a003c006440500080cf500028003200d4
:1019e00000c0e80080cf5000140032006840500072
:1019f00080cf500022003a000a00370040c7b300f1
:101a000080cf50001e0032006640400080cf500062
:101a10001b0032006940500080cf500018003a008f
:101a2000060037001480e900000a780010007800f2
:101a3000485c900008487800470037001480e900af
:101a4000000a78001002780068089000cf80de005d
:101a50000101780082017800009abe000292be0067
:101a60003d0037001480e900000a7800100178007a
:101a700068089000cf80de000089be003600370085
:101a80001480e900000a780010007800680c9000cb
:101a900008087800300037001180e90080087800dd
:101aa00010007800cf80de0001017800820178000c
:101ab000009cbe000294be0078009000000045002b
:101ac0006004980081c7b300080078002600070072
:101ad000210037001480e900000a780090017800a6
:101ae00063049800580990000200e00003003d00e4
:101af000030078001dfa07000a0037008000eb00a1
:101b0000030078000efd0700800078000000e00070
:101b10000300320068009000008050000100370090
:101b200058089000100c98000b00370078009000c7
:101b300002707d00060037007800900080004500ac
:101b40000904e00001003a0059c2b3008948780056
:101b50000000e800700498000000eb004f057800da
:101b60004f04be00000006006f02b000889fbe0058
:101b70008a9fbe008c9fbe008e1f780000067800f2
:101b8000d017210080bf9f0080c5b30080cf5000d8
:101b90000700320082002000f2b79f00c316210028
:101ba00083bf9f007740400080cf50000a00320082
:101bb00080c7b30080cf500005003200a400200091
:101bc000f4b79f0080c5b30080cf500002003a00f8
:101bd00000012000f0b79f003c04be002c05be00b1
:101be00040c6b30080cf5000030032006540400083
:101bf00080cf50000b003a00e00f5400e08f5c00f3
:101c0000e00f5d00e08f5d0006003d006000b80061
:101c10006011b80008045000898458000a05590072
:101c20008b855900e00f5400e08f5c00e00f5d00f1
:101c3000e08f5d0004003a005c0890008d012000f8
:101c40000000e0000c003200ffb0970001027800b5
:101c5000cfa2de0005037800860378000800be00ee
:101c60000a01be00e40a07000fba9700644078003a
:101c7000d0e79f007d0120007fb097000002780030
:101c8000cfa2de0005037800860378000800be00be
:101c90000a01be00d10a0700009ebe000296be00e7
:101ca0000d00e900e1fc2f008f804000008740001c
:101cb0001a0037007fb1970002027800cfa2de0041
:101cc00005037800860378003c00be002c01be00ae
:101cd000cd0a07000205be000004be008d06e90023
:101ce000ffb1970003027800cfa2de000503780061
:101cf000860378000800be000a01be004b0b0700f7
:101d00003fb29700000052008fb8970060cf780074
:101d1000089ebe000a96be000e07e9003c00be0009
:101d20002c01be00b0b79f00c1b79f00d2b79f0083
:101d3000e3b79f00e00f5000e08f5800e00f59001c
:101d4000e08f5900020034000d00e000d9ff3c0094
:101d5000ffb09700e88f500010003a000c10900080
:101d60000038a3000d003200f78f560006003e0039
:101d7000e2fc2f000d014100e2c07f0000c3b30070
:101d800080cf5000050032008d06e90000c3b3008b
:101d9000e3fc2f008d81410080f17f0078811600e7
:101da000120e98006c009000e3fc2f008f81410020
:101db0008d804100cafa07001c0990005c08900061
:101dc000800f510006003d0002005000000e9800f8
:101dd0000c1090000040a100001698000f00370082
:101de0000000e0000d003d000c1090007400600049
:101df000f00f500009003a007c089000fc009000b1
:101e0000010050008c0890000100500002005000ba
:101e10004240a90001003400000e98004f077800ee
:101e20004f06be004f05be004f04be006f02b1005a
:101e3000000006002f02b000889fbe008a9fbe00ef
:101e40008c9fbe008e1f7800800478006000900098
:101e50000000e00001003c00f0ff27000000e90066
:101e6000d0049800c90090000c0033000100e80085
:101e7000c004980099017800120020008000eb0057
:101e8000190090000300010000057800b002200056
:101e9000800f550006003a000b0037000100e800f3
:101ea000c00498002cfd2f000f0646001b003700d1
:101eb000d0022000800f5500030032002cfd2f00bf
:101ec0000f0646001600370030fd2f000f044000bb
:101ed000aad79f00590090000000e900d0049800a4
:101ee000c90090000a0033000100e800c004980017
:101ef00099017800120020008000eb00190090008a
:101f0000030001000005780008067800040037008f
:101f10000100e800c0049800080678000085eb0086
:101f2000d8142100390090009000fb0008007800d0
:101f30001ffc0700080050006114210060c47800f5
:101f40008805fb0000032000800f550033003a0095
:101f5000590090000000e900d0049800c9009000ea
:101f60000c0033000100e800c004980099017800db
:101f7000120020008000eb00190090000300010017
:101f80000005780080072000800f550005003a000a
:101f9000070037000100e800c00498000085eb004e
:101fa0001b00370080052000800f550018003a0004
:101fb0000804e00002003200f04f54001d003a0017
:101fc000590090000000e900d0049800c90090007a
:101fd000090033000100e800c0049800990178006e
:101fe000120020008000eb001900900003000100a7
:101ff00000057800030037000100e800c0049800e5
:102000000085eb000047eb000b01200011003700ba
:102010000804e000b8003200060037000047eb007b
:102020000804e00004003a00ad00200008477800f2
:102030001c0037001ec0b300ad002000ea4f540062
:1020400018003200e88f550002003a008b06780035
:10205000140037006d012000120037005900900075
:102060000000e900d0049800c90090000900330086
:102070000100e800c00498009901780012002000d7
:102080008000eb00190090000300010000057800bb
:10209000030037000100e800c00498000085eb0051
:1020a0001ec0b30000032000800f5500ebff32007c
:1020b0000e04e00018003200005e780016003700c1
:1020c0006f805700800f5600010031000a5e7800d3
:1020d000590090000000e900d0049800c900900069
:1020e000090033000100e800c0049800990178005d
:1020f000120020008000eb00190090000300010096
:1021000000057800030037000100e800c0049800d3
:102110000085eb001ec0b300e10f45000700320050
:102120000d0178008a0078005015210084fb07001b
:102130000000e000e2ff3a0066003700490090002e
:102140000000e900c00498000e04e00008003a0016
:1021500020fd2f000f004000800f56005b003a006a
:10216000e10f450059003a008a0078006500370009
:10217000004eeb0069489000110020000004e000d0
:1021800060003a00390090009040780040c6b300eb
:1021900080cf5000030032006540400080cf5000e7
:1021a0000a003a000b0178008000eb0020fd2f00b0
:1021b0000f004000930307000203be000002be00b0
:1021c00010c0b300805498000d0037000b01780058
:1021d0008000eb0020fd2f000f004000e30307000c
:1021e0000203be000002be0010c0b300805498007d
:1021f000b900900000c7b300914f10002c003200ce
:10220000f9489000c0c6b30080cf500022003200d1
:102210000a003c006440500080cf5000240032008f
:1022200000c0e80080cf5000140032006840500029
:1022300080cf50001e003a000a00370040c7b300ac
:1022400080cf50001a0032006640400080cf50001e
:10225000170032006940500080cf500014003a004f
:1022600006003700290090000080e900a0049800d3
:102270001000780004487800120037002900900010
:102280000080e900a0049800100078000498be00c7
:102290000690be000b003700290090000080e90086
:1022a000a0049800100078000488be0005003700e4
:1022b000290090000080e900a00498001000780038
:1022c00004087800110020000e0037008000eb00a9
:1022d0000c003700490090000000e900c00498009d
:1022e000990178000001eb008a0078001900900045
:1022f0000300010094ff37001ec0b3008b002000d4
:1023000052ff3700010078004f0778004f06be00eb
:102310004f05be004f04be002f02b10000000600b2
:1023200000027800110037008402e8009441780030
:10233000d0c2b300954f100008003a0081cf510081
:1023400003003e002440900080cf50001200360071
:1023500063024200630151000400370081cf510045
:102360000d0032000201e90005027800e20f510081
:10237000edff3e00840178000300370093cf10008a
:10238000050032008301e80002004200808f510006
:10239000faff3a000000050010000500ee87470034
:1023a000889fbe008a9fbe008c9fbe008e1f780053
:1023b00000047800810678000000eb00d0b79f0091
:1023c000f8489000c0c6b30080cf500002003a0029
:1023d00011002000d1b79f000d00e00024003d0057
:1023e000380190000200e800300498009040780026
:1023f0000040eb0080f79f00e0c5b30080cf5000a5
:1024000003003a000280e8003004980081f79f0042
:10241000b80490000901e800d0c5b300994f10003e
:102420000100320009017800d10520000200780087
:10243000dffa0700000778008000eb000000e000f2
:10244000bf00320009055000e20f550008003400bb
:102450000a81e9000900e800d1022000b8fa07006b
:1024600011c0b300c1ef9f000000e00002003a007d
:102470000040eb00c0ef9f00680090000000e0000b
:1024800004003c00f0ff27000d00e00001003a00ce
:102490001000200050049800684890000004e000fc
:1024a0000d003a0028009000dfb097000100e00026
:1024b000050032000080e900200498001000780038
:1024c000c0b79f00040037000080e9002004980096
:1024d00010007800f0b79f008045eb0061003700e6
:1024e0000d00e000030034000900780085fa0700c1
:1024f000200037000d00e000200032004fe8970078
:102500000004e0000d003a008ff097000104e000a5
:1025100005003a000a017800890078003800900030
:1025200087fa07000c0037000a017800890078005c
:102530003800900082fa07000e0037000ff0970075
:102540000004e00007003a000a01780089007800e2
:102550003800900072ff07000000e00007003a001a
:102560006e0037000a01780089007800380090007a
:102570006bff07000000e00068003a00dfb0970042
:102580000100e00009003a00684890000004e00003
:1025900033003a007fb0970009587800f0b79f00e9
:1025a00010c0b300005498002d003700e9e79f00e9
:1025b0000900fb008005fb00010032001000200034
:1025c000800478001c0020000000e00017003a00a2
:1025d0006fe097000004e00004003a007a805700a2
:1025e00062f707008004e800100037000c06e900dd
:1025f0007a005600e0c07f0048019000e1cf400023
:10260000080032000200e9004004980098017800b8
:102610000001eb008100fb001800900003000100a6
:10262000020037000200e900400498008c8f54003b
:10263000eeff3500684890000004e00005003a0015
:10264000cfb097008b187800c1b79f0010c0b300bf
:1026500000549800680090000000e90060049800b1
:102660002bc0b300580090000000e900500498000f
:10267000480190000b0033000200e800400498007d
:1026800098017800120020008000eb0018009000f4
:102690000300010080047800e10f400090ff3a0041
:1026a000020037000200e800400498004800900053
:1026b0000000e900400498000d00e0000200320034
:1026c000e2cf5500040032000b00fb008080eb00dd
:1026d0001b0032000f003700684890000004e00043
:1026e00009003a005fb097000000e00003003200ec
:1026f000cfb097008008eb0003003700afe89700e9
:102700007fb09700014878000d00e00001003d0017
:102710003e04980011002000090037004800900096
:102720000000e90040049800980178000001eb00e7
:10273000890078001800900003000100deff3700d8
:10274000010078004f0778004f06be004f05be001d
:102750004f04be00ef00b100000006002f04b000df
:10276000889fbe008a9fbe008c9fbe008e1f78008f
:1027700080bf9f00014778005001be004000be00ae
:10278000a09f9f00b19f9f00c29f9f00d39f9f006b
:1027900010c6b300804f57001500320010c4b300bc
:1027a000804f5700120032000fb997005208900076
:1027b0000000e00003003d00600020005009980088
:1027c0000b0037000000e00009003a0070c6b300bb
:1027d000804f57000300320070c4b300804f570091
:1027e00003003a00100020008fb99700d00998002c
:1027f0008fb8970020fb2f000f0040003d0307001b
:1028000000017800e20f500014003a003000200070
:102810000fba9700100a980010c6b300804f5700f7
:102820000a00320064404000804f57000700320029
:102830000040e800804f570004003200c1512200e0
:102840000040e800804f570001003a00015222008a
:102850008fba970065009000150037000000e00077
:1028600017003400300020008fb8970090089800bf
:1028700010c6b300804f57000a0032006440400089
:10288000804f5700070032000040e800804f57009b
:1028900004003200415222000040e800804f5700ff
:1028a00001003a00815222000fb9970062009000a7
:1028b000315878003158780011487800cb01370042
:1028c00014c6b300844f57000300320010c4b30095
:1028d000804f570011003a008fba9700e501900031
:1028e0008300780000c3b30080587800e1029800ac
:1028f00080c7b300844f57000100320080c5b30089
:10290000804878000380e8008fb89700e0009800c6
:10291000710090000080e800f00098000200e000e4
:1029200005003a00929f9f00c3fb2f000f814100da
:102930009f999700a9013700c4522200f4b79f0065
:1029400010c6b300804f57000500320010c4b3001a
:10295000804f5700b0003a00d5532200f5b79f00d2
:102960008fb897005108900012022000a2b79f0074
:102970000000e000020035000000e800a0b79f0062
:10298000afb197008301e800e3b79f006022b80071
:102990006033b8002f989700bf9897004f99970021
:1029a000df9997004f0807008fb897003102be00eb
:1029b0002103be000000e00004003d000400be0052
:1029c0000601be0003f0a200020037000400be00b2
:1029d0000601be00a09f9f00b19f9f00c29f9f0065
:1029e000d39f9f001f99970064015100929f9f0001
:1029f000c3fb2f000f8041000048eb00d4fb2f00e9
:102a00000f024200c4b79f0032003700c20120000d
:102a10000300200045fb2f000f804200e102070069
:102a20002f9c9700bf9c97004f9d9700df9d9700bc
:102a30000800be000a01be002f0807000006be0005
:102a40006fb1970067015100e2b79f004240a900b3
:102a50000a003400540807000002be000203be0052
:102a60000800be000a01be0052080700a09f9f0098
:102a7000b19f9f00c29f9f00d39f9f00cfb197003f
:102a80006780410071002000060037000000e90067
:102a90006f4866004c6add004466de000c0672007a
:102aa000c4eede00e00f5600e08f5e00050034004b
:102ab0008100e900e18f4000f4ff3a000100370097
:102ac0000060eb008100e900fdff3b006700400073
:102ad000c0b79f00efb297000500e0000900340086
:102ae0006022b8006033b8002f989700bf98970015
:102af0004f999700df999700300807000000e00029
:102b0000c2ff3c00c0fb2f008f0040004fb1970078
:102b1000010051000000e900afb19700830f5000a1
:102b200001003d00a0b79f00afb297000500e00094
:102b300004003d0085017800d0fb2f000f0140000c
:102b40002e0037002fb19700800f510005003d0087
:102b50000100410010409000f5c0b300e74f500065
:102b600001003c008042eb00d3fb2f000f804100ae
:102b70002fb29700040040008000e9000402e90041
:102b8000114178008100e900854f5100fbff3200c0
:102b90008401e800afb0970001005000000042003f
:102ba000efcf520001003a000248e80025fb2f0059
:102bb0008f8242006b8142000400e00005003d006e
:102bc0008301e8001f98970064004000909f9f00d9
:102bd0006a814200030041008000e900030278009e
:102be000040037001100fb00ffb29700e0c87a0034
:102bf0008100e9000402e900faff3b008fb897006a
:102c0000510890000000e000f4003d000300e900de
:102c1000d0089800f10037002f9c9700bf9c9700c8
:102c20004f9d9700df9d97006022b8006033b80089
:102c30000800be000a01be00aa0707000000e0006d
:102c400005003d000bf0a200a89f9f00b99f9f00c8
:102c5000ca9f9f00db9f9f001f9897007259270013
:102c60000280b900026a2800130020001306070042
:102c7000e4005000919f9f0015003b00e38010008e
:102c8000c0ff2f00008460000801ea00929f9f00af
:102c90002f989700bf9897004f999700df9997005a
:102ca00029032100070037000808a30003003200b1
:102cb0003902be002903be00c50707000884d10001
:102cc000e88444000800e000f7ff3c001c003700e7
:102cd0009f9997000300e0001d003400c0ff2f0003
:102ce00000806000909f9f00000478006000b800a2
:102cf0000200200003ff2300290321000700370002
:102d00000808a300030032003902be002903be00f8
:102d1000af0707000884d100e88444000800e00001
:102d2000f7ff3c000002be000203be002f98970090
:102d3000bf9897004f999700df99970019080700ef
:102d4000a09f9f00b19f9f00c29f9f00d39f9f00a5
:102d50000fba97005409900060c6b300804f570027
:102d6000040032006100200060c4b300804f5700af
:102d700002003a009f9a9700ea8042000101410058
:102d8000d2b79f00f30f5100020034003001200041
:102d9000d0b79f0000c3b300c07f9f00d1fb2f00be
:102da0008f804000b1b79f00310037000800be009f
:102db0000a01be00500707000006be005fb1970081
:102dc00068015100d2b79f004240a9000e003400b4
:102dd000750707000002be000203be000800be0027
:102de0000a01be00730707006022b80046782d0074
:102df0007719240076070700a09f9f00b19f9f00ce
:102e0000c29f9f00d39f9f00bfb19700688441007d
:102e10008900200008003700a200200003002000e5
:102e20000c00be005b0207000804e90004c3b30005
:102e3000044c41000006be00e00f5600e08f5e002b
:102e4000070034008904e900e18f4400f2ff3a00f2
:102e5000030037000804e90000c3b300004c780009
:102e60008904e900fbff3b0068044400b8b79f00f9
:102e7000dfb297000500e0000b0034002f9c9700a4
:102e8000bf9c97004f9d9700df9d97006022b80080
:102e90006033b8000800be000a01be004707070003
:102ea0000000e000c1ff3c00c1fb2f000f8040008c
:102eb0003fb19700000051008001e9001f9a970080
:102ec000e7004200d5fb2f000f81420001003700d0
:102ed0000201e80000c3b300924f1000fcff320073
:102ee000d4fb2f000f004200808040008280500001
:102ef0000080410082015000919f9f008fba97008f
:102f0000550a900060c6b300804f5700030032009e
:102f100060c4b300804f570002003a008100e8000f
:102f20000800370050c6b300804f5700040032003d
:102f30008000eb0050c4b300804f570001003a00fe
:102f40001100200001024200848f510001003d0069
:102f5000030278000400e00002003d0084017800d4
:102f60001e003700830f520005003d00e440790049
:102f700097c3b30040c3b30080cf500001003c00b2
:102f800007c3b300040041008001e9008402780017
:102f90008502e900134378008301e900874f53005d
:102fa000fbff32008501e8000400500080804200f1
:102fb00090c3b30080cf530001003a008648e80078
:102fc0000500e00005003d000201e9008301e80082
:102fd0001f9897000000e800909f9f001f9a97009d
:102fe0008e4078000fb89700040207004f07780062
:102ff0004f06be004f05be004f04be002f04b100b7
:10300000000006000200fa00889fbe008a9fbe00f2
:103010008c1f780080057800010578000206780092
:103020000100e00001003a006c8557000b047800b5
:10303000010037000804e800984478000900fb000c
:10304000b0f707000000e000faff3a00d0c2b3007a
:1030500080cf54000500320000c0e90080cf54004a
:103060000200320080447800010037000804e800c4
:103070000c0178008a007800080078003b00070007
:103080000203be000002be009a0f540001003a0085
:103090000b0d78009a8f550005003a00e00f5200a2
:1030a000e08f5a00e00f5b00e08f5b0014003a00f5
:1030b000b0c2b30080cf540006003a00e00f5200c7
:1030c000e08f5a00e00f5b00e08f5b0020003d00c6
:1030d0000b003700d0c2b30080cf54001c003a0070
:1030e0006000b80002002000030028000020e1007a
:1030f00001a8e10002b0e10003b8e1000e003600d3
:1031000020022000909088006b40400080cf540047
:1031100004003a006000b80002002000030028000c
:103120000d003700f0ff2f00f1ff2f00f2ff2f00fe
:10313000f3ff2700080037006000b8006011b800f6
:103140000402500085825800060359008783590005
:103150000400be000601be004f0678004f05be0009
:103160004f04be000080fa0000000600fc87470004
:10317000889fbe008a9fbe008c9fbe008e1f780075
:103180000007780081067800820478000004780047
:10319000010037000804e800184678000c00fb0026
:1031a00058f707000000e000faff3a00d0c2b30071
:1031b000804f56000500320000c0e900804f5600e5
:1031c0000200320000467800010037000804e800e1
:1031d0000900e00005003500e18f540003003200d3
:1031e00040022000808f5400040034000d00e000f5
:1031f000b00032008e0e7800ae0037000900e0000b
:103200000e003400f08f54001a003a0000c3b300df
:10321000984f100016003a009840900080c7b30005
:1032200080cf50000300320080c5b30080cf500033
:103230000f003a000884e8000e003700a9002000c3
:1032400000c3b300984f10000a003a009840900065
:1032500080c7b30080cf50000400320089002000f6
:1032600080c5b30080cf500002003a000884e80017
:103270000901200008057800010037000a05e80070
:1032800000c3b3009a4f1000fcff32008a0578009b
:103290006022b8006033b80026003700d00021005b
:1032a00080c0500081ef9f0009027800cfa2de00ad
:1032b00005037800860378000fb097009fb0970051
:1032c0002fb19700bfb19700d8050700d0b79f0076
:1032d000e1b79f00f2b79f0083bf9f000fe8970000
:1032e0000002fb00cfa2de00050378008603780011
:1032f0008b05e8000fb097009fb097002fb19700a3
:10330000bfb19700c0af9f00d1af9f00e2af9f0059
:10331000f3af9f005fb09700efb097007fb19700c9
:103320008fb997000002420081824a0002034b00dd
:1033300083834b0084b79f0095b79f00a6b79f007b
:10334000b7b79f001b00fb00f6f60700800078006f
:1033500009017800d0002100f9f60700800078000c
:103360000000e000cdff3a008b0f54000a003a0045
:103370000d00e0004f0032008e0e78006022b80091
:103380006033b80084b79f0095b79f00a6b79f0031
:10339000b7b79f004d0037008a80550080fe20009f
:1033a000694078000000fb00008050002c003300d2
:1033b0004240a90020003c008fea97000500fb0076
:1033c000cf80de0001017800820178000fb2970003
:1033d0009fb297002fb39700bfb397000000520031
:1033e00081805a0002015b0083815b000020e100c4
:1033f00001a8e10002b0e10003b8e1000e003900cd
:1034000009027800cfa2de00050378008603780069
:10341000f20407004faa9700dfaa97006fab97004e
:10342000ffab97000400e1000588e1000690e10091
:103430000798e1000a0032002002200090908800e6
:10344000f0ff2f00f1ff2f000001be0080b79f00aa
:1034500091b79f00a2b79f00b3b79f00110037003c
:10346000d0c2b300804f56000e003a006000b80092
:103470006011b8000fb297009fb297002fb397006a
:10348000bfb397000402500085825800060359001c
:103490008783590084b79f0095b79f00a6b79f0008
:1034a000b7b79f000d00e000080032008b0e7800d7
:1034b000060037006000b8006011b80080b79f00b8
:1034c00091b79f00a2b79f00b3b79f000fb09700be
:1034d0009fb097002fb19700bfb197004f077800ba
:1034e0004f06be004f05be004f04be00cf01b10025
:1034f00000000600889fbe008004780066844000bb
:1035000000ff2700180060004401de00f07f20006b
:10351000800f51000e003a00800ceb001804780078
:103520006f0064001c003a00210090000000e000e1
:1035300019003a00110090000000e00016003a0067
:10354000100020001100e0001400320012003700cb
:103550000200e00005003c0001007800db010700ec
:10356000000178000000e00008003c00f0002800a6
:103570001800600001fe2300010c700020c02f0025
:10358000800c41000080eb0004003700800ceb0051
:103590000000eb0001003700200020004f04be00b7
:1035a00000000600889fbe008a1f78008c9fbe0026
:1035b000000478000206be00e6044000190178000d
:1035c0000200d0004505de008a007800f07f200070
:1035d000800f55000c003a006f00610068003a004f
:1035e000280090000000e00065003a0018009000fc
:1035f0000000e00062003a00100020001800e00027
:10360000600032005e0037000a00e00007003a0068
:1036100008007800ad010700800078000000e0009d
:10362000020034000a007800560037006108b90033
:103630000c0140008d814800e07f2000800f510088
:10364000e08f59000d0034001900e00004003d0037
:103650006000b8000200200003ff2f0003003700c5
:103660006000b8000200200003ff2700009cbe009d
:103670000294be00100020004200370019027800ba
:10368000e00f5100e08f590008003400f1002800dd
:103690008100620002004100000040000000400084
:1036a00000004000808c70003300370000002800cc
:1036b000000362006f0062000040a000800c7800f0
:1036c00061015100e0815900c0fc2f00f1ff2f0083
:1036d000800f5100818f59000d003d00860c78004d
:1036e0000000eb002004980010049800000c780003
:1036f000240037008880e800110c78006400440042
:103700009008780019087800800ceb0070014100e7
:10371000f00f4100f7ff34008202ea00150032008a
:103720008881e80070821200980078008508de0029
:10373000130078000400dd00008c70006401440078
:10374000930078008508de00120078000400dd0098
:1037500080897000920078008508de0019007800ea
:103760000400dd0000897000190078000500de000b
:10377000800c7800990c73000080eb00010037008a
:10378000200020004f06be004f0578004f04be0009
:10379000000006000800fa00889fbe008a9fbe0055
:1037a0008c9fbe00e0b79f00f1b79f000206be00ed
:1037b0004203070080bf9f0091bf9f000001be0031
:1037c0000c00be004c0307006fb19700ffb19700db
:1037d00000055100818559000fbc97009fbc9700e0
:1037e0000800be000a01be004f06be004f05be0025
:1037f0004f04be000080fa0000000600ec8747007e
:10380000889fbe008a9fbe008c9fbe008e1f7800de
:1038100000047800014578000206780083047800ef
:10382000840678000300e00002003c00190020003c
:10383000ac59220060c6b300804f55000e00320024
:1038400060c4b300804f55000b00320070c6b30057
:10385000804f55000300320070c4b300804f550004
:103860009c003a00e48f4600800035005808900024
:10387000808f56007d003d008d05e80060c6b300d6
:10388000804f55001000320060c4b300804f5500d7
:103890000d003200081090000038a30004003a0028
:1038a00058089000808f540001003d00590c98008a
:1038b000580890000b005000500c980002003b008c
:1038c0000000eb00500c98000b00e00027003c00cb
:1038d000180990006800900001c3b30001717800de
:1038e0008201e800130c9800580890000000e000e6
:1038f00003003c00081090000038a30005003200cf
:1039000068009000e1c2b300817178000280e80095
:10391000100c9800d80890000b00ea00808f50002f
:1039200001003d008105ea000b00ea00200c980030
:103930000b804000500c9800890f500001003d00a2
:1039400080047800390c9800680090009808900076
:1039500001004000090178008c007800e0f30700c6
:1039600058089000090050001a003700980890008d
:10397000680090008b8f540018003d00010040004b
:10398000090178008c007800d5f307001808900032
:1039900009014000120c980009805500200c980085
:1039a000580890000000e00003003c000810900060
:1039b0000038a30006003200e8009000e0c2b30027
:1039c00000f17800380890000000e800300c980002
:1039d00058089000400c9800a400370001004000f7
:1039e0000b0178008c007800bdf3070018089000e8
:1039f0000b014000120c98008b8454005808900072
:103a00000000e00003003c00081090000038a30014
:103a10000500320068009000e1c2b3000171780037
:103a20000200e800100c980058089000890f500020
:103a300001003d0080047800680090009808900024
:103a4000010040008b00460009017800a4f3070044
:103a50001808900009004000100c980058089000c9
:103a600009005000200c98008000370070c6b30099
:103a7000804f55000300320070c4b300804f5500e2
:103a800014003a0058089000808f540004003d0054
:103a9000081090000038a30001003a00590c98006b
:103aa000580890000000e900500c980002003b000c
:103ab0000000eb00500c980070c6b300804f55001a
:103ac00002003a005ac6b3000b0037005ac4b300d4
:103ad0000900370010c6b300804f550002003a00bd
:103ae0000ac7b3000400370010c4b300804f55006c
:103af00001003a000ac5b300180990006800900060
:103b00003c7178008201e800130c98000c027800e8
:103b1000580890000000e00003003c0008109000ee
:103b20000038a30017003200e8009000e0c2b300a4
:103b300080f178008280e800110c9800580890000d
:103b40000000e0000f0034008904e900890f5000f4
:103b500001003d00800478006800900001004000f2
:103b600009017800840078005df3070018089000d0
:103b700009004000100c98005808900009005000ff
:103b8000200c980068009000980890000100400008
:103b90000086e8000a587800800078000d00e000f8
:103ba00004003500b0c2b300804878008c0478006f
:103bb00004003700d0c2b300804878008c0478003d
:103bc0008d06ea008005eb00788757000600370075
:103bd000a10020000d007800b5000700015f78000b
:103be0008b05e800800678000d00e000f8ff3c003f
:103bf000e18f550009003c0050c6b300804f5500ce
:103c00000300320050c4b300804f550003003a0057
:103c100000c3b300005e78008c0478000b00e00065
:103c2000040032000b00e900f880570000804000db
:103c30000700370000c3b300805c7800060037003f
:103c40008b05e90001c3b30090dc40000000e900ef
:103c50000b00e000faff3c0068009000980890001c
:103c60000100400000805400300c980008109000c3
:103c700074006000f00f50000e003a0078009000d1
:103c80009808900001004000a80890000100400042
:103c9000b808900001004000c80890008100400072
:103ca00078089000808f500002003d000100500015
:103cb000000c98004f0778004f06be004f05be006d
:103cc0004f04be00cf00b10000000600881f78003e
:103cd00000027800e602400015007800010028008c
:103ce000810360006f006000800a780012003a00d3
:103cf000240090000000e0000f003a001400900043
:103d00000000e0000c003a00160020001400e00063
:103d10006300320008003700e4004200910a780096
:103d20000480e8009008780014087800020a7800ff
:103d300070035300010037001600200015017800c1
:103d40001500e000f4ff3200130037006401420068
:103d500080004000120078004f00de00808a700072
:103d60008480e80012007800800140001100780093
:103d70004f00de000089710091017800038141004d
:103d8000140078004f00de008008710014047800f1
:103d9000080a44000603e90015007800ef0f500000
:103da000eaff36003a0037000481e8009400d100b1
:103db00092017800038041000000400000004000b4
:103dc00000004000000040000000400000004000f3
:103dd00000004000000040000000400000004000e3
:103de00000004000000040000000400000004000d3
:103df000008a7000e40042008301d10011047800c1
:103e000008004400000040000000400000004000a6
:103e100000004000000040000000400000004000a2
:103e20000000400000004000000040000000400092
:103e300000004000000040000000400000897100c8
:103e40001101d1009501780003804100000040007d
:103e50000000400000004000000040000000400062
:103e60000000400000004000000040000000400052
:103e70000000400000004000000040000000400042
:103e80000000400080087100950ad1000603e80098
:103e900015007800ff0f5000c3ff3e00ef0a6000de
:103ea000958a7300060078004f0478000000060031
:103eb00001017800801f7800110009000200d8007d
:103ec000800078004f0078000191b9008202500014
:103ed000010278000400be00000006000c02e200af
:103ee00004003d000f42ab00020032000f02ab00a5
:103ef000feff32000040da00feff3700889fbe0060
:103f000080047800109180000000e00003003a0077
:103f1000100007000000e0000a003500109180004a
:103f20000900e00002003a000004780006003700b3
:103f30000004780009004000060007000000e000cf
:103f400001003d000084eb00080078004f04be0033
:103f500000000600800078000000e00004003a0045
:103f6000c059220010918800010178000600370036
:103f70000081eb00e05c2200808f500002003e00d8
:103f8000119188000001eb0002007800000006009b
:103f9000889fbe008a9fbe00010578000100e000f6
:103fa0000400350008003c000000e0002000320062
:103fb0000500370060001000e080180002003b00a0
:103fc00001f02c001a0037000004be006011b80098
:103fd0006b0920000982cf00020039000882cf005f
:103fe0000441b000694252000e00320008003b005c
:103ff00082817100610164008904d1000884d300ca
:104000008b05e8000442e800f9ff3a00050037009c
:104010000804440089844c008b05e9000442e9004f
:10402000fbff3a00b90307000af0a70001f0a00067
:104030004f05be004f04be0000000600889fbe0072
:104040008a9fbe008c1f7800d60307001002200054
:1040500002003b0090908800da0337008a0062007b
:104060006408e10002003a0090908800e203370003
:104070006108e100fcff32000800be000304780084
:104080000b00070001f0a100de03070008f0a60006
:10409000040037000001be0091042400b0fd2000a0
:1040a0007900070009f0a70001f0a200ce03370055
:1040b000889fbe008a9fbe008c1f7800b90307004e
:1040c000c003330003866c006450e1002e00320010
:1040d0006420e100330032006150e1002f00320023
:1040e0006120e1003100320085855500eb07b0000a
:1040f00009002000080420000500370008044400df
:1041000089844c000a0031000603430087834b007a
:104110000001530081815b00f8ff33000203be0001
:104120000800a0000804440089844c00f6ff390010
:10413000c639dd0083017300010032001300200046
:104140008904d1000884d3000998a3000500320037
:104150000800a7000300a0008904d1000884d30050
:104160008b05e8008904d1000884d3000001eb002e
:104170000281d2006503070001f0a1000cf0a70046
:1041800001f0a000980337006420e1009a03320098
:104190000801be000200be00f7ff37006120e10009
:1041a000950332006000b800f3ff370000002000e4
:1041b00001f82700f0ff3700889fbe008a9fbe00ed
:1041c0008c1f7800770307007e03330003866c00a2
:1041d0006450e100240032006420e1002700320036
:1041e0006150e100220032006120e1002100320034
:1041f0008b854200eb07b1000134b800003ab800eb
:104200000804420089844a00013ab8000030b8002e
:104210008880400009014a0004003300000040008b
:1042200081804800020149008b05e900c909dd00d1
:10423000830170000100320013002000c814de006a
:104240004814dd004709de001200b200c808de0095
:10425000088470002d03070001f0a1000cf0a700f6
:1042600001f0a000600337006120e100620332002a
:104270000801be000200be00f7ff37006150e100f8
:10428000fcff3a005c03370003f0a200889fbe00e9
:104290008a9fbe008c1f7800420307004903330049
:1042a0006450e1004f0032006420e100520032000f
:1042b00003826c0007003b000905d0000306d00014
:1042c000820f54000c065d0002003900020032002b
:1042d00089017800030678008582550004003d00be
:1042e0000003fd008103fd008502ea008b8542008a
:1042f000840f720002003b0060001000e080180094
:104300006011b8000005eb007a28e1000a003900ce
:1043100006007800c75ddd00f707b20087807500f2
:104320002d003700828171000a017800610560006c
:104330008180d1000080d3008502e900f9ff3b00b5
:10434000060440008784480002003b00600414001b
:10435000e0841c000988a300070032008a817100f4
:1043600082817100610164008904d1000884d30056
:104370008b05e800170037000978a30013003a0006
:104380000b00e000130034008b05e9000804440032
:1043900089844c000a4474000978a3000d003a0097
:1043a0000b00e000070034008b05e900080444001e
:1043b00089844c0001003a000b0020000978a3001a
:1043c000f7ff32000001eb0002003700828171002c
:1043d0000a017800cd0207000cf0a70001f0a00050
:1043e000010337006420e10002003a00838f6c0073
:1043f000010333000801be000200be00fa023700cc
:104400000001eb00640307000400320002002000fa
:1044100003f8230001f0a7009bff0700000006003f
:104420000001be00830307000470a70003f0a10091
:104430006509b100160032000d0035006828e10062
:1044400006003500f0ff2f00f1ff27000300e00019
:1044500013003b00010028000000050000004000a0
:10446000818048008502e900fcff3a00080037001f
:10447000f88f420002003c008000eb0000000500c5
:104480008100d1000080d3008502e800fcff3a00e3
:104490000300e00002003b0060001000e080180014
:1044a000000006001400200077033700f4ff2f00ff
:1044b000750337000001eb008e033700839f68000f
:1044c0000100e00002003d0060001000e0801800e4
:1044d0000300e00002003d0060011100e0811900ce
:1044e0000b0007004f00e00002003b0060001000de
:1044f000e080180000000600020ab900001bb900a5
:104500000200b80081004200810043000000060064
:104510006022b800060220000000d0008180d20096
:104520000482d2008582d2000000a0000202520064
:1045300083825a0003003b000202420083824a0049
:104540000000a1000603e900f3ff3a0000000600a6
:1045500081037800370307000001be006000b80047
:104560000478a30013003a006220e10015003e0029
:104570000d0039008301d1000281d3008180d30076
:104580008301d1000281d3008180d3008301d10057
:104590000281d3008180d3000538b000c42add0039
:1045a000f300b2008381720007f0a70003f0a000bf
:1045b00000000600f3ff2700f2ff2f006110b90092
:1045c000fbff370003ff2700f7ff3700881f780045
:1045d000000478005001be004000be000000420010
:1045e00081804a0002014b0083814b00009cbe0089
:1045f0000294be000400e1000588e1000690e1009d
:104600000798e10002003100680044001008e8004b
:104610004f04780000000600f4874700889fbe0022
:104620008a9fbe008c9fbe008e1f78000205be00d0
:104630000004be00d4b79f00e5b79f00f6b79f0007
:1046400087bf9f000000eb00c0b79f00b0b79f007e
:10465000a0b79f0090b79f0080b79f000d04200077
:10466000bfb097004fb09700000140000000e0008d
:1046700014003d004f08de0000007100c0b79f002d
:10468000ad00070001003d0012002000b00007004f
:1046900001003d0012002000b500070001003d00b0
:1046a00012002000ba000700be000700feff3a001b
:1046b000c2000700c80007000f004000c3ff07004a
:1046c000270037004f08de0000067100ccb79f00be
:1046d0009900070001003d00120020009c00070027
:1046e00001003d0012002000a100070001003d0074
:1046f00012002000a6000700aa000700feff3a00f3
:10470000ae0007000fb297009fb297002fb397003b
:10471000bfb39700b60007000000520081805a0026
:1047200002015b0083815b0080b79f0091b79f000f
:10473000a2b79f00b3b79f000007eb00ac000700d3
:104740000020e10001a8e10002b0e10003b8e100af
:10475000010031001e0020000e005600c0b79f006f
:104760004fb297000400e000070035001000200061
:10477000010020006011b8000804700089847000f6
:104780000a0571008b8571008d06e900b4ff3a00bf
:104790000400e00003003d008f0007000f00400010
:1047a0008aff07004fa897000000e00004003a00cd
:1047b0000fb497009fb497002fb59700bfb597002f
:1047c000970007004f0778004f06be004f05be0058
:1047d0004f04be004f01b10000000600881f7800a2
:1047e00018002000881f78008bff07008f87e900e2
:1047f0004f04780000000600801feb0086ff0700d2
:104800008f87e90000000600889fbe008a9fbe00d7
:104810008c1f78007b00070005003d002f0007007b
:1048200007003d003d0007000006eb0004003700d4
:104830003f00070002003d00300007001c00200080
:1048400077000700e5ff07000203be000002be007c
:104850000c00e00001003200280007000400be0048
:104860000601be004f0678004f05be004f04be0093
:1048700000000600889fbe008a9fbe008c1f780043
:104880006000070003003d001400070006003d0023
:10489000040037002600070003003d006000b80058
:1048a0006011b8001d0007005d000700d2ff07007f
:1048b0000203be000002be000c00e0000100320056
:1048c0000e0007000400be000601be004f0678007f
:1048d0004f05be004f04be00000006006000b80097
:1048e0006011b80008045000898458000a05590076
:1048f0008b8559001c002000030037006000b800c1
:104900006011b80005003700e00f5200e08f5a0038
:10491000e00f5b00e08f5b00000006000402500027
:10492000858258000603590087835900000006005d
:104930000006eb00f4ff37000180400090b79f00b5
:104940000001eb008fb097000100e00000000600be
:104950000200700090b79f000180400080b79f0068
:104960000001eb00ffa897000100e0000000060036
:104970000200700080b79f0001804000f0af9f00f0
:104980000001eb00efa897000100e0000000060026
:1049900002007000f0af9f0001824000200007007d
:1049a000f50305008301d1000281d3008180d3008b
:1049b0000080d3008502e9000000060000027200ba
:1049c000e4af9f000804440089844c000a054d00b0
:1049d0008b854d00000006003fb29700cfb29700d4
:1049e0005fb39700efb3970000fe2f0000000600b2
:1049f0003fb09700cfb097005fb19700efb197003d
:104a0000000006000205be000004be00e00f5000da
:104a1000e08f5800e00f5900e08f590000000600b9
:104a20000800be000a01be0000000600889fbe000c
:104a30008a9fbe008c1f78000205be000004be00e5
:104a40000006eb00e00f5000e08f5800e00f590027
:104a5000e08f590007003d006000b8006011b80009
:104a600008045000898458000a0559008b855900b4
:104a70001c002000e00f5200e08f5a00e00f5b00a6
:104a8000e08f5b0002003d000f0007000c00a20059
:104a90000800be000a01be007d0207000203be003e
:104aa0000002be000c00e00001003200060007001a
:104ab0000400be000601be004f0678004f05be0090
:104ac0004f04be00000006006000b8006011b8008e
:104ad000040250008582580006035900878359005c
:104ae000000006008f1fd1008b0207008f87e900ae
:104af0000000e000000006001400fa00889fbe00dd
:104b00008a9fbe008c9fbe000004be000205be004e
:104b1000680047000a90be000890be00a702070088
:104b20000070a7000bf0a100304320009e0290000f
:104b300080825200b0fe2f000028e10011003d00ed
:104b4000b0fc2f000028e100150034001e09900081
:104b50008e0890007e0090000501b0000201d10097
:104b60008180d3000080d3008502e800fbff3a007b
:104b70000b00e000cc023b0060001000e080180059
:104b8000c9023700f0ff2f00f1ff27000b00e00003
:104b9000c5023b000100280000002000c2023700cf
:104ba0006000b800c00237004f89de008201780043
:104bb000c202370007f0a200f7023700809feb0027
:104bc000550207008f87e9000000e00000000600a2
:104bd0002800fa00889fbe008a9fbe008c9fbe00fe
:104be00003866b009c0207000028a30064003a00c3
:104bf0000128a30067003a000008a30062003a0001
:104c00000108a30065003a001e009000be08900055
:104c100081064000ed3fb100f4805700ee019000a6
:104c2000111ab8008e099000311bb8009e0990003f
:104c3000311cb800511db800f4855700460007002c
:104c4000fe0190003a0007008b85e8003e00070057
:104c50008e09900040000700ee019000340007002c
:104c60008b85e800380007008e099000400007009f
:104c70009e0990001b18b800890440000a8548006e
:104c8000fe019000340007008b85e8003800070023
:104c9000ee019000300007008e0990001b18b8004c
:104ca000890440000a8548000a98a30008003a00d9
:104cb0000402420085824a0006034b0087834b00b2
:104cc00008044c0089844c000a054d008d06e9005b
:104cd00084827200850273004c3add008502720006
:104ce0000100320015002000443ade001400b2003a
:104cf0004538de00cb45dd000b007000c540de000e
:104d0000cb4ddd008b8070004549de00cb55dd00ca
:104d10000b017100c551de000d0378001b03070075
:104d200003f0a1000cf0a70003f0a0005e02370022
:104d30001b18b8008502400006834800e0834b0042
:104d400060044c00070037001b18b8000603400041
:104d500087834800faff37001b18b800870340001c
:104d600008844800e0844c0060054d000000060007
:104d70001b18b8000804400089844800faff370077
:104d80000108a30045023a005800be005801be00c9
:104d9000e3ff37000008a30040023a00090478004e
:104da000f9ff37002800fa00889fbe008a9fbe00e6
:104db0008c9fbe0003866b00270207006400e100a1
:104dc000440032006408e1004a0032006100e10062
:104dd000460032006108e10049003200ec0647005d
:104de0006000b8003d02be003d03be00f4865700df
:104df0006011b8003d04be003d05be007d032000eb
:104e00000b0037000000a0008d06e90013003200ff
:104e10000402420085824a0006034b0087834b0050
:104e20000000400081804800020149008381490060
:104e30000802520089825a000a035b008b835b00e0
:104e4000f0ff3b000802420089824a000a034b003f
:104e50008b834b008d06e900edff3a0084827200df
:104e600086827200f707b20087827200010032006a
:104e7000150020001e0490003e0b90000603540015
:104e8000e63fb0000368a300070032000000a7005f
:104e90000500a0008301d1000281d3008180d300ee
:104ea0000080d3000603e8008301d1000281d30013
:104eb0008180d3000080d3000002eb000482d20086
:104ec000b202070003f0a1000cf0a70003f0a0005d
:104ed000f5013700640247006408e100ef01320089
:104ee0003400be003401be00f6ff37006108e10067
:104ef000ea0132006011b8006000b800f1ff37002d
:104f000003ff270002002000fbff37008100200084
:104f1000618055000b003d000b00200061fe2f005a
:104f20000100e1001d003400828171006101640014
:104f30008904d1000884d3000000e800faff3a0099
:104f40007100200061006400030070000200600036
:104f50000900320061044400e0844c000988a50087
:104f6000050032008b05e8006808e10002003a0005
:104f70008904d1000884d300f20f20000258e10018
:104f800005003d00c75ddd00f907b20089807500ae
:104f900008007800000006000bf827008b0078005e
:104fa000000005000004be00a20007000003be00d0
:104fb0000405be000200be009e000700844f75007d
:104fc000000006000200be006450e100050036004b
:104fd0006420e100020036000968a30001003a00e5
:104fe0000800be000160a0004f0678004f05be001b
:104ff0004f04be0000000600f0ff2f00f1ff270065
:10500000f9ff3700889fbe008a9fbe008c9fbe00bc
:105010000004be00870007000800be008906780073
:105020006420e10008003900040032000160a000a3
:1050300012022000929088005300370091fc230058
:10504000b0fd20004e0037000006eb0009f0a10083
:1050500003f82300020020000800be0011fd070035
:105060000600340001f82300000020000801be0003
:105070000ffc07000004be002c0020000800be004a
:1050800093e82300320a230006fd070012003400d3
:105090000801be00d1fd2300703d2b007bfc070002
:1050a0000005be00b3f32300f27a26000800be001c
:1050b00041fc070003f823000200200072fc0700f7
:1050c0000801be0071fc07000a01be00f8fb0700e2
:1050d0000004be000c06e8000800be0001f0a100bc
:1050e0000200200003982300eefc07000800be0029
:1050f000160035000801be002ffc07000005be00a9
:1051000032cd2c0043fb230060fc0700809fbe00d3
:105110001269280003d52b000a00be0026fc0700f8
:10512000620f210013ef2b0058fc07000a01be009c
:1051300021fc07004f01be00ddfb07000801be0097
:105140001dfc07000801be0050fc07000c00e00039
:105150000b0032000c10a70001f0a200b2fd2000ed
:1051600093fc23006260e1000400320022a92000c9
:1051700063f023000c10a70063f8230043fc070032
:105180000df0a70001f0a2004f06be004f05be00c3
:105190004f04be0000000600889fbe008a9fbe002c
:1051a0000003be00230007008505780082815200bd
:1051b000020020006220e10004003a00f307b10081
:1051c000040035007718e100040035000600be0039
:1051d000140037006000b8000f003700f50f200002
:1051e000faff2f008502d1000a85d3008301e90070
:1051f000fcff3b008184620000046500890f74009d
:10520000f2ff32008582ea000a85ea0081846200aa
:10521000000465003dff070007f0a70001f0a000b3
:105220000081eb000200e0004f05be004f04be000d
:1052300000000600c70ade00f107b200f50fb20059
:1052400008003200e1cf4200020032000170a000ed
:1052500024000500810f70000100320004080500e1
:1052600044000500810f700002003a0014000500a0
:105270008502e9000000400081c04800fcff3b00bf
:105280000170a00024000500889fbe008a9fbe0018
:10529000841f780043ff07004f007800110033009f
:1052a000f0ff2f00838f6c0006003b0004056500b3
:1052b0000a00a7000800370009f0a600100020002f
:1052c00008003700820f5400838f5c000300390010
:1052d0001000200001003e000000200009f0a7009f
:1052e0000000ea004f05be004f04be000000e000d1
:1052f00000000600889fbe008a9fbe008c9fbe00f3
:105300000206780001f0a7000cf0a0000004be0027
:10531000c8ff07000800be006420e1000700390054
:1053200002003a00f1ff2700f0ff2f000160a0000b
:1053300012022000929088005100370009f0a1006d
:105340000800be000200200003f8230057fc0700fd
:10535000f4ff3c000800be00020020000398230078
:1053600050fc07000800be0030003500020020009d
:1053700003f023004dfc070005003c000800be00c0
:105380000801be008cfb07000005be000e003700c0
:105390000c10a2000000200001f823000801be004c
:1053a000b9fb07000200200003f0230082fb070086
:1053b0000005be00a10107000200200003002c0030
:1053c0007dfb07000004be000a00be00b2d028002a
:1053d000130b2c00adfb07000a01be0076fb070093
:1053e000020f2500330b2400a8fb0700809fbe009e
:1053f0000a00be005206220013f02b006efb0700cd
:10540000b2662100f3f62300a0fb07000a01be00ec
:1054100069fb07004f01be0025fb07000801be0025
:1054200065fb07000801be0098fb07000c00a70001
:1054300007003700b2fd200093fc23000c10a700ea
:1054400092fb07000cf0a70001f0a2000c0037004f
:105450000cf0a7000200370001f0a20004003700a2
:10546000b2fd2000930424000c10a60003003700b6
:10547000b2fd200093fc23000c10a70083fb070063
:105480004f06be004f05be004f04be0000000600e0
:10549000889fbe008a9fbe008c9fbe000404b80097
:1054a0000506b8008904460060854e000606b8006f
:1054b0000a054600e0854e000706b8008b05460049
:1054c000040eb800890446000a854e00e0854d00b0
:1054d000050eb8000a0546008b854e00060eb80082
:1054e0008b0546000416b8000a0546008b854e0061
:1054f0000516b8008b054600041eb8008b05460053
:105500000800be000a01be004f06be004f05be00e7
:105510004f04be0000000600889fbe008a9fbe00a8
:105520008c9fbe000404be000605be00809fbe0026
:10553000829fbe0076010700040678000800be00c6
:105540000a01be0072010700840678004f03be0006
:105550004f02be008d4f76007fb0970013003300de
:10556000f0ff2f008b8f6b0006003b000d066600de
:105570000c00a7000a00370007f0a600100020006a
:105580000a003700880f5200898f5a008a0f5b008b
:105590008b8f5b00030039001000200001003e00eb
:1055a0000000200007f0a7000000ea004f06be0040
:1055b0004f05be004f04be000000060080007800ca
:1055c0005002be005003be004439de00f700b200b6
:1055d000f37f200003016100090032000218e1009e
:1055e00016003a0085017200830173008381730005
:1055f0000008200015003a0040002000130037008a
:1056000085017200830173008381730005003a00f5
:1056100004a8be0006a8be00100020000b00370042
:105620000201e9000402420085824a0006034b00a1
:1056300087834b000748a300f9ff32000740a00012
:1056400004a8be0006a8be0020002000800098002c
:105650009200980000000600680447000294be0013
:105660000094be00fc0447008694be008494be00f3
:1056700009007800d1ff070008007800cfff07007d
:1056800099007800814f70000b003b000800be00bd
:10569000310107004f00b10003003700f3ff27007e
:1056a000f2ff2f006110b9004f06be004f05be008b
:1056b0004f04be000080fa0000000600889fbe0074
:1056c000830478000300e0002c00350003003c0058
:1056d0000082700004027100260032003643200070
:1056e000c50020008383cf000a0039000541b100c6
:1056f0008283cf00070039000541b1008183cf00cc
:10570000040039000541b1008083cf000100390059
:105710000541b10085c353006022b8001200320079
:105720000a003b0084827200610260008301d100a4
:105730000281d3008180d3000080d3000603e800fb
:105740008743e800f7ff3a000700370000004000f9
:105750008180480002014900838149000603e90075
:105760008743e900f9ff3a008800070009f0a70025
:1057700003f0a0004f04be0000000600600010000f
:10578000e080180060011900e0811900d3ff3b00a0
:10579000033e2c00f7ff37002800fa00889fbe0068
:1057a0008a9fbe008c9fbe0007067800878669002e
:1057b0000c003b00030478008704780008f0a10087
:1057c00009f0a100840f5000858f5800860f590002
:1057d000890f5c00030033000cf0a20001003a00c6
:1057e0000cf0a1009cff07006400e1005f003200a4
:1057f000780147006408e100610032006c01470055
:10580000748557003200be001201be003a04be008b
:105810001a05be001e039000be0a900085035300c7
:1058200006003d000004fd008104fd000205fd00ae
:105830008305fd008703ea00050378000df8a30047
:105840000400320060041400e0841c0060051d00a8
:10585000e0851d006022b8007d0320000d38e100c6
:105860008006eb000b0039004433dd00f300b2008a
:105870008301730039003700848272000d027800c2
:10588000e10664008b85d1000a85d3008984d300aa
:105890000884d3008703e900f7ff3b0008004000bd
:1058a000898048000a0149008b81490004003b00bf
:1058b00060001000e080180060011900e08119000c
:1058c0000358a300090032008d82720084827200a6
:1058d000610260008301d1000281d3008180d30086
:1058e0000080d3000603e8001b0037000348a30034
:1058f00017003a000600e000170034000603e90034
:105900000d00a3000000480081804800020149000a
:10591000838149000348a3000f003a000600e0001d
:10592000090034000603e9000000400081804800bf
:10593000020149008381490001003a000003eb00a5
:105940000348a300f5ff32006022b80002003700d0
:1059500084827200618266000c00070003f0a100df
:105960000cf0a70003f0a0004fff370064014700d0
:105970006408e10002003a000df8a30047ff3a0076
:105980003200be001201be0047ff370018002000a1
:1059900057002000080453000d003d0006002000c1
:1059a00097fc2f000740e1001e0034008482720043
:1059b000610260008301d1000281d3008180d300a5
:1059c0000080d3000804e800f8ff3a0047002000f8
:1059d0006104600005047400040464000d003200da
:1059e00061004000e080480060014900e08149001a
:1059f00003b8a500070032000603e8006538e1009f
:105a000004003a008301d1000281d3008180d300d9
:105a10000080d300f87f20000830e100030035004b
:105a2000080378006000b8006011b8004433dd005e
:105a3000f300b2008301730000000600889fbe00df
:105a40008a9fbe008c1f78000004be00f9fd07008d
:105a50000478a30026003a006120e100250032000e
:105a600009f8a30025003a006420e100210032007b
:105a7000f507b1000508a300020032000000400055
:105a8000818048006044b80003102000020020001c
:105a900000004000818048000805440089854c00d2
:105aa0000a0541008b8549000a0550008b85580086
:105ab000030033000a00be000204740083847400f3
:105ac0008301d1000281d300830f7100f0ff3a00ff
:105ad0008904d1000884d300600149008201780064
:105ae000c1adde00fb07b00008fd07003efd37003a
:105af0000960a0000800be003bfd37001202200034
:105b000092908800f0ff2f00f1ff270036fd37004c
:105b100005ff270005826100070032000428e1002c
:105b200001003200240005000600070001003a00d1
:105b3000440005000408050002000700f9ff3a00d0
:105b4000140005006f8261008102700085027100ff
:105b50008502720000000600e48240001078a30075
:105b600007003200640240001178a3003400be0038
:105b70001401be00040032000330a700000006003c
:105b80003500be001501be000330a0000000060075
:105b900004002000bcfd37006000fa00889fbe00b2
:105ba0008a9fbe000040eb00304798000040eb00a9
:105bb000007f98000040eb00107f98000040eb0051
:105bc000207f9800772c0700802607002d2d0700e6
:105bd00040c7bf000080fb00610060000000e000e3
:105be000020032004007a9000000fe000080eb0028
:105bf000402798000000eb00502798008204200006
:105c00000e01410013002000e1ff2f00f0072000eb
:105c1000e812070050279800100020000017980095
:105c200080022000101798008002200020179800a2
:105c300080002000301798009e1090002e109000d9
:105c40000088b9000000d00040179800f01c070041
:105c5000ae1090003e109000008db9009e10900094
:105c60003e109000008cb900ae1090003e109000e5
:105c70000088b900021e2000000051002200200010
:105c8000110009000200d8008003780001007800ac
:105c90009e1090003e1090000088b900022820005d
:105ca0000000510022002000110009000200d8006d
:105cb0000e139000be1290003e1290008a017800f0
:105cc0000801780087007800861c0700110020007a
:105cd00010002000af1c0700c51c07008105200034
:105ce000806c2900382e0700432e07000000e000da
:105cf000fdff3a006c2f07000e007800022e07000f
:105d00000000e0006a003a00782d0700007f98004c
:105d1000712d0700107f98001e7890000004e000ad
:105d2000030032001e789000e84f5000f2ff3a0066
:105d30008e7890002e78900080cf5000eeff3200d9
:105d40000e7890000001fb00cf91de00022f98003a
:105d5000132f980090002000010020000e299000d1
:105d60009e299000800f5100818f590045003e0010
:105d70000e2890009e289000006001003600370039
:105d8000080037000c0037001000370014003700ff
:105d9000180037001c0037002000370024003700af
:105da000280037008025200050079800c0122000ee
:105db00060079800370037008025200050079800c2
:105dc000802520006007980032003700c0122000b4
:105dd0005007980080252000600798002d003700ac
:105de000802520005007980080da2f006007980077
:105df000280037000000eb00500798000000eb007f
:105e0000600798002300370080da2f0050079800c1
:105e100080252000600798001e00370080da2f00e0
:105e20005007980040ed2f006007980019003700d8
:105e300080da2f005007980080da2f006007980062
:105e40001400370040ed2f005007980080da2f0033
:105e5000600798000f003700805922001004e0000e
:105e600004003a00a52307008159220010c0b300a6
:105e70008048780001f5210040b12200ac230700e2
:105e8000040037000000eb00600798000000eb0002
:105e9000500798008e789000217f98006e00900047
:105ea000c92b07005e009000042c070092ff37000a
:105eb0001e04e000bd023d000000eb00200798003a
:105ec0001e00fb000000ea006101b900f0fb2f009a
:105ed000f1ff2f000201400083814800322f98001b
:105ee000432f980040032000010020003e2990002d
:105ef000ce299000800f5100818f590092023e0000
:105f00003e289000ce289000006001007d00370000
:105f10008d0237008c023700100137003501370041
:105f20008902370088023700870237005a0137009c
:105f3000850237008402370080013700ac0137004a
:105f4000bd013700dc0137007f023700fa0137005e
:105f50007d0237007c0237007b0237006902370080
:105f6000790237007802370077023700760237006f
:105f7000750237007402370073023700720237006f
:105f800071023700700237006f02370014003700cb
:105f90006d0237006c0237006b0237006a0237006f
:105fa000690237006802370067023700660237006f
:105fb000650237006402370063023700620237006f
:105fc00061023700600237005f0237005e0237006f
:105fd0005d0237005c0237005b02370003023700c6
:105fe000110020000000eb000a2e0700300f98007f
:105ff0001100200010002000062e0700400f98001e
:106000001100200020002000022e0700500f9800f1
:1060100042222100640247009400780001007800c9
:106020008201400000c1eb006e5090008249600088
:106030008100e800010a780042222100e4014700c3
:106040009300780001007800020140003e089000b3
:106050004880de00004978008100e800810978006e
:106060004222210064024700940078000100780079
:106070008201400000c1eb000e5890008249600090
:106080008100e800010a780042222100e401470073
:106090009300780001007800020140004e08900053
:1060a0004880de00004978008100e800810978001e
:1060b0004222210064024700940078000100780029
:1060c0008201400000c1eb002e5890008249600020
:1060d0008100e800010a780042222100e401470023
:1060e0009300780001007800020140005e089000f3
:1060f0004880de00004978008100e80081097800ce
:1061000011023700c00320000e004000772e070068
:10611000c00320000e004000001f98004222210012
:10612000e40147009300780001007800020140007c
:106130000e189000104978008100e800810978006d
:106140000e1890000000e800001f98004222210075
:10615000e40147009300780001007800020140004c
:106160000e189000104978008100e800810978003d
:106170000e1890000000e800001f98004222210045
:10618000e40147009300780001007800020140001c
:106190000e189000104978008100e800810978000d
:1061a0000e1890000000e800001f98004222210015
:1061b000e4014700930078000100780002014000ec
:1061c0000e189000104978008100e80081097800dd
:1061d000c00320000e00400064004000001f980033
:1061e00042222100e401470093007800010078007a
:1061f000020140000e189000104978008100e8006c
:10620000810978000e1890000000e800001f980037
:1062100042222100e4014700930078000100780049
:10622000020140000e189000104978008100e8003b
:10623000810978000e1890000000e800001f980007
:1062400042222100e4014700930078000100780019
:10625000020140000e189000104978008100e8000b
:10626000810978000e1890000000e800001f9800d7
:1062700042222100e40147009300780001007800e9
:10628000020140000e189000104978008100e800db
:1062900081097800c00320000e0040006800400023
:1062a000001f980042222100e4014700930078007b
:1062b00001007800020140000e189000104978009b
:1062c0008100e800810978000e1890000000e800c5
:1062d000001f980042222100e4014700930078004b
:1062e00001007800020140000e189000104978006b
:1062f0008100e800810978000e1890000000e80095
:10630000001f980042222100e4014700930078001a
:1063100001007800020140000e189000104978003a
:106320008100e800810978000e1890000000e80064
:10633000001f980042222100e401470093007800ea
:1063400001007800020140000e189000104978000a
:106350008100e800810978007b013700000000001f
:106360000e00e800682c07000000e000fcff32008f
:10637000000000000e80e800632c07000000e00031
:10638000fcff32001e4090008080fb002e409000f9
:106390000000fb004800dd0000804000600798001e
:1063a0000e00e800582c07000000e000fcff32005f
:1063b000000000000e80e800532c07000000e00001
:1063c000fcff32001e4090008080fb002e409000b9
:1063d0000000fb004800dd000080400050079800ee
:1063e0006e009000782a07005e009000b32a070034
:1063f00055013700422221006402470094007800d2
:10640000010078008201400000c1eb004e4890007e
:10641000824960008100e800010a780042222100e0
:10642000e401470093007800010078000201400079
:106430006e0090004880de00004978008100e8008e
:10644000810978004222210064024700940078000c
:10645000010078008201400000c1eb002e4890004e
:10646000824960008100e800010a78004222210090
:10647000e401470093007800010078000201400029
:106480005e0090004880de00004978008100e8004e
:10649000810978002c0137002e0090007122210024
:1064a000010040000021070010c0b30030479800f1
:1064b0004222210064024700940078000100780025
:1064c0008201400000c1eb000e6090008249600034
:1064d0008100e800010a780042222100640247009e
:1064e00094007800010078008201400000c1eb00b8
:1064f0002e609000824960008100e800010a780067
:1065000042222100640247009400780001007800d4
:106510008201400000c1eb004e60900082496000a3
:106520008100e800010a7800ae0090004e10900053
:1065300000804000200798000301370000000000a1
:106540000e00e800f02b07000000e000fcff320026
:10655000000000000e80e800eb2b07000000e000c8
:10656000fcff32001e4090000000fb00202f98002e
:106570002e299000e90f51000f003200ae29900043
:10658000e98f510004003c002e289000e80f5000d5
:106590000500320010003700ae289000ea8f50004e
:1065a000090032000c0037002e4090000000fb0074
:1065b000d8260700e40037002e4090000000fb00c2
:1065c000f3260700e00037002e4090000000fb009b
:1065d000d0260700dc0037002e4090008000fb0032
:1065e0001e4090000000fb0070250700d600370019
:1065f0000000eb00300798003e009000e50f5000cf
:10660000d1003c0042222100e401470093007800c1
:1066100001007800020140000040eb0000497800d2
:106620008100e800810978003e0090000000e80049
:1066300030079800f0ff37000000eb0030079800ab
:106640003e009000e70f5000bf003c003e0090006d
:10665000ee2e070040079800422221006402470006
:1066600094007800010078008201400000c1eb0036
:106670000e489000824960008100e800010a78001d
:1066800042222100e40147009300780001007800d5
:10669000020140004e0090004880de000049780072
:1066a0008100e800810978003e0090000000e800c9
:1066b00030079800e2ff37000000eb003007980039
:1066c0003e009000e70f50009f003c003e0090000d
:1066d000f12e070040079800422221006402470083
:1066e00094007800010078008201400000c1eb00b6
:1066f0000e489000824960008100e800010a78009d
:1067000042222100e4014700930078000100780054
:10671000020140004e0090004880de0000497800f1
:106720008100e800810978003e0090000000e80048
:1067300030079800e2ff37003e2a07004007980024
:106740004222210064024700940078000100780092
:106750008201400000c1eb000e48900082496000b9
:106760008100e800010a780042222100e40147008c
:106770009300780001007800020140004e00900074
:106780004880de00004978008100e8008109780037
:10679000322a070040079800422221006402470085
:1067a00094007800010078008201400000c1eb00f5
:1067b0000e489000824960008100e800010a7800dc
:1067c00042222100e4014700930078000100780094
:1067d000020140004e0090004880de000049780031
:1067e0008100e80081097800570037000000eb00c5
:1067f000082f07004007980042222100640247004a
:1068000094007800010078008201400000c1eb0094
:106810000e489000824960008100e800010a78007b
:1068200042222100e4014700930078000100780033
:10683000020140004e0090004880de0000497800d0
:106840008100e8008109780010002000f12e070087
:10685000400798004222210064024700940078001b
:10686000010078008201400000c1eb000e4890005a
:10687000824960008100e800010a7800422221007c
:10688000e401470093007800010078000201400015
:106890004e0090004880de00004978008100e8004a
:1068a0008109780020002000da2e070040079800b8
:1068b0004222210064024700940078000100780021
:1068c0008201400000c1eb000e4890008249600048
:1068d0008100e800010a780042222100e40147001b
:1068e0009300780001007800020140004e00900003
:1068f0004880de00004978008100e80081097800c6
:10690000110037006080200070179800812520005a
:106910007e1090002c2b0700127680004207980012
:1069200042222100640247009400780001007800b0
:106930008201400000c1eb000e48900082496000d7
:106940008100e800010a7800000000000e007800d5
:10695000ed2a07000000e000fcff32001e04e0000a
:1069600057fd3a002e0090000000e000e2fc3200eb
:106970003e4090000004e000050032000040eb00c3
:1069800030479800292007000000e000fdff32009a
:10699000ae009000402221000b2b0700162b0700b1
:1069a0000000e000fdff3a00d3fc37001e04e000c9
:1069b000d1fc3400a3c0b3009ecf1100030032000d
:1069c000d0c0b3009e4f100003003a000e007800c4
:1069d000cd2a0700f7ff3700402221001e4878002b
:1069e00010002000200798000e007800c62a07003b
:1069f0000000e0000800320042222100e4014700cc
:106a00001300780080007800828040009e48780063
:106a10000000e80080097800a1c0b3009ecf1000fc
:106a200003003200d2c0b3009e4f1100eeff3a00c7
:106a300042222100e4014700930078000100780021
:106a4000020140000040eb00004978008100e800ae
:106a50008109780048222100402221001000fb001b
:106a60003be60700004c78004022210010407800ef
:106a70000001fb00cf91de00f0fb2f00f1ff2f00a3
:106a80000201400083814800622f9800732f980014
:106a900090012000010020006e299000fe29900046
:106aa000800f5100818f590087033e006e289000af
:106ab000fe28900000600100190037003200370006
:106ac00041003700680037007b0037008c0037003a
:106ad0009b003700b10037004101370058013700f3
:106ae000c0013700f3013700050237000b02370001
:106af000300237005502370068023700790237004c
:106b0000800237008d023700cf023700e5023700e0
:106b1000fa0237006c0337001303370045033700d0
:106b200011002000200020003a2b0700801f780071
:106b30001100200010002000362b0700801f780075
:106b4000110020000000eb00322b0700801f7800ae
:106b500010722900801f78004022210025e60700de
:106b6000e88757004022210000e6070080007800f7
:106b700040222100942a07009f2a07000000e0001d
:106b8000fdff3a005cfc370074004700801f78006e
:106b9000e0722900801f78004022210006e60700ed
:106ba000e48757002e0890005a2507003100200086
:106bb00040732900842a07008f2a07000000e000a4
:106bc000fdff3a004cfc3700e7c2bf000080fb002d
:106bd0000000d1000080fb00610060008000d00058
:106be000e7c2bf000080fb00610060000080400041
:106bf0008000d000e6c2bf000080fb004700de003e
:106c00000080fb00008040008000d000e6c2bf0092
:106c10000080fb004600de000080fb006100600099
:106c200000804000600f9800ee089000811f7800ff
:106c300080732900801f780040222100ede50700c5
:106c4000e487570040222100c8e507008000780053
:106c5000402221005c2a0700672a07000000e000ac
:106c6000fdff3a0024fc37006a004700801f7800cf
:106c70006c004700801f7800f0732900801f7800a7
:106c800040222100cce50700e68757006e00900007
:106c90004d2807005e009000882807003100200082
:106ca00080742900482a0700532a07000000e000ea
:106cb000fdff3a0010fc37005e019000821f780053
:106cc000ee019000831f7800c0742900801f7800b7
:106cd00040222100c7e50700e68757004022210037
:106ce000a2e507008000780040222100362a070034
:106cf000412a07000000e000fdff3a00fefb3700dc
:106d000074004700801f780060752900801f78009c
:106d100040222100a8e50700e48757002e089000d4
:106d20001b25070031002000c0752900262a070016
:106d3000312a07000000e000fdff3a00eefb3700bb
:106d40006a2907000080fb00801f78006229070085
:106d50000080fb00801f78005a2907000080fb009c
:106d6000801f780000762900801f780040222100d3
:106d7000a0e50700e8875700402221007be50700d7
:106d800080007800402221000f2a07001a2a0700fd
:106d90000000e000fdff3a00d7fb370011002000a3
:106da00010792900082a0700132a07000000e000d4
:106db000fdff3a00b101200030792900022a0700c6
:106dc0000d2a07000000e000fdff3a00b10220009c
:106dd000f07a2900fc290700072a07000000e000dc
:106de000fdff3a00f1012000b07d2900f6290700df
:106df000012a07000000e000fdff3a0081022000a8
:106e0000b07f2900f0290700fb2907000000e000ff
:106e1000fdff3a008102200040822900ea29070094
:106e2000f52907000000e000fdff3a00c102200044
:106e3000d0842900e4290700ef2907000000e000c2
:106e4000fdff3a0091012000a0872900de290700fc
:106e5000e92907000000e000fdff3a00f1002000f2
:106e600040892900d8290700e32907000000e00035
:106e7000fdff3a0021022000408a2900d2290700a4
:106e8000dd2907000000e000fdff3a00d1042000ea
:106e9000708c2900cc290700d72907000000e000ea
:106ea000fdff3a009102200050912900c6290700f9
:106eb000d12907000000e000fdff3a00d1022000c8
:106ec000f0932900c0290700cb2907000000e0004b
:106ed000fdff3a0071012000d0962900ba29070071
:106ee000c52907000000e000fdff3a00b1012000c5
:106ef00050982900b4290700bf2907000000e000ce
:106f0000fdff3a00b1022000109a2900ae290700c7
:106f1000b92907000000e000fdff3a00b10220009f
:106f2000d09c2900a8290700b32907000000e00031
:106f3000fdff3a00a1012000909f2900a22907002f
:106f4000ad2907000000e000fdff3a00b10220007b
:106f500040a129009c290700a72907000000e000a4
:106f6000fdff3a00c102200000a429009629070075
:106f7000a12907000000e000fdff3a0061022000a7
:106f8000d0a62900902907009b2907000000e000f7
:106f9000fdff3a00f101200040a929008a290700dd
:106fa000952907000000e000fdff3a005102200093
:106fb00040ab2900842907008f2907000000e0006a
:106fc000fdff3a0041022000a0ad29007e29070004
:106fd000892907000000e000fdff3a0046fb37006a
:106fe0004e109000801f7800be109000811f780026
:106ff0002e119000821f78009e119000831f780050
:107000000e109000801f7800f0af2900801f7800dc
:1070100040222100f7e40700ec87570040222100be
:10702000d2e4070080007800402221006629070092
:10703000712907000000e000fdff3a002efb370039
:107040000080eb00501798000080eb00601798005c
:10705000c00220000e004000801f7800a002200027
:107060000e004000801f7800600220000e004000eb
:10707000801f7800400220000e004000801f780032
:10708000200220000e004000801f78000002200037
:107090000e004000801f780020b12900801f78007a
:1070a00040222100c4e40700ee8757000e10900034
:1070b0000000e00005003a009e1090002e109000a5
:1070c0000088b90040179800050037009e10900016
:1070d0002e1090000088b9000000d00040179800e2
:1070e000ce10900030002100808f50000b00340043
:1070f0001000200000179800800220001017980050
:1071000080022000201798009e1090002e10900002
:107110000088b9000000d00040179800bc17070095
:107120005e109000e10f400009003a009e109000b0
:107130003e1090000088b900022820000000510095
:1071400022002000110009000200d800501798000a
:107150006e109000e10f400009003a00ae10900060
:107160003e1090000088b900021e2000000051006f
:1071700022002000110009000200d80060179800ca
:10718000ae1090003e1090000089b9009e10900053
:107190003e1090000088b9000e139000be129000bf
:1071a0003e1290008201780000017800ee109000fd
:1071b0005e1090004b170700110020001000200007
:1071c000741707008a1707003100200070b22900e9
:1071d000fd280700082907000000e000fdff3a0035
:1071e000c5fa3700e1032000b0b22900f6280700f5
:1071f000012907000000e000fdff3a001100200017
:1072000080002000692207006000b8006027980015
:10721000712798006e219000fe219000f023240039
:10722000f1002000800f5100818f590007003c00c1
:107230006e209000fe20900061004000e080480039
:107240006027980071279800f2ff3700a6230700f7
:107250006000b80060279800712798006e219000a8
:10726000fe219000f070220001002000800f5100ec
:10727000818f590007003c006e209000fe20900096
:1072800061004000e0804800602798007127980066
:10729000f2ff37005f2b070091012000a0b6290004
:1072a000c9280700d42807000000e000fdff3a00cd
:1072b00091fa370074004700801f78007200470081
:1072c000801f780040b82900801f780040222100ec
:1072d00039e40700e6875700ae0890001e089000ca
:1072e0003222070031002000d0b82900b62807005c
:1072f000c12807000000e000fdff3a007efa3700d9
:107300009100200010b92900af280700ba28070013
:107310000000e000fdff3a0077fa3700700020001f
:10732000ba2b0700801f780060002000b72b0700f1
:10733000801f780050002000b42b0700801f7800c9
:1073400040002000b12b0700801f78003000200093
:10735000ae2b0700801f780020002000ab2b070019
:10736000801f780010002000a82b0700801f7800e5
:107370000000eb00a52b0700801f7800b0b92900a2
:10738000801f7800402221001ae40700f28757008e
:1073900040222100f5e30700800078004022210010
:1073a00089280700942807000000e000fdff3a004c
:1073b00051fa370070002000b72b0700801f7800bb
:1073c00060002000b42b0700801f780050002000d0
:1073d000b12b0700801f780040002000ae2b070073
:1073e000801f780030002000ab2b0700801f780042
:1073f00020002000a82b0700801f7800100020002c
:10740000a52b0700801f78000000eb00a22b0700cf
:10741000801f780070bb2900801f78004022210067
:10742000f4e30700f287570040222100cfe3070072
:107430008000780040222100632807006e280700a2
:107440000000e000fdff3a002bfa37006e00470015
:10745000801f780070004700801f780030bd290031
:10746000801f780040222100d3e30700e687570001
:107470000e089000f32607007e009000fb26070010
:1074800031002000c0bd29004f2807005a280700fe
:107490000000e000fdff3a0017fa3700ef26070072
:1074a000801f7800e3260700801f780000be2900b7
:1074b000801f780040222100cee30700e6875700b6
:1074c00040222100a9e3070080007800402221002b
:1074d0003d280700482807000000e000fdff3a00b3
:1074e00005fa370031002000a0be29003628070029
:1074f000412807000000e000fdff3a000000fe0008
:10750000fdf937000000eb002f2607000000eb001c
:107510006a2607008000eb0080002000a3210700fe
:1075200031002000e0be290027280700322807008c
:107530000000e000fdff3a00eff937007e00470051
:10754000801f780020bf2900801f78004022210082
:1075500099e30700e4875700805922001004e000f7
:1075600004003a00e51d07008159220010c0b30055
:1075700080487800fe089000512f98005e29900006
:10758000e30f510019003200de299000e38f510013
:1075900007003c005e289000e10f50000b00320015
:1075a000de289000e28f50000c0032001b003700f4
:1075b0005e299000e40f510010003200de29900097
:1075c000e58f5100110032001400370001842000c3
:1075d0000000eb00d61d070014003700016e2000ec
:1075e00040842000d21d07001000370041d5200044
:1075f00060f22000ce1d07000c00370041e920009a
:10760000e0c72100ca1d07000800370001f521006e
:1076100040b12200c61d070004003700ce1d070040
:10762000815922000040eb008048780031002000a2
:1076300070bf2900e4270700ef2707000000e000e3
:10764000fdff3a00acf9370020002000712b070045
:10765000801f7800100020006e2b0700801f78002c
:107660000000eb006b2b0700801f7800b0bf2900e3
:10767000801f7800402221005ee30700e887570062
:107680004022210039e307008000780040222100d9
:10769000cd270700d82707000000e000fdff3a00d3
:1076a00095f937006102200080c02900c627070035
:1076b000d12707000000e000fdff3a004e209000b7
:1076c000801f7800f0c22900801f7800402221002e
:1076d00048e30700e48757004022210023e3070026
:1076e0008000780040222100b7270700c22707004a
:1076f0000000e000fdff3a007ff937006003200042
:107700000e004000801f7800400320000e00400063
:10771000801f7800200320000e004000801f7800aa
:1077200000c42900801f78004022210022e30700c6
:10773000e8875700a91f07006e719000ce70900077
:107740002e709000e41f0700a81f070031002000e2
:10775000c0c429009c270700a72707000000e000fd
:10776000fdff3a0064f93700400320000e0040009e
:10777000801f7800200320000e004000801f78004a
:1077800000c52900801f7800402221000ae307007d
:10779000e6875700ae189000811f78001e199000f0
:1077a000821f780090c52900801f780040222100a8
:1077b00010e30700e687570040222100ebe20700b4
:1077c00080007800402221007f2707008a270700d9
:1077d0000000e000fdff3a00801f0700ce7090001f
:1077e0002e709000851f07000000fb00301f9800de
:1077f0007e1f0700be199000831f780030c6290045
:10780000801f780040222100fae20700e487570039
:1078100040222100d5e207008000780040222100ac
:1078200069270700742707000000e000fdff3a0009
:1078300031f937002000200030079800be0090008a
:10784000e00f2000808f50002bf93c00631f0700e1
:107850008040eb006e409000681f07000000fb00b6
:10786000301f9800611f07003e1890000000e000e4
:10787000110035003e189000801f7800be00900077
:10788000811f7800a0c62900801f780040222100b7
:10789000d8e20700e687570040222100b3e2070044
:1078a0008000780040222100472707005227070068
:1078b0000000e000fdff3a003e0090000080e8007c
:1078c00030079800ddff37005101200030c7290044
:1078d0003d270700482707000000e000fdff3a00b1
:1078e00005f937000400fa0085260700aa1f0700e3
:1078f0002c250700c72607000040eb00322b0700ad
:1079000040c7bf000080fb00610060000000e00095
:10791000020032004007a9000000fe007d0b0700b6
:10792000000f78001e007800801f7800a0c8290092
:10793000801f780040222100aee20700e487570054
:107940004022210089e207008000780040222100c7
:107950001d2707001e00e00002003a00a7000700f4
:1079600046003700100020009e0f100002003a0071
:107970005806070041003700200020009e0f10002d
:1079800002003a005e0a07003c0037003000200089
:107990009e0f100002003a007ff807003700370002
:1079a000500020009e0f100002003a00c40707009c
:1079b00032003700600020009e0f100002003a00e5
:1079c000e20607002d003700700020009e0f100017
:1079d00002003a00080b0700280037008000200052
:1079e0009e0f100002003a00e30207002300370058
:1079f000d00020009e0f100015003a009c260700c2
:107a00004022210059e20700800078004022210036
:107a10003b2707000e80e800bb2607000000e000bf
:107a2000030032000e80e800110020003427070018
:107a30000e80e800022707000000e000f5ff32009a
:107a40000e80e80011002000df260700f1ff37005c
:107a5000e00020009e0f100002003a00aa0207007a
:107a600006003700f00020009e0f100002003a00d0
:107a70005e08070001003700b102070000000000a7
:107a8000ffff37001400fa006000b80040079800bc
:107a9000510798006000b8006007980071079800cf
:107aa0006000b800000f9800110f98000000eb0074
:107ab000000f7800f00120009e0f100036003c00ff
:107ac0000000eb001c2707001007980010002000a2
:107ad000192707002007980020002000162707001c
:107ae000300798001e0090006101b9004e00900020
:107af000de009000000041008180490040079800ae
:107b0000510798002e0090006101b9006e009000ae
:107b1000fe0090000000410081804900600798004d
:107b2000710798003e0090006101b9000e089000b6
:107b30009e0890000000410081804900000f9800dd
:107b4000110f98003e019000821f78002e009000d7
:107b5000801f78001e019000821f7800c0c9290094
:107b6000801f78004022210022e20700e8875700aa
:107b700040222100fde10700800078004022210022
:107b80009126070080bb200001002000ce0a0700dc
:107b90001e0fe800c7ff37004e009000de00900087
:107ba0004b09dd004500de0000007100c588de00e5
:107bb000902c89006e009000fe0090004b09dd00c3
:107bc0004500de0000007100c588de00a02c8900a1
:107bd0000e0890009e0890004b09dd004500de0075
:107be00000007100c588de0082d12f000200400035
:107bf000b02c89000080fa00000006001800fa008e
:107c0000889fbe003d1c070011002000800020005e
:107c1000e61f07009bff07009625f8009425f80053
:107c20009225f80090ca2900801f78004022210088
:107c3000f0e10700e887570040222100cbe1070070
:107c400080007800402221005f2607008000eb00c2
:107c500080002000d51f07000000eb00700798008f
:107c6000803e200001002000500798006107980026
:107c70000000eb00b0260700000f78001000200085
:107c8000ad2607001007980020002000aa26070054
:107c900020079800902c81001e0f10009e0090007d
:107ca000a02c81000080500010079800ae009000ca
:107cb000b02c810000805000200798002e0090001a
:107cc0000000e00006003d00ae00900080da2f00ca
:107cd000808f5000020034000000eb002007980065
:107ce0001e0078001e81b9009e0090001e009000ca
:107cf0000088b9000201400083814800ae00900076
:107d00002e0090000088b9000200400083804800e7
:107d100030079800410798005e009000ee00900048
:107d2000c289de004e0add004201de00020172005f
:107d30003e009000ce00900002004000838048008a
:107d40005007980061079800d08e80000000e00086
:107d50000a003a007e0090000000e00007003200b8
:107d60000000eb00700798008000eb00800020000e
:107d70008e1f07000000eb00e62007005e01900068
:107d8000ee019000703e200001002000800f5100a5
:107d9000818f590029003c007e009000e10f5000c7
:107da000b3ff320010002000700798001000200080
:107db000c08e8800d08e80000000e000fdff3a00f9
:107dc0003e009000ce009000809fbe00ae0090006c
:107dd000811f78001e029000841f78001e0078002a
:107de000801f78005e009000ee009000809fbe0033
:107df000a0cc2900801f7800402221007de10700ef
:107e0000f08757004022210058e1070080007800e9
:107e100040222100ec25070001f5210040b122009d
:107e2000c31b070010002000ba2007008000eb00f1
:107e3000800020005d1f07008dff37005e0190006d
:107e4000ee01900000902000d1032000800f51002f
:107e5000818f590086ff34007e009000e20f5000b1
:107e600083ff3200200020007007980010002000df
:107e7000c08e8800d08e80000000e000fdff3a0038
:107e80003e009000ce009000809fbe00ae009000ab
:107e9000811f78001e029000841f78001e00780069
:107ea000801f78005e009000ee009000809fbe0072
:107eb00020cf2900801f7800402221004de10700db
:107ec000f08757004022210028e107008000780059
:107ed00040222100bc2507009e00780063806000de
:107ee000300f98003e0890000000e00004003a00c7
:107ef000018420000000eb008d1b07000a00370002
:107f00003e089000e10f500004003a00016e20008e
:107f100040842000861b07000300370041d5200065
:107f200060f22000821b07000000eb0079200700b0
:107f30001e007800cf80de0015f007000004be00b0
:107f40001e009000cf80de0011f007000801be0087
:107f50003af00700100f9800210f98001e007800db
:107f6000cf80de000af007000004be001e00900073
:107f7000cf80de0006f007000801be002ff00700ea
:107f8000b2fd20009304240049f007000200200005
:107f90000308240088f00700b2fd200093fc2300b2
:107fa000baf00700b2fd200093ec2300b7f0070001
:107fb00013f107001af10700000f98000e08900057
:107fc000e80f5000040034000e08900068005000d4
:107fd000000f9800f9ff3700000000000e08900025
:107fe0000000e00004003d000e0890006800400022
:107ff000000f9800f9ff37000e0a9000841f7800e8
:108000001e089000ae089000809fbe009e00900069
:10801000811f78001e027800841f780060d129003b
:10802000801f780040222100f2e00700ec87570013
:1080300040222100cde0070080007800402221008e
:1080400061250700110020000e089000d71e0700d0
:1080500007ff37000600fa00889fbe008a1f7800dd
:108060000000eb007027890070278100e10f5000ad
:108070004d003c00024f220071278100400020008b
:108080000008b800000141006000b8000089be008f
:108090000000eb006027890060278100e70f500097
:1080a0001c003c00024f220071278100400020008c
:1080b0000008b80080044100024f220071278100af
:1080c000400020000008b80000054100a34c220039
:1080d00071278100800020000008b800622781001d
:1080e000020040000000d00003044000602781002f
:1080f000462807001880b900cf80de00ba1c400077
:10810000aa944800602781000000e80060278900e9
:10811000e1ff3700702781000000d000814f22006e
:1081200081004000010f7800024f2200712781007a
:10813000400020000008b800000041001000be0010
:1081400010079800210798001e019000ae019000d2
:10815000e00f5100e08f590006003d001e00900026
:10816000ae00900063004000e080480010079800d7
:10817000210798001e019000ae0190004e1add000c
:108180004210de0000007200c298de006322200070
:108190001e01780003094000702781000000e800fc
:1081a00070278900b0ff3700d1278100100320001d
:1081b000808f500014003c00d1278100e0fc2f008c
:1081c000808f500010003400c12781001003200070
:1081d000808f50000c003c00c1278100e0fc2f0084
:1081e000808f500008003400d1278100400120001a
:1081f0000088b900d0278900c127810040012000f4
:108200000088b900c0278900d1278100803e200066
:10821000808f500003003400803e2000d02789006a
:1082200006003700d127810080c12f00808f5000c9
:1082300002003d0080c12f00d0278900c1278100a6
:10824000803e2000808f500003003400803e2000dc
:10825000c027890006003700c127810080c12f0098
:10826000808f500002003d0080c12f00c027890090
:10827000d0278100d4220700c02781000f230700e8
:108280004f0578004f04be000080fa000000060091
:108290001000fa00889fbe008a9fbe00000f780081
:1082a000110798004006200020079800d0cc2c0031
:1082b000c1d4230030079800410798003000200007
:1082c000500798002e0090001e0050006007980094
:1082d00040258100cf80de002def07000005be00a5
:1082e0006e009000cf80de0029ef07003e01900075
:1082f000ce019000b0ef07000004be005e009000c9
:10830000cf80de0022ef07000001be000800be00a3
:1083100067ef07000001be000a00be00dbef0700a8
:108320003ff0070040258900ee00900040258100c5
:10833000808040001e0090000088b90070079800ff
:10834000fe009000703e2000808f5000110034002d
:10835000703e20001e019000110009000200d800ac
:108360008000fd006e0090000080500040258900d4
:1083700041258100c0032000808f5000020034009e
:10838000c003200040258900703e2000700798003f
:1083900013003700fe00900080c12f00808f500036
:1083a0000f003c0090c12f001e0190001100090039
:1083b0000200d8008000fd006e00900000804000a8
:1083c0004025890040258100ea0f400002003d0061
:1083d00060ff2f004025890090c12f007007980092
:1083e0007e0090004f05be004f04be000080fa00e2
:1083f000000006000a00fa00000f7800110798003c
:108400000000eb00200798000000eb003007980008
:108410002e0090001e00500040079800ce009000f3
:108420001e0090000088b90030079800be00900040
:10843000703e2000808f500003003400703e20000a
:108440003007980006003700be00900080c12f0062
:10845000808f500002003c0090c12f003007980030
:108460003e0090000080fa00000006000400fa00c0
:10847000889fbe0070002000642707000004780079
:108480000000eb00612707000000440022002000ec
:10849000110009000200d800610020007cff0700e5
:1084a000000f78000000eb00582707000004780058
:1084b00010002000552707008004440070002000b1
:1084c0005227070000047800600020004f270700b3
:1084d000000044000080540041002000c5ff070058
:1084e000100798001e0090001e00100036220700a2
:1084f0001e0090001e004000702207004f04be00c6
:108500000080fa00000006000000fa007c2307004b
:10851000242207000040eb002b280700bd2607009f
:10852000419c2000e03d2800b01c0700a12820004d
:1085300060232400ad1c0700971c0700ffff3700d5
:108540000000fa006e230700162207000040eb002f
:108550001d280700af26070041382000e03528001d
:10856000a21c0700a1282000a00224009f1c0700d5
:10857000891c0700ffff37000000fa006023070096
:108580000040eb001028070047250700a925070039
:10859000feff37000400fa00889fbe000000eb00d9
:1085a000102489001076800040118900411181005b
:1085b00010768000808f5000fcff32001076800023
:1085c000401189000000eb00100798001e00900089
:1085d000e20f50000e003e00424822009e00900034
:1085e000400020000008b800000441001e00900078
:1085f0003a270700cf80de0065ee0700008cbe0042
:108600001e0090000000e80010079800efff370000
:108610000000eb00100798001e009000e20f5000d1
:108620004b003e000000eb00000f7800100320001c
:108630009e0f100014003e00a22222009e00900017
:10864000200320000008b8009e00400040002000e9
:108650000008b80000044100424822009e0090003b
:10866000400020000008b80000004100a2702d006a
:1086700033ca23001000be00cfee0700008cbe00fe
:108680001e0fe800e9ff3700c24922009e0090005b
:10869000400020000008b8000004410042482200c9
:1086a0009e009000400020000008b80080044100b7
:1086b000424822009e009000400020000008b800c0
:1086c00000004100d2cc2c00c3d423001000be0017
:1086d000b9ee07000001be001900be00eaee070077
:1086e000008cbe00024922009e0090004000200045
:1086f0000008b80000044100424822009e0090009b
:10870000400020000008b8008004410042482200d8
:108710009e009000400020000008b80000004100ca
:10872000d2cc2c00c3d423001000be00a2ee070060
:108730000001be001900be00d4ee0700008cbe0090
:108740001e0090000000e80010079800b2ff3700fc
:108750004f04be000080fa00000006000000fa008e
:108760000000eb00107688001176800020062000c3
:10877000808f5000fcff36000080fa0000000600e9
:108780000800fa00881f78000e84e8000000eb0063
:10879000d2260700000c78000e84e80010002000ac
:1087a000ce260700100498000e84e8002000200068
:1087b000ca260700200498000000eb00000f780094
:1087c0000e80e80010007800cf80de00f0ed07009a
:1087d0000002be00004922001001be000400be00dd
:1087e00030ef07000000e0000b003d000e80e800c5
:1087f00010007800cf80de00e5ed07000002be002b
:10880000c04922001001be000400be0027ef07008f
:108810000000e00030003c000e80e80010009000f6
:10882000cf80de00daed07000002be000049220022
:1088300020019000b00190000400be0019ef070075
:108840000000e0000c003d000e80e80010009000e9
:10885000cf80de00ceed07000002be00c04922003e
:1088600020019000b00190000400be000fef07004f
:108870000000e00018003c000e80e800200090009e
:10888000cf80de00c2ed07000002be0000492200da
:1088900040019000d00190000400be0001ef0700ed
:1088a0000000e0000e003d000e80e8002000900077
:1088b000cf80de00b6ed07000002be00c0492200f6
:1088c00040019000d00190000400be00f7ee0700c8
:1088d0000000e0000200340010002000000f7800cb
:1088e0000e80e800530007001e0078004f04780057
:1088f0000080fa00000006000400fa00881f7800db
:108900000000eb00000f7800200020009e0f1000f8
:1089100045003c000000eb00100798009e0090000e
:1089200030062000808f50003d003c006380200016
:108930009e007800400620000008b8001e0190004c
:10894000020040000000d0000304400063802000cb
:108950009e007800400620000008b8001e0190002c
:10896000020040000000d00003004000100078002a
:10897000cf80de0086ed07000002be0042482200e4
:108980009e007800400020000008b8000000410070
:108990001001be000400be003bee0700a0ee070081
:1089a000000c7800638020009e00780040062000c4
:1089b0000008b8001e019000020040000000d00036
:1089c000030040001000e00011003d006380200023
:1089d0009e007800400620000008b8001e019000ac
:1089e000020040000000d0008301400064802000ad
:1089f0009e007800400620000008b8001e0190008c
:108a0000020040000000d000040040009009ea008d
:108a10001e0090000000e80010079800bfff37001c
:108a20001e0fe800b8ff37004f0478000080fa00fe
:108a3000000006000400fa00889fbe00000f7800c6
:108a40004111810010768000808f5000fcff3200c1
:108a500010768000401189000000eb00100798009c
:108a60001e009000e20f500073003c0042482200bc
:108a70009e009000400020000008b8000004410063
:108a8000424822009e009000400020000008b800ec
:108a900000024100a32222009e009000200320003b
:108aa0000008b8001224810082004000400020002d
:108ab0000008b800008041001001be001400be0094
:108ac000f1ed0700008cbe00a32222009e00900062
:108ad000200320000008b80012248100820040001a
:108ae000400020000008b800008441001e009000f3
:108af0000000d0001e00400010007800cf80de0093
:108b000023ed0700a2702d0033ca2300aaed070051
:108b1000008cbe00424822009e00900040002000d1
:108b20000008b80000044100424822009e00900066
:108b3000400020000008b80000024100a3222200eb
:108b40009e009000200320000008b800122481003d
:108b500082004000400020000008b8000080410072
:108b60001001be001400be00c8ed0700008cbe005e
:108b7000c24922009e009000400020000008b8007a
:108b800000044100424822009e0090004000200066
:108b90000008b80080044100424822009e00900076
:108ba000400020000008b80000004100d2cc2c009a
:108bb000c3d423001000be007fed07000001be00fb
:108bc0001900be00b0ed0700008cbe000249220073
:108bd0009e009000400020000008b8000004410002
:108be000424822009e009000400020000008b8008b
:108bf00080044100424822009e0090004000200076
:108c00000008b80000004100d2cc2c00c3d42300df
:108c10001000be0068ed07000001be001900be0094
:108c20009aed0700008cbe001e0090000000e800d6
:108c3000100798008aff37001124810000032000ec
:108c4000808f500004003c00102481000000e800e8
:108c500010248900020037000000eb001024890076
:108c60004f04be000080fa00000006001000fa0069
:108c7000110020000000eb00b0000700000f78009a
:108c80001e007800cf80de00c1ec0700020020004b
:108c9000030c240005ee07000000e000050035008d
:108ca00060e5200091fc23004007980051079800e0
:108cb000160037001e007800cf80de00b4ec0700fd
:108cc00002002000030c2c00f6ed07000000e0007d
:108cd00005003c0060e5200091fc2b004007980057
:108ce00051079800090037001e007800cf80de0091
:108cf000a7ec070002002000030c2400ecec0700a6
:108d0000eced070040079800510798006011b8008b
:108d10004e009000de009000e4ed07000000e0004f
:108d20003b003400110020002000200083000700d9
:108d3000100798001e009000cf80de0094ec070022
:108d400002002000030a2400d8ed07000000e00024
:108d50000500350060e5200091fc230060079800c5
:108d600071079800160037001e009000cf80de00cb
:108d700087ec070002002000030a2c00c9ed070061
:108d80000000e00005003c0060e5200091fc2b00a5
:108d90006007980071079800090037001e009000d6
:108da000cf80de007aec070002002000030a2400d6
:108db000bfec0700bfed070060079800710798003f
:108dc000f298200063f023006e009000fe009000f7
:108dd000b6ed07000000e000080034004e019000ee
:108de000de01900060e520009104240026ed0700dc
:108df00020079800310798003f0037004e00900090
:108e0000de00900020079800310798003a003700f4
:108e1000210020000000eb00480007001007980028
:108e20001e009000cf80de0059ec070002002000f9
:108e3000030a24009ded07000000e0000500350056
:108e400060e5200091fc23006007980071079800fe
:108e5000160037001e009000cf80de004cec0700ab
:108e600002002000030a2c008eed07000000e00045
:108e700005003c0060e5200091fc2b006007980095
:108e800071079800090037001e009000cf80de00b7
:108e90003fec070002002000030a240084ec0700d6
:108ea00084ed07006007980071079800f298200091
:108eb00063f02b006e009000fe00900079ed07003b
:108ec0000000e00008003d004e019000de0190002f
:108ed00060e5200091042400ebec070020079800d7
:108ee00031079800040037004e009000de0090002b
:108ef00020079800310798006011b8002e009000fc
:108f0000be00900067ed07000000e00007003d0094
:108f100062e52000930c24002e009000be0090001b
:108f2000daec070020079800310798002e00900027
:108f3000be0090000080fa00000006001a00fa004f
:108f4000000f78001107980090ff2f00100f980075
:108f500070002000200f980080002000300f980043
:108f6000c0052000400f98006000b800700798000e
:108f7000010f98001e08900030079800be00900076
:108f80002e089000808f500038003d006000b8002f
:108f90005007980061079800be08900041079800ac
:108fa000ce0090004e089000808f50001e003d00c3
:108fb000638020009e007800400620000008b80072
:108fc0004e019000020040000000d00083024000eb
:108fd000648020009e009000400620000009b80038
:108fe000ce0090003e009000008040000200400053
:108ff0000000d00084004000150078001181b90005
:109000005e009000ee009000000041008180490069
:1090100050079800610798004e0090000000e8009b
:1090200040079800deff37005e019000ee019000df
:109030007e0090008e089000800f5100818f5900b3
:10904000060034005e009000ee009000700798006b
:10905000010f9800be009000210798003e0090008c
:109060000000e80030079800c4ff37002e00900091
:109070000080fa00000006000a00fa00008fbe001f
:10908000600020002007980062e5200093ec230098
:109090001e00be0005ed07000000e00002003400e5
:1090a000700020002007980002ac2c0063f9230018
:1090b0001e00be00fdec07000000e00002003400ce
:1090c0009000200020079800c21e2500b3ff230057
:1090d0001e00be00f5ec07000000e00002003400b6
:1090e000c000200020079800b2c82e00f302240020
:1090f0001e00be00edec07000000e000020034009e
:10910000a00020002007980012022300230624005c
:109110001e00be00e5ec07000000e0000200340085
:10912000d000200020079800b29d2300a30824004f
:109130001e00be00ddec07000000e000020034006d
:10914000e00020002007980062ba2500330a2400be
:109150001e00be00d5ec07000000e0000200340055
:10916000f00020002007980012d72700c30b24002e
:109170001e00be00cdec07000000e000020034003d
:109180006000200020079800110020002e009000b1
:109190000008dd00201688006000b8003007980045
:1091a000410798003e019000ce019000f0112a0086
:1091b00071002000800f5100818f590007003c0092
:1091c0003e009000ce00900061004000e08048002a
:1091d0003007980041079800f2ff37000000eb00cd
:1091e000201688000080fa00000006000600fa0041
:1091f000008fbe0062e52000930424001e00be0024
:10920000a8ec07000000e00015003d000000eb00a6
:109210008c1f070062e52000930c24001e00be0096
:10922000a3eb070002002800234a2400e2eb07001a
:109230007bec070020079800803e2000e21e07001c
:1092400080c12f001d1f07007a1f070080007800d3
:109250002e009000808f5000fbff35001700370074
:109260000000eb00811f07001e01be0060e520002a
:10927000910c240004ec070062e52000930c24000c
:109280008beb070002002800234a2400caeb0700ea
:1092900063ec07002007980080c12f00ca1e07005a
:1092a000803e2000051f07006c1f0700800078002b
:1092b0002e009000808f5000fbff35000000eb0077
:1092c000c11e07000000eb00fc1e07000080fa0032
:1092d000000006000800fa00b21e0700adfc0700ff
:1092e00060e5200091fc230063ff0700a0d3290064
:1092f000801f7800402221003edc07008f87e900b4
:109300004022210019dc0700800078004022210063
:10931000ad2007009ffc070010002000000f780020
:109320001e00e0000300320015fd0700000f78006a
:10933000fbff370009fd0700a1e2a9006efd070051
:1093400090d42900801f78004022210029dc0700ea
:109350008f87e9004022210004dc070080007800ac
:1093600040222100982007000000eb003007980001
:10937000be009000c0022000808f500014003e000c
:10938000618020003e0090000000d00001004000fd
:1093900010007800801f7800e0d42900801f78003a
:1093a0004022210013dc0700e487570040222100ff
:1093b000eedb0700800078004022210082200700b9
:1093c0003e0090000000e80030079800e8ff3700fa
:1093d00030d52900801f78004022210005dc0700dd
:1093e0008f87e90040222100e0db07008000780041
:1093f00040222100742007000000eb003007980095
:10940000be009000c0022000808f500015003e007a
:10941000618020003e0090000000d000010040006c
:10942000800cb00010007800801f7800e0d4290084
:10943000801f780040222100eedb0700e487570000
:1094400040222100c9db0700800078004022210073
:109450005d2007003e0090000000e8003007980003
:10946000e7ff3700a0d52900801f780040222100a7
:10947000e0db07008f87e90040222100bbdb07000b
:1094800080007800402221004f2007000000eb0000
:1094900030079800be009000c0022000808f50006e
:1094a00015003e00618020003e0090000000d000ca
:1094b000010040000019b00010007800801f780003
:1094c000e0d42900801f780040222100c9db07007a
:1094d000e487570040222100a4db070080007800c9
:1094e00040222100382007003e0090000000e800e4
:1094f00030079800e7ff370010d62900801f78005a
:1095000040222100bbdb07008f87e90040222100b9
:1095100096db070080007800402221002a20070007
:10952000d2fd07001007980021079800a1e2a800cb
:109530001e009000ae009000cffe07001e009000bd
:10954000ae00900029ff070072ff37001a00fa00f2
:10955000889fbe008a9fbe000080eb00300f9800fd
:109560000000eb00400f9800760147001300200038
:10957000e1ff2f00f00720008e040700400f980045
:109580004e08900063006000400f98000000eb0060
:10959000000f78004e089000e30f500003003200e7
:1095a0004e0890000000e00005003a001000200086
:1095b00010079800c003200020079800040037001f
:1095c000c00320001007980010002000200798001a
:1095d00080002000300798009e0090002e00900030
:1095e0000088b90040079800890e0700ae0090007f
:1095f0003e009000008db9009e0090003e0090005b
:10960000008cb900ae0090003e0090000088b900c8
:10961000021e20000000510022002000110009005d
:109620000200d80080037800010078009e009000be
:109630003e0090000088b900022820000000510080
:1096400022002000110009000200d8001e0378004b
:10965000be0290003e0290008a0178000801780066
:10966000870078001f0e0700110020001000200066
:10967000480e07005e0e0700402221008a140700f2
:10968000991a07000000eb00a21a07000000eb0087
:10969000bf1a0700e51407000000e000fdff3200dc
:1096a00040222100600798000000eb00000f9800a6
:1096b0000000eb00100f98000000eb00200f980056
:1096c0000040eb00704f98000000eb00500798003e
:1096d0005e009000fd0f500017003c006e009000ef
:1096e00010407800604f98006e0090000000e80085
:1096f000600798006e4890008080fb000e08900084
:1097000001004000000f9800ee4890007e48900055
:1097100080cf5000040036006e489000704f9800d3
:109720005e019000220f98005e0090000000e800ab
:1097300050079800e6ff370000000000de009000b0
:109740002e009000808f500017003d006e009000aa
:1097500010407800604f98006e0090000000e80014
:10976000600798006e4890008080fb001e08900003
:1097700001004000100f9800ee4890007e489000d5
:1097800080cf5000040036006e489000704f980063
:109790005e019000220f98005e0090000000e8003b
:1097a00050079800e5ff37002e089000f30f500097
:1097b00004003e001100200070002000fb1807008c
:1097c0000b003700ae08900070022000808f500020
:1097d00004003e00110020000000eb00f318070019
:1097e000030037001100200010002000ef180700d0
:1097f0004e089000e30f5000030032004e08900026
:10980000e20f50000c003a00ae089000a0002000cb
:109810000008b80042ed2f00020040006a1d07005a
:10982000ae08900060ff2f000008b800c012b00022
:10983000a21d07000b003700ae08900060ff2f004c
:109840000008b800c012b0005f1d0700ae0890000d
:10985000a00020000008b80042ed2f0002004000e8
:10986000961d07002e089000801f78007e4890000b
:109870000080fb00801f78001e099000821f780086
:109880000e089000801f780040d62900801f7800c5
:1098900040222100d7da0700ea8757004022210042
:1098a000b2da07008000780040222100461f07003e
:1098b0008038210001002000830307006eff37007d
:1098c0001200fa00889fbe008a9fbe000000eb00d5
:1098d000000f780040012000100798004001200090
:1098e0002007980080002000300798009e0090001c
:1098f0002e0090000088b90040079800c40d0700b2
:10990000ae0090003e009000008db9009e009000d7
:109910003e009000008cb900ae0090003e00900028
:109920000088b900021e2000000051002200200023
:10993000110009000200d8008003780001007800bf
:109940009e0090003e0090000088b9000228200090
:109950000000510022002000110009000200d80080
:109960001e037800be0290003e0290008a0178003b
:1099700008017800870078005a0d070011002000c8
:1099800010002000830d0700990d070046200700f6
:1099900040222100c4130700d31907000000eb0088
:1099a000dc1907000000eb00f91907000000eb00cc
:1099b00098220700fe0f500008003c001000200015
:1099c00094220700fe0f500004003c0020002000fd
:1099d00090220700fe0f500002003400100020000b
:1099e000cc1907000000eb00f2210700800078008e
:1099f00000192000808f5000030034001100200067
:109a00000000eb006918070010002000e9210700a2
:109a10008000780000192000808f5000030034007f
:109a20001100200010002000601807002000200016
:109a3000e02107008000780000192000808f50008e
:109a400003003400110020002000200057180700f8
:109a500030002000d7210700800078000019200086
:109a6000808f5000030034001100200030002000df
:109a70004e18070040002000ce210700800078002b
:109a800000192000808f50000300340011002000d6
:109a9000400020004518070050002000c5210700a5
:109aa0008000780000192000808f500003003400ef
:109ab00011002000500020003c180700600020002a
:109ac000bc2107008000780000192000808f500022
:109ad000030034001100200060002000331807004c
:109ae00070002000b32107008000780000192000da
:109af000808f50000300340011002000700020000f
:109b00002a18070000000000c81307000000e0004a
:109b1000fdff32006000b8006007980071079800f0
:109b200040222100000f98000000eb005007980031
:109b3000de0090004e009000808f500011003d002c
:109b40000e089000104078000081fb000300200008
:109b50006e009000fe0090000000410081804900ee
:109b600060079800710798000e0890000000e80058
:109b7000000f98005e0090000000e8005007980079
:109b8000ebff37006e009000fe009000809fbe004b
:109b900020d92900801f78004022210015da070013
:109ba000e687570040222100f0d9070080007800a6
:109bb00040222100841e07006e019000fe019000eb
:109bc00000b82b0001002000800f5100818f590048
:109bd00002003600100020006d19070080382100b7
:109be00001002000b802070069ff37003200fa00c8
:109bf00040062000400798006a00470021da29004b
:109c000050179800611798005e109000ee109000b9
:109c100007000900311878007a00470021db29008d
:109c200070179800011f98007e1090008e18900009
:109c300007000900311878002b1907000000eb001d
:109c4000341907000000eb00511907000000eb0079
:109c5000582107008000780080252000808f500068
:109c600003003400110020000000eb00cf170700b4
:109c7000100020004f210700800078008025200080
:109c8000808f5000030034001100200010002000dd
:109c9000c61707002000200046210700800078003a
:109ca00080252000808f5000030034001100200028
:109cb00020002000bd170700300020003d210700d4
:109cc0008000780080252000808f50000300340041
:109cd0001100200030002000b417070040002000d1
:109ce000342107008000780080252000808f5000fc
:109cf000030034001100200040002000ab170700d3
:109d0000500020002b2107008000780080252000d3
:109d1000808f50000300340011002000500020000c
:109d2000a2170700600020002221070080007800b1
:109d300080252000808f5000030034001100200097
:109d4000600020009917070070002000192107000b
:109d50008000780080252000808f500003003400b0
:109d60001100200070002000901707000000eb0099
:109d7000102107008000780080252000808f50008f
:109d80001e003c00100020000a210700800078001f
:109d900080252000808f500018003c00200020000b
:109da000042107008000780080252000808f50006b
:109db00012003c0050002000fe20070080007800c8
:109dc00080252000808f50000c003c0060002000a7
:109dd000f82007008000780080252000808f500048
:109de00006003c0070002000f22007008000780090
:109df00080252000808f50005b0034001000200080
:109e0000c4180700800c200020079800800c200058
:109e1000300798000000eb00000f78007000200071
:109e20009e0f100025003c001e007800e120070076
:109e3000100798009e009000811f780020dc290008
:109e4000801f7800402221006ad90700e48757006c
:109e50004022210045d907008000780040222100df
:109e6000d91d0700ea0047001e0078000000d0005e
:109e7000810040001e0090004480de001180b90087
:109e80002e0190000000410020079800fa004700d2
:109e90001e0078000000d000810040001e009000ed
:109ea0004480de001180b9003e01900000004100b6
:109eb000300798001e0fe800d8ff37003e009000e2
:109ec000801f7800ae009000811f780070dc2900b0
:109ed000801f78004022210046d90700e6875700fe
:109ee0004022210021d90700800078004022210073
:109ef000b51d0700ae00900000322000808f50009a
:109f0000020034000032200020079800be009000bc
:109f100000322000808f5000020034000032200008
:109f200030079800ae00900000ce2f00808f5000c8
:109f300002003d0000ce2f0020079800be009000d8
:109f400000ce2f00808f500002003d0000ce2f0079
:109f5000300798002e0090009b1b07003e009000e9
:109f6000d61b070019003700c02b2000961b0700e6
:109f70004e0090000000e80040079800ce009000de
:109f8000c02b2000808f50000200340040062000cb
:109f9000400798004e009000c81b07004e0090003c
:109fa000801f780080dd2900801f7800402221007a
:109fb00010d90700e487570040222100ebd80700a2
:109fc00080007800402221007f1d070000e224006d
:109fd00001002000bc01070017ff37002400fa0031
:109fe000889fbe000000eb00000f7800700020008a
:109ff0009e0f100009003c00640147009e0078009d
:10a00000400020000008b800000141006000b800d6
:10a010000089be001e0fe800f4ff37000000eb00cf
:10a02000100798001e009000ff0f50001d003c001c
:10a030000000eb00000f7800720020009e0f11005e
:10a0400011003c00640147009e00780040002000a1
:10a050000008b80080044100640147009e007800b9
:10a06000400020000008b800000441001e007800f5
:10a0700050200700cf80de00b81c4000a8944800a4
:10a080001e0fe800ecff37000071220001002000e5
:10a090008d0107001e0090000000e80010079800e6
:10a0a000e0ff37000000eb00000f78007000200098
:10a0b0009e0f100021003c00e15622001e00780097
:10a0c0000000d00081014000640147009e0078003c
:10a0d000400020000008b800000041001000be0051
:10a0e0004b09dd004500de0000007100c588de0080
:10a0f00080097800e15622001e0078000000d000a0
:10a100000100400010007800801f780040de290028
:10a11000801f780040222100b6d80700e48757004e
:10a120004022210091d807008000780040222100c1
:10a13000251d07001e0fe800dcff370090de290018
:10a14000801f780040222100aad807008f87e900ed
:10a150004022210085d8070080007800402221009d
:10a16000191d0700006a2800110020005601070091
:10a170004f04be000080fa00000006000200fa0052
:10a18000e7c2bf000080fb000000d1000080fb00a0
:10a1900061006000000f78001e0078000000d00011
:10a1a000000f7800e7c2bf000080fb006100600084
:10a1b0009e00780080804000010f78001e0078002b
:10a1c0000000d000000f7800e6c2bf000080fb0056
:10a1d0004700de000080fb009e0078008080400089
:10a1e000010f78001e0078000000d000000f7800fa
:10a1f000e6c2bf000080fb004600de000080fb00de
:10a20000610060009e00780080804000010f7800af
:10a210001e0078000080fa00000006000400fa002a
:10a22000881f7800000f78000000eb0010079800ee
:10a230001e009000e70f50000f003e001e0090002f
:10a240000000d0001e0440001e009000d91f07002f
:10a2500000017800e15622001e0090000000d000ae
:10a2600001004000100c51001e0090000000e800aa
:10a2700010079800eeff37004f0478000080fa00c6
:10a28000000006000400fa00000f78001107980093
:10a2900000ce2f009e0f100002003d0000ce2f00c8
:10a2a000000f7800003220009e0f100002003400e2
:10a2b00000322000000f78009e00900000ce2f009a
:10a2c000808f500002003d0000ce2f001007980044
:10a2d0009e00900000322000808f50000200340069
:10a2e00000322000100798001e007800b61a070000
:10a2f0001e009000f11a07000080fa00000006001e
:10a300001a00fa00fe1b0700a61a070033ff070019
:10a310000000eb00400f980064004700bfff0700fb
:10a320000000eb00300f980094ff07006100600010
:10a330000000e000400032008000eb0060002000e0
:10a340001a16070011002000200020001716070031
:10a350000000eb00200f98002e089000e70f50003f
:10a360000b003c00e40047002e0890000000d000e5
:10a370008100400020032000910f100004003c00e9
:10a380002e0890000000e800200f9800f2ff370030
:10a390002e089000e80f500003003a001000200043
:10a3a000300f980063003700e154220060ff2f0057
:10a3b00080087800e154220060ff2f00f000980030
:10a3c000e1552200a000200080087800e15522001d
:10a3d000a0002000f000980064004700a00090005a
:10a3e000c0122000808f500052003400e40047006b
:10a3f000640047001000900082f32f00020040002c
:10a4000090009800e400470064004700200090009e
:10a4100082da2f0002004000a0009800e40047000c
:10a420006400470030009000c2f92f000200400095
:10a43000b00098003f0037001100200060002000ad
:10a44000da1507008000eb0020002000d715070078
:10a450000000eb00200f98002e089000e70f50003e
:10a460000b003c00e40047002e0890000000d000e4
:10a470008100400020032000910f100004003c00e8
:10a480002e0890000000e800200f9800f2ff37002f
:10a490002e089000e80f500003003a001000200042
:10a4a000300f980023003700e1542200a000200064
:10a4b00080087800e1542200a0002000f0009800fd
:10a4c000e155220060ff2f0080087800e15522004e
:10a4d00060ff2f00f000980064004700d00090005b
:10a4e000c0122000808f500012003400e4004700aa
:10a4f0006400470040009000c2f92f0002004000b5
:10a50000c0009800e400470064004700500090003d
:10a5100082da2f0002004000d0009800e4004700db
:10a52000640047006000900082f32f0002004000aa
:10a53000e0009800800c2000000f7800800c2000c4
:10a54000100798003e0890000000e00023003a0049
:10a550000000eb00200f98002e089000e70f50003d
:10a560001e003c00e15422002e0890000000d000a4
:10a5700001014000e40047002e0890000000d000d8
:10a5800001004000100078004480de001280b90015
:10a590001e0f4000e15522002e0890000000d00060
:10a5a00001014000e40047002e0890000000d000a8
:10a5b00001004000100078004480de001280b900e5
:10a5c0001e01900000004100100798002e08900026
:10a5d0000000e800200f9800dfff37009e00900089
:10a5e0001e00780027ff070080a92300010020003b
:10a5f0003500070048ff37000400fa00310520004d
:10a60000e0df2900f01b0700fb1b07000000e00053
:10a61000fdff3a00ed1307000e007800ba1b07009b
:10a620001e4078000040d000004f78000e00e80087
:10a63000b51b07001e4090000004e0000c003d0028
:10a64000e61307001e409000804078000174a100ce
:10a650001e407800e913070020479800e313070025
:10a660000e80e80011002000d71b0700eaff37002a
:10a670000e80e800a41b0700d81307002e419000ad
:10a680009e4090001e40780013140700d713070067
:10a69000e1ff37000400fa007105200020e52900e1
:10a6a000c91b0700d41b07000000e000fdff3a00b3
:10a6b000c61307000e007800931b07000e00e80089
:10a6c000911b0700fbff37000800fa00008fbe0057
:10a6d0006000b80020079800310798002e00900015
:10a6e000be009000be0f5000ae8f580007003d0026
:10a6f0002e009000be00900061004000e080480005
:10a700002007980031079800f4ff37000080fa0016
:10a71000000006000200fa00e7c2bf000080fb0054
:10a720000000d1000080fb0061006000000f780095
:10a730001e0078000000d000000f7800e7c2bf00c4
:10a740000080fb00610060009e0078008080400077
:10a75000010f78001e0078000000d000000f780084
:10a76000e6c2bf000080fb004700de000080fb0067
:10a770009e00780080804000010f78001e00780065
:10a780000000d000000f7800e6c2bf000080fb0090
:10a790004600de000080fb00610060009e00780043
:10a7a00080804000010f78001e0078000080fa00d1
:10a7b000000006003200f800900188006118e100f6
:10a7c000040032007018e10002003200f0ff2f0098
:10a7d000030037003119ba008301e900fdff3a0098
:10a7e0003200f90000000600849fbe004220a9004c
:10a7f000440424006110e1000a00320054042400e3
:10a800007010e1000700320064042400f5ff2f00ff
:10a810000510e10003003200f0ff2f004f02be00e0
:10a82000000006003200f800203b8800113b880041
:10a83000043b88004200f800000e20004220b700d0
:10a8400050052000303b8800a00a2000303b8800e3
:10a8500061e7a800000000000000000061e7af0011
:10a86000feff37000000eb004200f9003200f90063
:10a870004f02be0000000600841f78004220a9009d
:10a88000440024006118e100060032005400240056
:10a890007018e100030032004f027800f0ff2f0033
:10a8a000000006003200f80091018800821f780045
:10a8b0003019bb008301e900fdff3a00213b88000d
:10a8c0004f017800123b8800043b88004200f800ea
:10a8d000000e20004220b70050052000303b8800c9
:10a8e000a00a2000303b880061e7a80000000000bb
:10a8f0000000000061e7af00feff37000000eb0042
:10a900004200f9003200f9004f0278000000060012
:10a910001c00fa000000eb0010079800e0aa2000dd
:10a9200035030700000f78000000eb0020079800b7
:10a930002e0090009e0f5000ba003d000000eb007a
:10a9400040079800ae009000d00120000008b80039
:10a9500042ab2000020040001004e00002003a0078
:10a9600010002000400798008000eb00510798007d
:10a97000ae009000d00120000008b80052ab2000cb
:10a98000020040001004e00002003a001000200025
:10a9900050079800ce0090005e0190008280600019
:10a9a000610798000000eb0070079800ae0090006f
:10a9b000d00120000008b80062ab20000200400077
:10a9c0001004e00002003a00100020007007980018
:10a9d000ee0090007e01900082806000010f9800e0
:10a9e0000000eb00100f9800ae009000d001200096
:10a9f0000008b80032ab20000200400081c0b30064
:10aa000090cf100002003a0012002000120f9800b0
:10aa10008e0890001e099000028060000000e00097
:10aa20007c003200ae009000d00120000008b80089
:10aa3000e2aa2000000041007e0307000000eb00b6
:10aa4000200f9800ae009000d00120000008b80050
:10aa500072ab20008200400050c6b300914f10003e
:10aa600002003a0010002000200f98008000eb0048
:10aa7000310f9800ae009000d00120000008b8000f
:10aa800082ab200082004000d0c2b300914f100082
:10aa900002003a0010002000300f9800ae0890002d
:10aaa0003e09900082806000410f98000000eb009a
:10aab000500f9800ae009000d00120000008b800b0
:10aac00092ab20008200400000c7b300914f1000fd
:10aad00002003a0010002000500f9800ce089000ad
:10aae0005e099000028060000000e0004900320032
:10aaf0000000eb00300798003e009000e30f50008c
:10ab000022003c009e009000b00020000008b80029
:10ab10003e0190000200400001bd20008101400084
:10ab2000ae009000d00120000008b8003e01900067
:10ab300002004000e2aa2000020040009049780094
:10ab40009e009000b00020000008b8003e01900078
:10ab50000200400061bd200081014000ae00900075
:10ab6000d00120000008b8003e0190000200400023
:10ab7000e2ab200002004000904978003e009000c7
:10ab80000000e80030079800dbff37009e009000cf
:10ab9000b00020000008b800a2bd200082004000e4
:10aba0000040eb008048780040002000300798000b
:10abb0003e009000e50f500013003c009e00900006
:10abc000b00020000008b8003e01900002004000e4
:10abd00001bd200081014000ae009000d0012000a6
:10abe0000008b8003e01900002004000e2aa2000e8
:10abf00002004000904978003e0090000000e8000c
:10ac000030079800eaff37001e0090000000e800bf
:10ac1000100798002e0090000000e8002007980020
:10ac200043ff37001e0090000080fa00000006007d
:10ac30000600fa00e0c32000f200070034ff07001e
:10ac4000000f78001e00e0000b00320060bd200005
:10ac50009601070000bd2000670307002047980009
:10ac6000e0c32000910107002e4090000000fb008f
:10ac700020079800020037003006200020079800c7
:10ac80002e0090000080fa00000006003000fa005c
:10ac900020c0b300004f780020c5b30010479800d3
:10aca00060c2b300204798000040eb003047980096
:10acb0000040eb004047980080c7b3005047980021
:10acc00030c0b30060479800710020000e0078008b
:10acd0003d1a07000000eb00301798000040eb0021
:10ace000006f9800e80047003e1090000080400090
:10acf000051a07000000e00008003200e8004700e5
:10ad00003e1090000080400010407800006f9800d6
:10ad10003e1090000000e800301798000e68900088
:10ad2000e34f5000efff3a006800470030409000ca
:10ad30000000fb00e60040003e109000810f500034
:10ad4000e8ff3500e80047003e109000808040009a
:10ad50000040eb00804878000000eb0030179800be
:10ad600068004700604090008000fb003e109000ab
:10ad7000810f50000d003d00a10220008e80400098
:10ad80003e10900000814000e80047003e10900017
:10ad90000080400067004000104978003e1090009d
:10ada0000000e80030179800edff3700a1022000f6
:10adb0008e8040003e109000808040000040eb00fc
:10adc00080487800a00220000e004000a200200071
:10add0008000eb0098d507000080fa000000060014
:10ade0001600fa0020c0b300004f780020c5b30061
:10adf00010479800a0c1b300204798000040eb0026
:10ae0000304798000040eb0040479800c0c6b300b0
:10ae10005047980030c0b300604798007100200090
:10ae20000e007800e81907000000eb00100f9800f2
:10ae30000040eb0040579800e80047001e089000d3
:10ae400000804000b01907000000e0000800320058
:10ae5000e80047001e089000008040001040780085
:10ae6000405798001e0890000000e800100f98005e
:10ae70004e509000e34f5000efff3a00680047004b
:10ae8000304090000000fb00e60040001e089000eb
:10ae9000810f5000e8ff3500e80047001e089000d1
:10aea000808040000040eb00804878006800470048
:10aeb000604090000000fb000080fa0000000600e7
:10aec0001600fa0020c0b300004f780020c5b30080
:10aed0001047980010c1b3002047980010c0b3007d
:10aee000304798000040eb004047980040c6b30050
:10aef0005047980010c0b3006047980030c0b300be
:10af000070479800810020000e007800ae190700fd
:10af10000000eb00100f98000040eb004057980035
:10af2000e80047001e0890000080400076190700e6
:10af30000000e00008003200e80047001e08900012
:10af40000080400010407800405798001e08900094
:10af50000000e800100f98004e509000e34f5000a2
:10af6000efff3a0068004700304090000000fb000f
:10af7000e60040001e089000810f5000e8ff3500f9
:10af8000e80047001e089000808040000040eb0071
:10af90008048780068004700604090000000fb0097
:10afa0000080fa00000006000400fa000de2a9008b
:10afb000de62a900e262a9006000b800008fbe0056
:10afc0001e00be00f2e307006266260063662400ee
:10afd00034e507000000e00005003d0010002000ff
:10afe000010020001e0f40005e974800f4ff37006c
:10aff000e262a800de62a800061907000080fa00dd
:10b00000000006002c00fa00000f78008e80e80097
:10b0100020c0b300804878008e80e80020c5b300cf
:10b02000904098008e80e80060c1b300a040980076
:10b030008e80e8000040eb00b04098008e80e80071
:10b040000040eb00c04098008e80e80080c6b3004e
:10b05000d04098008e80e80030c0b300e0409800f7
:10b060000e80e80071002000571907000000eb0077
:10b07000401798000040eb00206f9800ea0047005e
:10b080004e109000008040001f1907000000e000f3
:10b0900008003200ea0047004e1090000080400097
:10b0a00010407800206f98004e1090000000e800db
:10b0b000401798002e689000e34f5000efff3a00d1
:10b0c0006a004700304090000080fb00e60040002e
:10b0d0004e109000810f5000e8ff3500ea00470055
:10b0e0004e109000808040000040eb0080487800c7
:10b0f0000000eb00401798006a0047007040900085
:10b100008080fb004e109000810f50000b003d002e
:10b110004e1090001e014000ea0047004e109000c3
:10b120000080400068004000104978004e109000f8
:10b130000000e80040179800efff37004e10900025
:10b140009e0040000040eb00804878006a00470005
:10b15000604090000000fb000080fa000000060044
:10b160003600fa00000f78008e80e80020c0b3009f
:10b17000804878008e80e80020c5b3009040980099
:10b180008e80e80030c0b300a04098008e80e800b8
:10b190000040eb00b04098008e80e8000040eb00db
:10b1a000c04098008e80e80050c5b300d0409800a1
:10b1b0008e80e80030c0b300e04098000e80e800c8
:10b1c00071002000001907000000eb00101f98001c
:10b1d0000040eb0040779800ea0047001e189000fe
:10b1e00000804000c81807000000e000080032009e
:10b1f000ea0047001e1890000080400010407800d0
:10b20000407798001e1890000000e800101f98007a
:10b210004e709000e34f5000efff3a006a00470085
:10b22000304090000000fb00e60040001e18900037
:10b23000810f5000e8ff3500ea0047001e1890001b
:10b24000808040000040eb00804878000000eb0068
:10b25000101f98006a004700704090008000fb00bb
:10b260001e189000810f50000b003d001e1890002a
:10b270001e014000ea0047001e18900000804000b8
:10b2800068004000104978001e1890000000e80097
:10b29000101f9800efff37006a00470060409000e1
:10b2a0000000fb000080fa00000006003000fa00f9
:10b2b000000f78001e0078002cd40700701798004b
:10b2c0008e80e80020c0b300804878008e80e800bf
:10b2d00020c5b300904098008e80e80070c1b30094
:10b2e000a04098008e80e8006e6890000040e80062
:10b2f000b04098008e80e8000040eb00c04098000d
:10b300008e81e8000e80e8008e80e80010419000f9
:10b3100021409000804041000e80e80030409000c5
:10b3200000c04000d04198000e80e800ee68900018
:10b33000614098000000eb0050179800de1090006c
:10b340007e109000808f50000b003d008e80e80042
:10b350005e10900000804000e70040005e1090000a
:10b360001e004000904878005e1090000000e80049
:10b3700050179800f1ff37008e80e8007e10900093
:10b3800000804000e700400030c0b30080487800f3
:10b390007e109000e80040000e80e8008a18070048
:10b3a0000000eb00501798000040eb00406f980041
:10b3b000010220008e8040005e109000008040005e
:10b3c000511807000000e0000900320001022000cf
:10b3d0008e8040005e109000008040001040780099
:10b3e000406f98005e1090000000e8005017980031
:10b3f0004e689000e34f5000edff3a00000220003d
:10b400000e004000304090000000fb00e6004000cd
:10b410005e109000810f5000e5ff35000102200012
:10b420008e8040005e109000808040000040eb0065
:10b4300080487800000220000e004000604090002c
:10b440000000fb000080fa00000006003a00fa004d
:10b45000000f78001e007800c4d30700401f98003a
:10b460004e1890000000e800401f98008e80e80011
:10b4700020c0b300804878008e80e80020c5b3006b
:10b48000904098008e80e80040c0b300a040980033
:10b490008e80e8000e7890000040e800b0409800f0
:10b4a0008e80e8000040eb00c04098008e81e800ec
:10b4b0000e80e8008e80e80010419000214090004e
:10b4c000804041000e80e8003040900000c0400005
:10b4d000d04198000e80e8008e789000614098007e
:10b4e0000000eb00201f9800ae1890004e1890004e
:10b4f000808f50000b003d008e80e8002e189000d9
:10b5000000804000e70040002e1890001e00400020
:10b51000904878002e1890000000e800201f980046
:10b52000f1ff37008e80e8004e1890000080400048
:10b53000e700400030c0b300804878004e1890000b
:10b54000e80040000e80e8001f1807000000eb0034
:10b55000201f98000040eb0060779800a1022000b7
:10b560008e8040002e18900000804000e6170700f3
:10b570000000e00009003200a10220008e8040009f
:10b580002e189000008040001040780060779800ee
:10b590002e1890000000e800201f98006e709000a8
:10b5a000e34f5000edff3a00a00220000e004000e3
:10b5b000304090000000fb00e60040002e18900094
:10b5c000810f5000e5ff3500a10220008e80400071
:10b5d0002e189000808040000040eb0080487800ea
:10b5e000a00220000e004000604090000000fb0020
:10b5f0000080fa00000006004a00fa00000f780000
:10b600008e80e80020c0b300804878008e80e8007b
:10b6100020c5b300904098008e80e8000040eb0009
:10b62000a04098008e80e80030c0b300b040980081
:10b630008e80e8000040eb00c04098008e80e8005b
:10b6400050c5b300d04098008e80e80050c0b300d1
:10b65000e04098008e80e800a0c0b300f040980061
:10b660008e80e8000040eb00804898008e80e80063
:10b6700030c0b300904898000e80e800a100200080
:10b68000d11707000000eb00701f98000000eb00ce
:10b69000102798000000eb00002798000040eb0006
:10b6a00040c798000000eb0000279800ec0047001e
:10b6b0000e20900000804000931707000000e0007b
:10b6c00008003200ec0047000e209000008040008f
:10b6d0001040780040c798000e2090000000e8005d
:10b6e000002798004ec09000e34f5000efff3a0053
:10b6f0006c004700304090000000fb00e600400076
:10b700000e209000810f5000e8ff35006c004700cc
:10b710009040900090c6b30080cf50002c003a00bb
:10b720000000eb00002798000e209000e50f50006d
:10b730000f003c00fe189000d00120000008b80067
:10b740009e0040000e20900000814000ec00470069
:10b750000e209000008040006600400010497800f4
:10b760000e2090000000e80000279800eeff370050
:10b770000000eb00002798000e209000e20f500020
:10b7800010003c00fe189000d00120000008b80016
:10b790009e0040000e2090000080400066014000a6
:10b7a000ec0047000e209000008040006c0040003c
:10b7b000104978000e2090000000e8000027980053
:10b7c000edff37007e1890000000e800701f980021
:10b7d0000000eb00302798006c004700904090007c
:10b7e00030c4b30080cf50000200320011002000ae
:10b7f000312798000001eb00422798006c004700b9
:10b80000204090000004e000020032001000200000
:10b8100040279800be2090004e21900002806000da
:10b820000000e0009fff3a007e1890000080fa00c0
:10b83000000006004600fa00000f78008e80e80045
:10b8400020c0b300804878008e80e80020c5b30097
:10b85000904098008e80e80020c0b300a04098007f
:10b860008e80e80060c0b300b04098008e80e80091
:10b870000040eb00c04098008e80e800a0c5b300f7
:10b88000d04098008e80e8001e00780010407800bc
:10b89000e04098008e80e8001e0078001040900084
:10b8a000f04098008e80e8001e0078002040900054
:10b8b000804898008e80e8001e007800304090009c
:10b8c000904898008e80e8001e007800404090006c
:10b8d000a04898008e80e8001e007800504090003c
:10b8e000b04898008e80e80030c0b300c04898008f
:10b8f0000e80e800d1002000331707000000eb00a5
:10b90000102798000040eb0040c79800f000470067
:10b910001e20900000804000fb1607000000e000a1
:10b9200008003200f00047001e2090000080400018
:10b930001040780040c798001e2090000000e800ea
:10b94000102798004ec09000e34f5000efff3a00e0
:10b9500070004700304090000000fb00e60040000f
:10b960001e209000810f5000e8ff3500f0004700d6
:10b970001e209000808040000040eb00804878004e
:10b9800070004700604090000004e00015003a009d
:10b990000000eb001027980070004700504890000e
:10b9a0008000fb001e209000810f50000d003d0024
:10b9b0009e0078001e209000008040006901400039
:10b9c000f00047001e209000008040006e00400004
:10b9d000104978001e2090000000e8001027980011
:10b9e000edff370070004700604090000000fb0052
:10b9f0000080fa00000006004c00fa00000f7800fa
:10ba00008e80e80020c0b300804878008e80e80077
:10ba100020c5b300904098008e80e800a0c0b3001d
:10ba2000a04098008e80e80080c0b300b04098002d
:10ba30008e80e8000040eb00c04098008e80e80057
:10ba400040c6b300d04098008e80e80010c0b3001c
:10ba5000e04098008e80e8001e00780010407800da
:10ba6000f04098008e80e8001e00e800104078004a
:10ba7000804898008e80e8001e80e8001040780022
:10ba8000904898008e80e8001e0178006300410015
:10ba900010407800a04898008e80e8001e017800d1
:10baa0006400410010407800b04898008e80e800a3
:10bab0001e0178006500410010407800c0489800e1
:10bac0008e80e80010c0b300d04898008e80e80057
:10bad00030c0b300e04898000e80e800f10020007c
:10bae000b91607000000eb00202798000040eb008b
:10baf00060c798000000eb0020279800f200470084
:10bb00002e209000008040007f1607000000e0001b
:10bb100008003200f20047002e2090000080400014
:10bb20001040780060c798002e2090000000e800c8
:10bb3000202798006ec09000e34f5000efff3a00be
:10bb400072004700304090000000fb00e60040001b
:10bb50002e209000810f5000e8ff35000000eb0020
:10bb60004027980072004700a040900090c6b300a4
:10bb700080cf5000020032001100200041279800c1
:10bb80000001eb005227980072004700204090000f
:10bb9000eb4f5000020032001000200050279800a8
:10bba000ce2090005e219000028060000000e00046
:10bbb000d0ff3a0072004700604090000000fb0098
:10bbc0000080fa00000006002000fa0020c0b30048
:10bbd000004f780020c5b30010479800d0c0b300d4
:10bbe0002047980010c0b300304798000040eb0099
:10bbf0004047980000c6b3005047980010c0b300fb
:10bc00006047980030c0b300704798008100200062
:10bc10000e0078006c1607000000eb00100f980073
:10bc20000040eb0040579800e80047001e089000d5
:10bc300000804000341607000000e00008003200d9
:10bc4000e80047001e089000008040001040780087
:10bc5000405798001e0890000000e800100f980060
:10bc60004e509000e34f5000efff3a00680047004d
:10bc7000304090000000fb00e60040001e089000ed
:10bc8000810f5000e8ff3500e80047001e089000d3
:10bc9000808040000040eb00804878000000eb000e
:10bca000400f98006800470020409000ed4f500082
:10bcb00002003a0011002000410f98000001eb0043
:10bcc000520f980068004700604090000004e000b8
:10bcd0000200320010002000500f9800ce089000a3
:10bce0005e099000028060000000e0000500320064
:10bcf00068004700604090000000fb00300f980093
:10bd000036003700000000000000eb00100f980024
:10bd1000e80047001e08900000804000fa15070068
:10bd20000000e00008003200e80047001e08900014
:10bd30000080400010407800405798001e08900096
:10bd40000000e800100f98004e509000e34f5000a4
:10bd5000efff3a0068004700304090000000fb0011
:10bd6000e60040001e089000810f5000e8ff3500fb
:10bd70000000eb00600f98006800470090409000c2
:10bd800090c6b30080cf50000200320011002000a6
:10bd9000610f98000001eb00720f980068004700e7
:10bda000a040900010c5b30080cf500002003200c8
:10bdb00010002000700f9800ee0890007e0990009f
:10bdc000028060000000e000cfff3a0068004700fa
:10bdd000604090000000fb00300f98003e0890008b
:10bde0000080fa00000006008a00fa00000f7800c8
:10bdf00021479800e400470020c0b3008048780045
:10be0000e400470020c5b30090409800e4004700dc
:10be1000f0c0b300a0409800e40047002e4090001e
:10be200063404000b0409800e40047000040eb0051
:10be3000c0409800e401470064004700e400470068
:10be40001041900021409000804041006400470074
:10be50003040900000c04000d0419800e40047000e
:10be600010c0b300e040980064004700ae4090006e
:10be700071409800e40047000040eb0080489800c3
:10be80000000eb00308798002e4090008000fb00ff
:10be90003e809000810f50000b003d00e400470001
:10bea0003e80900000804000e90040003e8090000d
:10beb0001e004000904878003e8090000000e8009e
:10bec00030879800f0ff3700e40047002e409000d4
:10bed0000000fb0001004000e900400030c0b3005a
:10bee000804878002e4090000000fb00ea004000ef
:10bef00064004700b41507000000eb00308798008d
:10bf00000040eb00004f9900c10720008e804000e8
:10bf10003e809000008040007b1507000000e0009c
:10bf200009003200c10720008e8040003e80900052
:10bf30000080400010407800004f99003e80900043
:10bf40000000e800308798000e489100e34f500051
:10bf5000edff3a00c00720000e0040003040900086
:10bf60000000fb00e60040003e809000810f500082
:10bf7000e5ff3500c10720008e8040003e80900024
:10bf8000808040000040eb0080487800c00720001f
:10bf90000e004000604090000000fb000080fa00ae
:10bfa000000006004800fa0020c0b300004f7800ef
:10bfb00020c5b30010479800c0c1b30020479800c7
:10bfc0000040eb00304798000040eb0040479800ed
:10bfd000e0c6b3005047980030c0b30060479800f7
:10bfe000710020000e007800771507000000eb00bc
:10bff000102798000000eb00202798000040eb007d
:10c0000060c79800e80047002e20900000804000a4
:10c010003d1507000000e00008003200e80047007e
:10c020002e209000008040001040780060c79800eb
:10c030002e2090000000e800202798006ec090009d
:10c04000e34f5000efff3a00680047003040900097
:10c050000000fb00e60040002e209000810f500001
:10c06000e8ff350068004700704090000000fb00ca
:10c07000102798001e2090000000e00014003200fd
:10c080000000eb00202798009e2090006000200018
:10c090000088b9002e219000800f51000c003d0057
:10c0a0002e209000e1a7200001014000e800470099
:10c0b0002e20900000804000680040001049780069
:10c0c0002e2090000000e80020279800eeff3700a7
:10c0d0002ec090000000fb000080fa000000060067
:10c0e0001e00fa00000f78008e80e80020c0b30028
:10c0f000804878008e80e80020c5b300904098000a
:10c100008e80e800b0c1b300a04098008e80e800a7
:10c1100060c0b300b04098008e80e8000040eb00a3
:10c12000c04098008e80e80030c7b300d04098002f
:10c130000e81e8009e007800600020000008b80032
:10c14000e3a7200003004000104078006041980001
:10c150000e81e8009e007800600020000008b80012
:10c16000f3a72000030040001040780070419800c1
:10c170000e81e8009e007800600020000008b800f2
:10c1800003a82000030040001040780000499800f8
:10c190000e81e8009e007800600020000008b800d2
:10c1a00013a82000030040001040780010499800b8
:10c1b0000e81e8009e007800600020000008b800b2
:10c1c00023a8200003004000104078002049980078
:10c1d0000e81e8009e007800600020000008b80092
:10c1e00033a8200003004000104078003049980038
:10c1f0008e80e80030c0b300c04898000e80e80090
:10c20000d1002000f01407000000eb00500f980050
:10c210000040eb00405f9800f00047005e0890008f
:10c2200000804000b81407000000e0000800320061
:10c23000f00047005e089000008040001040780049
:10c24000405f98005e0890000000e800500f9800e2
:10c250004e589000e34f5000efff3a007000470047
:10c26000304090000000fb00e60040005e089000b7
:10c27000810f5000e8ff3500f00047005e08900095
:10c28000808040000040eb0080487800700047004c
:10c29000604090000000fb000080fa0000000600f3
:10c2a0001a00fa00004f78008e80e80020c0b3002a
:10c2b000804878008e80e80020c5b3009040980048
:10c2c0008e80e800e0c4b300a04098008e80e800b3
:10c2d00010c0b300b04098008e80e8000040eb0032
:10c2e000c04098008e80e80010cab300d04098008b
:10c2f0000e80e8009e407800614098008e80e80043
:10c3000030c0b300f04098000e80e80081002000ab
:10c31000ad1407000000eb00200f98000040eb0078
:10c320006057980010c0b3009e4f10000300340007
:10c330008000eb00410f9800220037000000000051
:10c34000ea0047002e089000008040006e140700ad
:10c350000000e00008003200ea0047002e089000cc
:10c360000080400010407800605798002e08900030
:10c370000000e800200f98006e509000e34f50003e
:10c38000efff3a006a004700304090000000fb00d9
:10c39000e60040002e089000810f5000e8ff3500b5
:10c3a000ea0047002e089000808040000040eb002b
:10c3b000804878006a004700604090000000fb0061
:10c3c000400f98004e0890000080fa000000060020
:10c3d0001600fa0020c0b300004f780020c5b3005b
:10c3e00010479800f0c4b300204798000040eb00cd
:10c3f000304798000040eb004047980010cab30057
:10c400005047980030c0b30060479800710020008a
:10c410000e0078006c1407000000eb00100f98006d
:10c420000040eb0040579800e80047001e089000cd
:10c4300000804000341407000000e00008003200d3
:10c44000e80047001e08900000804000104078007f
:10c45000405798001e0890000000e800100f980058
:10c460004e509000e34f5000efff3a006800470045
:10c47000304090000000fb00e60040001e089000e5
:10c48000810f5000e8ff3500e80047001e089000cb
:10c49000808040000040eb00804878006800470042
:10c4a000604090000000fb000080fa0000000600e1
:10c4b0002200fa00000f7800110798002207980068
:10c4c00033079800440798005507980066079800be
:10c4d000200d20001e0f40001e009000670040004d
:10c4e000100798005e0090000000e000030032009a
:10c4f0004e0090000000e00003003a008080eb0056
:10c50000610f9800ff0037002e0090009e00400051
:10c5100020352000808f5000030036000080eb00a3
:10c52000600f9800f70037009e0090003e009000da
:10c5300080804000701e2000808f50000300360075
:10c540008080eb00610f9800ee0037002e00900015
:10c550004e019000110009000280d8008000fd000b
:10c560000000e000030032000080eb00600f980044
:10c57000e40037003e0090005e01900011000900c9
:10c580000280d8008000fd000000e00003003200bf
:10c590008080eb00610f9800da0037005e009000a9
:10c5a000630060000000e0002e003a004e009000a2
:10c5b000630060000000e0000e003a00300320003d
:10c5c000500f98005e0090004200de00300f98008f
:10c5d0004e0090004200de00400f98001e009000c8
:10c5e00064005000100798001e007800640f50008f
:10c5f000460037004e009000610060000000e0003f
:10c600000d003a0010012000500f98005e009000cd
:10c610000000d100300f98004e0090000000d100c3
:10c62000400f98001e0090000080e900100798005d
:10c630001e8fe9003500370040042000500f98009d
:10c64000de009000310f98004e009000400f9800df
:10c650001e0090000000e900100798001e0fe9007e
:10c660002a0037005e009000610060000000e000da
:10c670001c003a004e009000610060000000e000e5
:10c680000d003a0010012000500f98005e0090004d
:10c690000000d100300f98004e0090000000d10043
:10c6a000400f98001e0090000080e90010079800dd
:10c6b0001e8fe9001500370040042000500f98003d
:10c6c000de009000310f98004e009000400f98005f
:10c6d0001e0090000000e900100798001e0fe900fe
:10c6e0000a00370040042000500f9800ce00900050
:10c6f000410f98005e009000300f98001e009000df
:10c700000000e900100798001e0fe9004e08900095
:10c710000000e900000f98003e0890000000e900ca
:10c72000700798002e0090004e0190001100090043
:10c730000280d800100f98003e0090005e0190002b
:10c74000110009000280d800200f98006e009000b0
:10c75000a00207000000e000030032008080eb0030
:10c76000610f9800670037005e089000bc02070068
:10c770000000e000030032000080eb00600f980032
:10c78000600037006e0090000000e0001b003a00df
:10c79000de089000710f980030032000fe08900022
:10c7a000808f50001200320030032000fe089000fd
:10c7b000808f500004003c007e089000f10f500074
:10c7c000080032002700370040042000fe089000d7
:10c7d000808f500023003a0000032000b5020700bc
:10c7e0002000370000022000b20207001d003700c1
:10c7f0000000eb00af0207001a0037005e0890004f
:10c8000000179800300320008e109000808f500099
:10c8100012003200300320008e109000808f5000f4
:10c8200004003c000e109000f10f50000800320090
:10c830000c003700400420008e109000808f5000c4
:10c8400008003a00000420009a02070005003700a3
:10c8500000032000970207000200370000022000ba
:10c8600094020700313520001e007800b402070052
:10c870000000e000030032000080eb00600f980031
:10c8800020003700811e20001e009000d402070007
:10c890000000e000030032008080eb00610f980090
:10c8a000180037001e01e800711e20001e009000d5
:10c8b000f20207000000e000030032000080eb00fd
:10c8c000600f98000f0037006e0090001000070006
:10c8d000000178007e0290008e0990009e08900072
:10c8e0002e089000fc0707000000e0000300320063
:10c8f0008080eb00610f9800020037000000eb0021
:10c90000600f98006e0890000080fa00000006009a
:10c910000600fa00000f78001e007800200798003b
:10c920002e009000e10f50000e0032002e0090000b
:10c93000e10f500004003c002e0090000000e000d9
:10c94000050032000d0037002e009000e20f50006d
:10c95000070032000900370010002000100798007f
:10c96000080037002000200010079800050037005d
:10c97000200020001007980002003700100020005f
:10c98000100798001e0090000080fa0000000600ca
:10c990002400fa00000f7800110798002207980081
:10c9a00033079800440798005507980066079800d9
:10c9b0001e007800700f40001e00900068004000cc
:10c9c000100798005e0090000000e00003003200b5
:10c9d0004e0090000000e00003003a008080eb0071
:10c9e000710f98001c0137002e0090009e0040003f
:10c9f000002d2000808f5000030036000080eb00e7
:10ca0000700f9800140137009e0090003e009000c7
:10ca100080804000801e2000808f50000300360080
:10ca20008080eb00710f98000b0137002e00900002
:10ca30004e019000110009000280d8008000fd0026
:10ca40000000e000030032000080eb00700f98004f
:10ca5000010137003e0090005e01900011000900c6
:10ca60000280d8008000fd000000e00003003200da
:10ca70008080eb00710f9800f70037005e00900097
:10ca8000630060000000e00034003a004e009000b7
:10ca9000630060000000e00010003a000008200081
:10caa000600f980040002000500f98005e0090003a
:10cab0004200de00300f98004e0090004200de0081
:10cac000400f98001e00900064005000100798006e
:10cad0001e007800640f5000500037004e00900098
:10cae000610060000000e0000f003a000004200038
:10caf000600f980020002000500f98005e0090000a
:10cb00000000d100300f98004e0090000000d100ce
:10cb1000400f98001e0090000080e9001007980068
:10cb20001e8fe9003d00370000022000600f9800d2
:10cb300010002000500f9800de009000310f980088
:10cb40004e009000400f98001e0090000000e90089
:10cb5000100798001e0fe900300037005e009000bb
:10cb6000610060000000e00020003a004e009000ec
:10cb7000610060000000e0000f003a0000042000a7
:10cb8000600f980020002000500f98005e00900079
:10cb90000000d100300f98004e0090000000d1003e
:10cba000400f98001e0090000080e90010079800d8
:10cbb0001e8fe9001900370000022000600f980066
:10cbc00010002000500f9800de009000310f9800f8
:10cbd0004e009000400f98001e0090000000e900f9
:10cbe000100798001e0fe9000c003700100020000d
:10cbf000500f980000022000600f9800ce009000b7
:10cc0000410f98005e009000300f98001e009000c9
:10cc10000000e900100798001e0fe9004e08900080
:10cc20000000e900000f98003e0890000000e900b5
:10cc3000700798002e0090004e019000110009002e
:10cc40000280d800100f98003e0090005e01900016
:10cc5000110009000280d800200f9800102d20003c
:10cc60005e099000110009000200d8008000fd005c
:10cc70001e0078005e099000811f780011000900f5
:10cc80000280d80001017800cf0078003706070045
:10cc90000000e000030032008080eb00710f98007c
:10cca0006d003700901e20005e0990001100090001
:10ccb0000200d8008000fd001e0090005e09900078
:10ccc000811f7800110009000280d800010178005e
:10ccd000cf0078004d0607000000e000030032009e
:10cce0000080eb00700f98005b003700811e200071
:10ccf0001e0090004b0607000000e0000300320019
:10cd00008080eb00710f9800530037006e00900098
:10cd10000000e0001d003a006e0890000017980027
:10cd2000000420008e109000808f5000110032000f
:10cd3000000420008e109000808f500005003c0001
:10cd4000000220008e109000808f500006003200fc
:10cd50002a003700000820008e109000808f5000bd
:10cd6000070032002500370000c9b3002305070083
:10cd70002200370000c5b300200507001f00370060
:10cd800000c1b3001d0507001c0037006e089000ad
:10cd900010179800000420009e109000808f500013
:10cda00011003200000420009e109000808f50007f
:10cdb00005003c00000220009e109000808f500073
:10cdc000060032000d003700000820009e10900081
:10cdd000808f5000070032000800370000cbb300fe
:10cde000060507000500370000c9b300030507006a
:10cdf0000200370000c5b30000050700ce589000c0
:10ce00004e489000a90507000000e0000300320032
:10ce10000080eb00700f98000f0037006e0090004c
:10ce200010000700000178007e0290008e0990003b
:10ce30009e0890002e089000a70607000000e00062
:10ce4000030032008080eb00710f98000200370071
:10ce50000000eb00700f98007e0890000080fa0040
:10ce6000000006000600fa00000f78001e0078009f
:10ce7000200798002e009000e10f50000e003200b5
:10ce80002e009000e10f500004003c002e009000a6
:10ce90000000e000050032000d0037002e00900079
:10cea000e20f500007003200090037001000200098
:10ceb0001007980008003700200020001007980095
:10cec00005003700200020001007980002003700fe
:10ced00010002000100798001e0090000080fa004b
:10cee000000006001200fa00000f780011079800f9
:10cef00022079800330798004407980055079800c8
:10cf000066079800a0908000000f9800000323009f
:10cf10008e089000808f500005003200000326002c
:10cf20008e089000808f50000b00320014003700f4
:10cf30006e039000de0290004e029000be01900051
:10cf40002e0190009e0090001e00780058fd070002
:10cf5000700798000c0037006e039000de0290000e
:10cf60004e029000be0190002e0190009e009000a5
:10cf70001e00780086fe0700700798000200370048
:10cf80000080eb00700798007e0090000080fa009f
:10cf9000000006000600fa00000f78001107980054
:10cfa000a09080002007980000032300ae009000ae
:10cfb000808f50000500320000032600ae00900074
:10cfc000808f500005003200070037009e0090005f
:10cfd0001e00780061010700030037009e009000ea
:10cfe0001e007800ed0507000080fa000000060032
:10cff0000000fa00a190800000032300808f500001
:10d0000001003a00490007000080fa000000060015
:10d010000400fa00ba1007006c090700d1a2a900a9
:10d0200040062000000f78001e00e00003003200e0
:10d03000000000001e0fe900fbff3700d1a2a8008e
:10d0400040062000000f78001e00e00003003200c0
:10d05000000000001e0fe900fbff370081e0a9007f
:10d06000f1048000f0002f000080600001662000c5
:10d0700001004000f00488008040eb00c0cdb30008
:10d080005e0907002047980011c0b300c0cdb3006f
:10d090005a090700304798002e4090000080fb009e
:10d0a000c800dd003e4090000080fb000080700062
:10d0b000a09088000080fa000000060000a0fe009a
:10d0c00086a0a9001421ef0000000000116280007a
:10d0d000c2c4200013002000321ce1000500320011
:10d0e0000800350000000000000000000000000003
:10d0f000f9ff3700a01680004800de008058780055
:10d10000f5ff370011628800482cec004062800077
:10d110004a0ce30003003a0010002000206288005f
:10d120001fe1a9000080fe00004006000200fa0096
:10d130002a0907000000eb00000f7800700d2000a6
:10d140009e0f10000a003e0071ec20001e8040007f
:10d1500062ec20009e004100104178009140780070
:10d16000c0cdb3005c0907001e8fe800f3ff370055
:10d170001e0907000080fa00000006000200fa0005
:10d18000881f7800150907000000eb00000f7800e9
:10d19000700d20009e0f10000a003e0070ec200071
:10d1a0001e04400061ec20001e804000904078008a
:10d1b000c0cdb30011090700004c78001e8fe800b5
:10d1c000f3ff3700090907004f0478000080fa00d8
:10d1d000000006000600fa00000f78001e0078002c
:10d1e000200798002e009000e10f50000e00320042
:10d1f0002e009000e10f500004003c002e00900033
:10d200000000e000050032000d0037002e00900005
:10d21000e20f50000700320009003700c0c0b30021
:10d2200009efb7000900370080c0b30009efb7006d
:10d230000600370020c0b30009efb7000300370035
:10d240000080eb0010079800020037000000eb00a0
:10d25000100798001e0090000080fa0000000600f1
:10d260000400fa00000f7800400420009e0f100018
:10d2700006003200100120009e0f10000300320053
:10d28000300320009e0f100005003a001e40780079
:10d29000f9eeb7000000eb0010079800020037001d
:10d2a0000080eb00100798001e0090000080fa003c
:10d2b000000006000400fa00000f78001e00e000e5
:10d2c00015003200000220009e0f100012003200f4
:10d2d000000320009e0f10000f0032000004200009
:10d2e0009e0f10000c003200000520009e0f100061
:10d2f00009003200000620009e0f100006003200d8
:10d30000000620009e0f10000300320000012000e4
:10d310009e0f100005003a001e407800f3eeb700a3
:10d320000000eb0010079800020037000080eb00bf
:10d33000100798001e0090000080fa000000060010
:10d340000a00fa00000f7800110798001e009000f4
:10d350009e0f1000030039000080eb00400798008a
:10d360001c0037009e00900030382000808f500055
:10d37000030036000080eb004007980015003700de
:10d380001e0fe9001e407800504798001e007800ec
:10d390004800de00404798002e40900070479800fb
:10d3a0001e0090004800de00604798004e4090004c
:10d3b000cfeeb7005e409000d1eeb7006e40900017
:10d3c000d7eeb7007e409000d9eeb7000000eb002a
:10d3d000400798004e0090000080fa000000060010
:10d3e0000a00fa00000f7800110798001e00900054
:10d3f0009e0f1000030039000080eb0040079800ea
:10d400001b0037009e009000301f2000808f5000ce
:10d41000030036000080eb0040079800140037003e
:10d420001e407800504798001e0078004800de003b
:10d43000404798002e409000704798001e009000d2
:10d440004800de00604798004e409000d3eeb700e1
:10d450005e409000d5eeb7006e409000dbeeb70066
:10d460007e409000ddeeb7000000eb004007980022
:10d470004e0090000080fa00000006000e00fa0046
:10d48000000f780011079800220798001e009000f6
:10d490009e0f1000030039000080eb006007980029
:10d4a0002b0037009e009000301f2000808f50001e
:10d4b000030036000080eb0060079800240037006e
:10d4c000ae00900030382000808f500003003600fe
:10d4d0000080eb00600798001d0037001e407800b8
:10d4e000704798001e0078004800de0060479800f2
:10d4f0002e409000104f98001e0090004800de0063
:10d50000004f98004e409000204f98002e00900051
:10d510004800de00304f98006e40900057efb70093
:10d520007e40900059efb7000e4890005befb700c7
:10d530001e4890005defb7003e4890005fefb700d7
:10d540002e48900061efb7000000eb0060079800e4
:10d550006e0090000080fa00000006000600fa004d
:10d56000000f7800110798001e00e000060032004e
:10d570001e0090000000e00003003200a0ccb300c9
:10d58000404798000d0037001e00e0000300320005
:10d59000a0c4b30040479800080037001e00900068
:10d5a0000000e00003003200a0c8b300404798002c
:10d5b00002003700a0c0b300404798004e409000e2
:10d5c000f5eeb7000080fa00000006000600fa0041
:10d5d000004f7800114798000000eb0010079800fa
:10d5e0009e009000700d2000808f500012003e00c1
:10d5f0001e00900061ec2000010040001040780007
:10d600009e4f500008003a001e00900071ec200070
:10d61000010040009e409000014878000000eb00af
:10d6200020079800060037001e0090000080e800e8
:10d6300010079800eaff37008080eb002107980070
:10d640002e0090000080fa00000006000800fa009a
:10d65000004f7800110798000000eb0020079800a9
:10d66000ae009000700d2000808f500012003e0030
:10d670002e00900061ec2000010040001040780076
:10d680009e4f500008003a001e009000ae0090002f
:10d6900072ec200082804000114878000000eb000e
:10d6a00030079800060037002e0090000080e80048
:10d6b00020079800eaff37008080eb0031079800d0
:10d6c0003e0090000080fa00000006000200fa0010
:10d6d000004f7800114798001e409000dfeeb70021
:10d6e0001e407800e1eeb7000080fa00000006005e
:10d6f0000800fa00004f7800114798002247980070
:10d700003347980044479800f0c4b3009e4f100080
:10d71000030036000080eb00300798000c00370053
:10d720001e407800e3eeb7001e409000e5eeb70023
:10d730002e409000e7eeb7004e409000e9eeb700b3
:10d740003e409000ebeeb7000000eb003007980081
:10d750003e0090000080fa00000006000400fa007d
:10d76000008fbe001e00be004a09dd004600de003c
:10d7700000007100c608de00efeeb7001e00be001c
:10d780004209dd004e00de0000007100ce08de0020
:10d79000edeeb7000040eb00f1eeb7000080fa00bc
:10d7a000000006000200fa00004f78001e407800da
:10d7b000fbeeb7000080fa00000006000200fa004d
:10d7c000000f78001e00e000050032000bcfbf0004
:10d7d00001c8b300014070000befb7000300370031
:10d7e0000bcfbf000074a1000befb7000080fa0060
:10d7f000000006000400fa00004f7800114798006e
:10d80000224798001e4078000fefb7001e4090009e
:10d8100011efb7002e40900013efb7000080fa0020
:10d82000000006000200fa00004f7800114798003f
:10d830009e4078007fc060000045b00015efb70043
:10d840001e40900017efb7000080fa0000000600ad
:10d850000600fa00000f7800214798002e40900043
:10d860000000fb0063006000c500dd0000c8b300dd
:10d8700000c040009defb7000000eb0020079800bb
:10d880002e009000e10f50000b003e002e00900093
:10d890000000d00092f12000820040002e00900095
:10d8a0001e004000904878002e0090000000e80024
:10d8b00020079800f2ff37000080fa000000060001
:10d8c0000000fa0045070700d2f920001241780055
:10d8d000c1f9200091407800c0cdb3007e07070059
:10d8e00042070700e1f220009140780018cfbf0006
:10d8f000020007000080fa00000006000600fa009f
:10d90000004f7800114798000000eb0020079800b6
:10d91000320707000000eb00100798009e009000ff
:10d92000700d2000808f50001d003e001e009000f2
:10d9300061ec200001004000104078009e4f500034
:10d94000130039001e00900062ec200082004000ad
:10d950001e409000914f10000d003e001e009000f0
:10d9600072ec2000820040001e00900062ec20005b
:10d97000020040001141780090407800c0cdb30013
:10d98000550707002e0090000000e80020079800cf
:10d990001e0090000080e80010079800dfff3700ad
:10d9a000120707002e0090000080fa000000060019
:10d9b0000400fa00000f78000000eb001007980048
:10d9c0001e009000e10f50000b003e001e00900072
:10d9d0000000d00012f32000820040001e009000e2
:10d9e0001e004000904878001e0090000000e800f3
:10d9f00010079800f2ff37000080fa0000000600d0
:10da00000200fa00004f7800114798001e4078008d
:10da100043efb7001e40900045efb7000080fa00ca
:10da2000000006000200fa00004f7800114798003d
:10da30001e40780047efb7001e40900049efb70046
:10da40000080fa00000006000200fa00004f780093
:10da5000114798001e4078004befb7001e40900021
:10da60004defb7000080fa00000006000200fa0047
:10da7000004f78001e80fb004400dd006f40400036
:10da800063efb7000080fa00000006000200fa0011
:10da9000004f7800114798001e80fb00c400dd0095
:10daa0001e4090006f40600000c0400065efb7006e
:10dab0000080fa00000006000200fa00004f780023
:10dac000114798001e4090000080fb00c400dd005c
:10dad0001e4178006f40610000c0400067efb70052
:10dae0000080fa00000006000400fa00008fbe006b
:10daf0001e00be004088de00cf80de0069efb70068
:10db00001e00be004809dd004800de000000710074
:10db1000c888de006befb7001e4078006defb700dd
:10db20000080fa00000006000200fa00004f7800b2
:10db30001e4078006fefb7000080fa00000006007a
:10db40000400fa00000f7800110798001e0078000a
:10db50004800de0075efb7001e40780077efb70091
:10db60001e0090004800de0079efb7002e409000c4
:10db70007befb7000080fa00000006000600fa0004
:10db8000004f7800114798002247980033479800cb
:10db900044479800554798002e4090007defb7000d
:10dba0003e4090007fefb7001e40780081efb70045
:10dbb0001e40900083efb7004e40900085efb70005
:10dbc0005e40900087efb7000080fa00000006007a
:10dbd0000a00fa00000f7800110798002207980049
:10dbe00033079800200d20001e0f40001e009000fb
:10dbf000200db000100798002e0090006700400034
:10dc0000200798003e009000670040003007980011
:10dc10009e00900020352000808f500003003600c9
:10dc20000080eb004007980039003700be009000ec
:10dc3000701e2000808f5000030036000080eb0033
:10dc400040079800320037001e0090009e0f100021
:10dc500004003100ae0090003e009000808f500024
:10dc6000030039000080eb004007980028003700cf
:10dc7000501a20009e0f10000c0036009e009000ed
:10dc800090272000808f500008003e00ae009000da
:10dc9000700a2000808f500004003600be00900003
:10dca00060142000808f5000030036000080eb00dd
:10dcb00040079800160037001e0078004800de007c
:10dcc00089efb7001e4078008befb7001e00900070
:10dcd0004800de008defb7002e4090008fefb700b8
:10dce0002e0090004800de0091efb7004e409000fb
:10dcf00093efb7003e0090004800de0095efb700bc
:10dd00006e40900097efb7000000eb0040079800ce
:10dd10004e0090000080fa00000006000600fa00a5
:10dd2000000f7800110798001e00e0000600320086
:10dd30001e0090000000e00003003200c0c3b300ea
:10dd4000404798000d0037001e00e000030032003d
:10dd5000c0c2b30040479800080037001e00900082
:10dd60000000e00003003200c0c1b300404798004b
:10dd700002003700c0c0b300404798004e409000fa
:10dd800099efb7000080fa00000006000200fa00d8
:10dd9000000f78001e00e00006003200f0c7b3005c
:10dda000d1ef20009140780000c06000fdeeb70088
:10ddb00004003700fdcebf0001c8b3000140700071
:10ddc000fdeeb7000080fa00000006000400fa0033
:10ddd000000f7800110798001e00e00005003200d7
:10dde000fdcebf00f1cbb30001406000fdeeb700f7
:10ddf00004003700fdcebf0001c4b3000140700035
:10de0000fdeeb7001e0090000000e00005003200ab
:10de1000fdcebf00f1cdb30001406000fdeeb700c4
:10de200004003700fdcebf0001c2b3000140700006
:10de3000fdeeb7000080fa00000006000a00fa00bc
:10de4000f3cebf000080fb004007980000032000d5
:10de5000ce009000808f500035003200000320007b
:10de6000ce009000808f50000f003c004e009000cc
:10de7000f00f500026003200ce009000f08f5000ce
:10de800004003c004e0090000000e0001c00320046
:10de90003b00370000022000ce009000808f500031
:10dea0001f0032003600370000052000ce00900031
:10deb000808f50002600320000052000ce00900028
:10dec000808f500005003c0000042000ce00900030
:10ded000808f50001a003200290037000006200011
:10dee000ce009000808f50001d00320000072000ff
:10def000ce009000808f50001d00320020003700bf
:10df00000000280001072000008fbe00200037001d
:10df10000000200061092000008fbe001c003700b7
:10df20000000240081032000008fbe00180037008d
:10df300000002200c1012000008fbe001400370045
:10df400000002100e1002000008fbe00100037001b
:10df50000080200071002000008fbe000c00370000
:10df60000040280031002000008fbe00080037006c
:10df700000202c0011002000008fbe00040037009c
:10df80006000b800200798003107980013003700a0
:10df900090f02000c1c0b30090cf10000c003a00f8
:10dfa0001e01be00200020000012b8000000eb009f
:10dfb0000093b90085007800868040000300780057
:10dfc0000000d0008080400081027800048fbe00f5
:10dfd0001e00be0020079800310798002e00900018
:10dfe000be0090000080fa00000006001000fa0059
:10dff000000f780011079800220798003307980057
:10e00000440798003e0090000000e0000300350047
:10e010003e009000e30f5000030034000080eb004e
:10e02000700798004b0037004e0090000000e000a1
:10e03000030035004e009000e30f50000300340051
:10e040000080eb0070079800420037007bff07005c
:10e05000626a20000203b8000001eb000282b900ee
:10e060000701780004014100636a20000388b900b9
:10e0700000014100820378001e0078006101b900b0
:10e080000600be000dd90700500798006bff07007f
:10e09000626a20000203b8000001eb000282b900ae
:10e0a0000701780004014100636a20000388b90079
:10e0b00000014100820378001e0090006101b90058
:10e0c0000600be00fdd80700600798005e009000c3
:10e0d0004800de0001efb7002e48900003efb700c4
:10e0e0006e0090004800de0005efb7004e4890003b
:10e0f00007efb7002e0090000000e000040032009f
:10e10000fdcebf000044a000fdeeb70004003700c4
:10e11000fdcebf00f1ceb30001406000fdeeb700c0
:10e120000e489000e34060003e00900063006000f5
:10e130004200dd0000c1400001cfb300fdcebf00b2
:10e1400000c0600000404100fdeeb7000000eb00a1
:10e15000700798007e0090000080fa000000060022
:10e160000200fa00004f78001c0507001e417800ed
:10e1700031c0b300c0cdb300570507001b05070031
:10e180000080fa00000006000400fa00004f78004a
:10e1900011479800224798001e407800f0ff0700c2
:10e1a0000e0507002e4190009e409000c0cdb300a8
:10e1b000490507000d0507000080fa000000060071
:10e1c0000400fa00004f7800114798001e407800c4
:10e1d000e3ff0700010507009e409000c0cdb3009b
:10e1e0000605070020479800000507002e40900014
:10e1f0000080fb000080fa00000006000200fa0028
:10e20000004f78001e41780011c9b3000040eb00b8
:10e21000ddff07000080fa00000006000200fa009f
:10e22000004f78001e41780081c6b30010c0b300d3
:10e23000d5ff07000080fa00000006000600fa0083
:10e24000004f78001e80fb0020079800000420008b
:10e25000ae009000808f50001f00320000042000ac
:10e26000ae009000808f500005003c0000022000ae
:10e27000ae009000808f500006003200380037005a
:10e2800000082000ae009000808f50002300320074
:10e290003300370010c0b300e0ff07001e417800d4
:10e2a00001c8b30010c0b300b7ff07001e417800db
:10e2b00011c8b30010c0b300b3ff070012c0b30011
:10e2c00021c8b30010c0b300afff07000000eb008f
:10e2d000100798002400370030c0b300cfff0700bc
:10e2e0001e41780001c8b30010c0b300a6ff0700ac
:10e2f0001e41780011c8b30010c0b300a2ff070090
:10e3000012c0b30021c8b30010c0b3009eff0700c5
:10e310008000eb00110798001300370070c0b300b5
:10e32000beff07001e41780001c8b30010c0b30053
:10e3300095ff07001e41780011c8b30010c0b3005c
:10e3400091ff070012c0b30021c8b30010c0b30092
:10e350008dff07000000eb00100798000200370057
:10e360008080eb00110798001e0090000080fa00ea
:10e37000000006000600fa00004f78001e80fb0037
:10e380002007980000042000ae009000808f50000d
:10e390001f00320000042000ae009000808f50006b
:10e3a00005003c0000022000ae009000808f50006d
:10e3b000060032003800370000082000ae00900050
:10e3c000808f500023003200330037000040eb0004
:10e3d00092ff07001e41780001c8b30010c0b300cf
:10e3e00069ff07001e41780011c8b30010c0b300d8
:10e3f00065ff070012c0b30021c8b30010c0b3000e
:10e4000061ff07000000eb001007980024003700b0
:10e4100010c0b30081ff07001e41780001c8b3009f
:10e4200010c0b30058ff07001e41780011c8b300a8
:10e4300010c0b30054ff070012c0b30021c8b300de
:10e4400010c0b30050ff07008000eb0011079800d8
:10e450001300370030c0b30070ff07001e41780082
:10e4600001c8b30010c0b30047ff07001e41780089
:10e4700011c8b30010c0b30043ff070012c0b300bf
:10e4800021c8b30010c0b3003fff07000000eb003d
:10e4900010079800020037008080eb0011079800f9
:10e4a0001e0090000080fa00000006000600fa003e
:10e4b000004f7800114798001e80fb00200798004d
:10e4c0002e009000e10f5000130032002e0090004b
:10e4d000e10f500004003c002e0090000000e0001e
:10e4e000050032001c0037002e009000e20f5000a3
:10e4f0001100320018003700d2c0b30081c3b3004e
:10e5000010c0b30020ff07001e4090004bff070023
:10e51000100798001200370082c0b30081c3b30017
:10e5200010c0b30018ff07001e40900091ff0700c5
:10e53000100798000a00370022c0b30081c3b3005f
:10e5400010c0b30010ff07001e40900089ff0700b5
:10e5500010079800020037000080eb0010079800b9
:10e560001e0090000080fa00000006000a00fa0079
:10e57000000f7800110798001e0090009e0f1000f9
:10e58000030039000080eb00400798001c003700b2
:10e590009e009000f0312000808f50000300360074
:10e5a0000080eb0040079800150037001e0fe900bf
:10e5b0001e407800504798001e0078004800de009a
:10e5c000404798002e409000704798001e00900031
:10e5d0004800de00604798005e41900011c5b3001e
:10e5e00010c0b300e8fe07004e41900001c5b30023
:10e5f00010c0b300e4fe07000000eb0040079800e5
:10e600004e0090000080fa00000006000800fa00aa
:10e61000000f7800110798000000eb000080fa005e
:10e62000000006000a00fa00000f780011079800a9
:10e630001e0090009e0f1000030039000080eb00c8
:10e6400040079800230037009e009000301f2000f4
:10e65000808f5000030036000080eb0040079800d8
:10e660001c0037001e407800504798001e007800bc
:10e670004800de00404798002e4090007047980008
:10e680001e0090004800de00604798004e41900058
:10e6900001c6b30010c0b300bbfe07005e4190008e
:10e6a00011c6b30010c0b300b7fe07006e41900062
:10e6b00021c6b30010c0b300b3fe07007e41900036
:10e6c00031c6b30010c0b300affe07000000eb007e
:10e6d000400798004e0090000080fa0000000600fd
:10e6e0000200fa00000f780012c0b300a1c5b30009
:10e6f00020c0b300a4fe070012c4b30021c3b300be
:10e7000010c0b300a0fe07001e00e00011003a0098
:10e7100000c1eb0081c8b30010c0b3009afe07002f
:10e7200000c1eb0091c8b30010c0b30096fe070013
:10e7300082c0b300a1c8b30010c0b30092fe0700ae
:10e7400000c1eb00b1c8b30010c0b3008efe0700db
:10e750001000370002c2b30081c8b30010c0b3007c
:10e7600089fe070002c8b30091c8b30010c0b3000f
:10e7700085fe070082c0b300a1c8b30010c0b3007b
:10e7800081fe070000c1eb00b1c8b30010c0b300a8
:10e790007dfe07000080fa00000006000600fa0077
:10e7a000000f78001107980001c9b3000040eb008a
:10e7b00083fe0700404798001e00e000050032007d
:10e7c0004e40900001c8b3000140700040479800df
:10e7d00004003700f0c7b300ce40900000c06000d6
:10e7e000404798001e0090000000e0000500320045
:10e7f0004e40900001c4b3000140700040479800b3
:10e80000040037004e409000f1cbb300014060009f
:10e81000404798004e41900001c9b3000040eb0012
:10e8200059fe07000080fa00000006000000fa0010
:10e8300086c0a9001fe1a80021e1a9000080fa001c
:10e84000004006000000fa002000200000098800b7
:10e850000000eb00c008880010002000e0088800dd
:10e8600086c0a9008ec0a80021e1a8000080fa009f
:10e87000000006000000fa0020002000f0088800d8
:10e8800030628000a0088800306280000000e8004c
:10e89000d008880086a0a9001fe1a9008ea0a800ca
:10e8a0000080fa00000006000200fa00000f780065
:10e8b0000000eb00406288001e00780010628800b3
:10e8c0000000eb0020628800eaff0700ddff070080
:10e8d0000080fa00000006001200fa00000f780025
:10e8e0001107980022079800330798004407980002
:10e8f0000000eb00600798009e0090002e00900042
:10e900000089b9003e0090000000e8000280b900d4
:10e910008000e800a0142000808f50000300360023
:10e920000080eb00000f98003d0037000000eb0076
:10e9300050079800de0090001e009000808f50006d
:10e940002c003d000000eb0070079800fe009000d6
:10e950002e009000808f50000d003d00ec0147001c
:10e960009300780001007800c4c420000401400036
:10e9700010c0b300004978008100e80081097800e8
:10e980007e0090000000e80070079800efff37005d
:10e990000000eb0070079800be0090002e00900071
:10e9a0000088b9007e019000800f51000d003d00ed
:10e9b000ec0147009300780001007800c4c42000f7
:10e9c000040140000040eb00004978008100e800ad
:10e9d000810978007e0090000000e8007007980030
:10e9e000edff37005e0090000000e800500798003f
:10e9f000d0ff37006e009000c2c4200082004000ab
:10ea000020c0b300804878004e0290003462880035
:10ea10001e007800506288000001eb00020f980091
:10ea20000e0890000080fa00000006000000fa00c6
:10ea3000206280000080fa0000000600811f78003c
:10ea4000801f7800f0ff2700c012880000302000ef
:10ea50000000b300d0128800de02a9000000000010
:10ea6000e002a9009001090000000000e002a800f7
:10ea700041e2a8004602ae00feff3700f0ff27008b
:10ea8000c0128800004020003001b300d01288007e
:10ea90004602ae00feff3700f0ff2700c0128800dc
:10eaa000001020000030a0000040a000d01288001c
:10eab0004602ae00feff3700f0ff2700c0128800bc
:10eac00000202000d01288004602ae00feff370072
:10ead000f0ff2700c0128800006020000010a00096
:10eae000d01288004602ae00feff3700f0ff27007c
:10eaf000c012880000702000f005b300d01288001a
:10eb00004602ae00feff370001f020003012800008
:10eb1000010060000000e000fcff3a0030128000bd
:10eb2000010060000000e000fcff320030128000b5
:10eb3000010060000000e000fcff3a00301280009d
:10eb4000010060000000e000fcff32004662ae0001
:10eb500002003700801280009012800041e2a9007c
:10eb6000f01e2000101288004362a8004342a80053
:10eb70008920a900a8c0a800a8a0a900a880a90071
:10eb80009120a80041e2a8004f007800cf00780053
:10eb900000000600801f78004022ef004222ef00b4
:10eba0004422ef004822ef004c22ef00c6e2a8000a
:10ebb000e5a2a900e582a800e5e2a900e5c2a90056
:10ebc0004002a9004022a90040a2a9004122a900b8
:10ebd00040c2a8004102a9004142a900f00e200055
:10ebe000101288004362a9004342a80030002000b0
:10ebf000201288004c02a8004802a8008920a90021
:10ec00009120a90041e2a9004f0078000000060011
:10ec10008920a900809fbe00829fbe0080128000d4
:10ec200090128000a0128000b0128000d811e20083
:10ec300026003a00dc11e200240032003400f80023
:10ec40004400f8004440a800f08e8000a001880035
:10ec5000b190800070760200000000001100780082
:10ec60000000a100c01288007076020000000000c1
:10ec7000110078000000a100d01288007076020018
:10ec800000000000110078000000a100e0128800e0
:10ec90007076020000000000110078000000a10062
:10eca000f0128800dcb1ed00dcb1ed00b19088001d
:10ecb000a1018000f18e88004400f9003400f900c1
:10ecc0004f01be004f00be0000400600da31ef00e9
:10ecd000d8b1ef004f01be004f00be00004006005b
:10ece000e280400004003900a1018000e180400082
:10ecf000a101880001002800000006000200fa00bf
:10ed0000e202a8000000eb00000f7800f070220083
:10ed10009e0f100002003c001e0fe800fbff3700b2
:10ed20009cff070045ff07000080fa000000060076
:10ed30000400fa00000f780011079800dab1ef0024
:10ed4000d831ef009e0090001e00780006000700fa
:10ed50000080fa00000006000000fa00e202a900ac
:10ed60000080fa0000000600811f7800821f7800f2
:10ed70004100dd00030037004f017800cf0078002c
:10ed800000000600e18e88000001eb00a1ea2900e6
:10ed9000810040000300390002002800828040000a
:10eda000120020004400f8003400f8004440a8009d
:10edb0001000200002004000a001880000000000b8
:10edc0001c77020000000000110078000000a10084
:10edd000c01288001c7702000000000011007800bb
:10ede0000000a100d01288001c7702000000000083
:10edf000110078000000a100e01288001c770200da
:10ee000000000000110078000000a100f01288004e
:10ee1000dcb1ed00dcb1ed00b1908800a101800013
:10ee2000f18e88003400f900000000004400f90071
:10ee30008920a900d0ff3700e2804000040039009b
:10ee4000a1018000e1804000a101880001002800ac
:10ee5000000006000000fa000000000006c2bf002b
:10ee60000080fb00610060000000e000fbff3a0052
:10ee700006c2bf000080fb004200de000080fb00f5
:10ee8000610060000000e000f4ff3a0006c2bf002d
:10ee90000080fb004300de000080fb00610060009a
:10eea0000000e000edff3a0006c2bf000080fb005a
:10eeb0004400de000080fb00610060000000e00014
:10eec000e6ff3a0009c2bf000080fb004600de00fa
:10eed0000080fb00610060000000e000dfff3a00fe
:10eee0000080fa00000006000400fa00600920001b
:10eef0002010880007e2a90007e2a80085c0a90049
:10ef000085a0a900b10920009140780080cfb3000e
:10ef100000c060005040b3009be0b7008da0a90086
:10ef20000071220001002000008fbe001e00be0004
:10ef3000e00f5000e08f5800050032000080eb0029
:10ef40008080eb001e0f40005e974800f7ff3700ff
:10ef5000100020000080fa00000006000400fa0003
:10ef60006000b800008fbe0007e2a90085c0a900bc
:10ef700085a0a9008da0a900007122000100200039
:10ef8000008fbe001e00be00e00f5000e08f580052
:10ef9000050032000080eb008080eb001e0f400077
:10efa0005e974800f7ff3700cfff07000f0007000c
:10efb0000071220001002000008fbe001e00be0074
:10efc000e00f5000e08f5800050032000080eb0099
:10efd0008080eb001e0f40005e974800f7ff37006f
:10efe000100020000080fa00000006000000fa0077
:10eff00085c0a9008dc0a800100020000080fa0084
:10f00000000006000000fa0085c0a9008dc0a9001c
:10f01000100020000080fa00000006000600fa0040
:10f0200010c0b300e0f1b70008c2bf000080fb00d1
:10f030004400de000080fb00610060000000e00092
:10f04000150032000602a800007122000100200015
:10f05000008fbe001e00be00e00f5000e08f580081
:10f060000a003200e051e20003003a0010002000e4
:10f07000200798000a0037000080eb008080eb003a
:10f080001e0f40005e974800f2ff37008000eb0043
:10f0900021079800020037000000eb0020079800cd
:10f0a0002e0090000080fa00000006000600fa0022
:10f0b00060c0b300e0f1b70008c2bf000080fb00f1
:10f0c0004300de000080fb00610060000000e00003
:10f0d000150032000622a800007122000100200065
:10f0e000008fbe001e00be00e00f5000e08f5800f1
:10f0f0000a003200e051e20003003a001000200054
:10f10000200798000a0037000080eb008080eb00a9
:10f110001e0f40005e974800f2ff37008000eb00b2
:10f1200021079800020037000000eb00200798003c
:10f130002e0090000080fa00000006000600fa0091
:10f1400050c0b300e0f1b7000642a80000712200f1
:10f1500001002000008fbe001e00be00e00f500026
:10f16000e08f58000a003200e051e20003003a004c
:10f170001000200020079800070037000080eb00f7
:10f180008080eb001e0f40005e974800f2ff3700c2
:10f190008000eb00210798002e0090000080fa000c
:10f1a000000006000600fa0030c0b300e0f1b7002e
:10f1b00006c2bf000080fb00610060000000e000ac
:10f1c0001c003a0006c2bf000080fb004200de00c7
:10f1d0000080fb00610060000000e00015003a00c4
:10f1e00006c2bf000080fb004300de000080fb0081
:10f1f000610060000000e0000e003a0006c2bf009f
:10f200000080fb004400de000080fb006100600025
:10f210000000e00007003a0006c2bf000080fb00cb
:10f220000000d1000080fb00610060000000e000f1
:10f23000030032000000eb002007980015003700a3
:10f2400006a2a9000682a800007122000100200089
:10f25000008fbe001e00be00e00f5000e08f58007f
:10f260000a003200e051e20003003a0011002000e1
:10f2700021079800070037000080eb008080eb003a
:10f280001e0f40005e974800f2ff37008000eb0041
:10f29000210798002e0090000080fa000000060070
:10f2a0000600fa0030c0b300e0f1b70006c2bf00ac
:10f2b0000080fb00610060000000e0001c003a00dc
:10f2c00006c2bf000080fb004200de000080fb00a1
:10f2d000610060000000e00015003a0006c2bf00b7
:10f2e0000080fb004300de000080fb006100600046
:10f2f0000000e0000e003a0006c2bf000080fb00e4
:10f300004400de000080fb00610060000000e000bf
:10f3100007003a0006c2bf000080fb000000d100d9
:10f320000080fb00610060000000e000030032008c
:10f330000000eb00200798001500370006a2a80087
:10f340000682a8000071220001002000008fbe008c
:10f350001e00be00e00f5000e08f58000a0032008f
:10f36000e051e20003003a0011002000210798005c
:10f37000070037000080eb008080eb001e0f40008c
:10f380005e974800f2ff37008000eb0021079800ed
:10f390002e0090000080fa00000006000c00fa0029
:10f3a000000f780000712200010020001007980073
:10f3b000210798000040eb006047980040c0b30070
:10f3c000e0f1b70000712200010020001007980052
:10f3d000210798001e009000ae009000e00f500042
:10f3e000e08f58002b00320006c2bf000080fb00f7
:10f3f000610060000000e0001f003a0006c2bf008c
:10f400000080fb004200de000080fb006100600025
:10f410000000e00018003a0006c2bf000080fb00b8
:10f420004300de000080fb00610060000000e0009f
:10f4300011003a0006c2bf000080fb004400de005d
:10f440000080fb00610060000000e0000a003a005c
:10f4500009c2bf000080fb004600de000080fb0008
:10f46000610060000000e00003003a0010c0b3003b
:10f4700060479800070037001e009000ae00900023
:10f4800061005000e08058001007980021079800a4
:10f49000d0ff37006e4090000004e00003003a0007
:10f4a0000000eb00400798001d0037000662a8002e
:10f4b000006a28001100200010079800210798001a
:10f4c0001e009000ae009000e00f5000e08f58004a
:10f4d00011003200e051e20008003a009e0078007e
:10f4e0005107980000c2bf00de00900080487800fd
:10f4f0001000200040079800090037001e0090000f
:10f50000ae00900061005000e080580010079800a5
:10f5100021079800eaff37008000eb0041079800c0
:10f520004e0090000080fa00000006000800fa007b
:10f53000004f780020c0b300e0f1b7001e40780013
:10f5400002e2b700007122000100200010079800bd
:10f55000210798001e009000ae009000e00f5000c0
:10f56000e08f58000c003200e051e20003003a0046
:10f570001000200030079800090037001e0090009e
:10f58000ae00900061005000e08058001007980025
:10f5900021079800efff37000000eb0030079800cc
:10f5a0003e0090000080fa0000000600801f7800f6
:10f5b0000000fa0085c0a9000040eb00e0f1b700b0
:10f5c0000080fa004f007800004006000000fa00ba
:10f5d00045fe07000080fa00000006000000fa0067
:10f5e00082fe07000080fa00000006000000fa001a
:10f5f00084fe07000080fa00000006000400fa0004
:10f60000004f7800114798000040eb002047980019
:10f610002e4090000004e0002b003a0010c0b30020
:10f62000204798007dfe0700804078002e40900023
:10f6300001406000204798001e407800bbff070093
:10f64000804078002e4090000140600020479800e4
:10f650001e409000b5ff0700804078002e409000cb
:10f66000014060002047980090fe0700804078002d
:10f670002e40900001406000204798001e40e800a6
:10f68000aaff0700804078002e40900001406000f3
:10f69000204798006300470040ff07008040780043
:10f6a0002e4090000140600020479800fcfe0700bb
:10f6b000a2fe07002e4090000004e00002003a0085
:10f6c00026fe0700d2ff37003e4090000000fb00fe
:10f6d0000080fa00000006000400fa00004f7800e5
:10f6e00011479800224798000040eb0030479800ef
:10f6f0003e4090000004e00023003a0010c0b30038
:10f700003047980045fe0700804078003e4090005a
:10f7100001406000304798001e40780083ff0700da
:10f72000804078003e4090000140600030479800e3
:10f730001e4090007dff0700804078003e40900012
:10f7400001406000304798002e40900077ff07008e
:10f75000804078003e4090000140600030479800b3
:10f7600076fe0700804078003e4090000140600037
:10f77000304798003e4090000004e00002003a004c
:10f78000f6fd0700daff37003e4090000000fb0066
:10f790000080fa00000006000000fa000000eb0004
:10f7a000800888000111200091407800f0ccb3005f
:10f7b00000c0600010e1b7000000eb0030088800d6
:10f7c000205c20006008880084c0a9008cc0a800cc
:10f7d00011e1a8000080fa00000006000000fa0015
:10f7e00011e1a9000080fa00000006000800fa00fc
:10f7f000000f780011079800c09080002007980043
:10f800002e0090000000e0000b0032002e0090005f
:10f81000300090009e0f500003003a0011002000bd
:10f82000310798001f0037002e0090004000900024
:10f8300020079800f2ff3700a000200092c30700c5
:10f84000200798002e0090000000e00002003a001f
:10f8500010002000ddc307002e0090009e009000e5
:10f8600001087800ae0090000000eb0090009800c6
:10f87000ae00900010c0b300c04098002e00900071
:10f880009e007800310098002e009000c19080000a
:10f89000410098002e009000c090880011002000c8
:10f8a000310798003e0090000080fa00000006003a
:10f8b0000800fa00000f78000000eb001007980025
:10f8c000c0908000200798002e0090000000e0000b
:10f8d0001a0032002e009000300090009e0f500061
:10f8e00010003a001e0090000000e0000500320009
:10f8f0009e0090002e00900040009000c0009800f4
:10f90000030037002e00900040009000c090880057
:10f910002e009000bfc307001000200030079800a1
:10f92000080037002e009000100798002e0090006d
:10f930004000900020079800e3ff370020002000df
:10f94000300798003e0090000080fa00000006009a
:10f950000800fa00000f780011079800c09080009e
:10f96000200798002e0090000000e0000e003200fa
:10f970002e009000300090009e0f500006003a00cc
:10f980002e0090009e0090000108780010002000da
:10f9900030079800060037002e00900040009000cd
:10f9a00020079800efff3700210020003107980062
:10f9b0003e0090000080fa00000006000600fa00f9
:10f9c000000f7800c0908000100798001e00900083
:10f9d0000000e0000e0032001e0090003000900099
:10f9e0009e0f500006003a009e0090000000eb00c1
:10f9f00090009800100020002007980006003700b3
:10fa00001e0090004000900010079800efff3700a4
:10fa100020002000200798002e0090000080fa00af
:10fa2000000006000600fa00000f7800c090800079
:10fa3000100798001e0090000000e0000e00320049
:10fa40001e009000300090009e0f500006003a000b
:10fa50009e0090000040eb00c04098001000200085
:10fa600020079800060037001e009000400090001c
:10fa700010079800efff37002000200020079800b3
:10fa80002e0090000080fa00000006000600fa0038
:10fa9000000f7800c0908000100798001e009000b2
:10faa0000000e0000e0032001e00900030009000c8
:10fab0009e0f500006003a009e00900010c0b30058
:10fac000c040980010002000200798000600370072
:10fad0001e0090004000900010079800efff3700d4
:10fae00020002000200798002e0090000080fa00df
:10faf000000006003600f800809fbe00829fbe0016
:10fb0000849fbe00869fbe000200fa00c090800065
:10fb1000000f780084c0a9001e00e0001c00320025
:10fb20001e00780040409000e14f500014003a0061
:10fb30001e0078001000e000110032009e007800e6
:10fb40001e007800100090000000e800900098006f
:10fb50001e0178001e0078009000e900120090005d
:10fb6000810f5000060036001e0078003000900023
:10fb7000000001009e0078000000eb00900098005b
:10fb80001e00780040009000000f7800e2ff370070
:10fb90000080fa004f03be004f02be004f01be00be
:10fba0004f00be003600f900004006000600fa00d3
:10fbb000000f7800110798001e00780020079800b9
:10fbc0002e009000e30f5000640032002e009000e1
:10fbd000e30f500007003e002e009000e10f5000a0
:10fbe0002d0032002e009000e10f50003f003e003b
:10fbf0000d0037002e009000e50f50008f003200fe
:10fc00002e009000e40f5000700036002e0090008f
:10fc1000e60f5000a50032002e009000e70f5000c4
:10fc2000be003200d20037001e009000e10f5000ed
:10fc30000f003600c4c2bf000080fb004600de009b
:10fc40000080fb00610060000000a20061406000d5
:10fc50004601dd00412c200091407800f0cbb3003c
:10fc600000c0600002407000c4e2b7001c01370011
:10fc70002e409000614060004601dd00412c2000d4
:10fc800091407800f0cbb30000c0600002407000eb
:10fc9000c4e2b700120137001e009000e10f5000cf
:10fca0000b003600c4c2bf000080fb004700de002e
:10fcb0000080fb000000a200c700dd00c4c2bf003e
:10fcc0000074a10001407000c4e2b70004013700d5
:10fcd0002e409000c700dd00c4c2bf000074a10028
:10fce00001407000c4e2b700fd0037001e00900024
:10fcf000e10f50000f003600c5c2bf000080fb00be
:10fd00000000d1000080fb00610060000000a20044
:10fd1000614060000041d000512c200091407800eb
:10fd2000d0cfb30000c0600002407000c5e2b70051
:10fd3000eb0037002e409000614060000041d00091
:10fd4000512c200091407800d0cfb30000c060005b
:10fd500002407000c5e2b700e10037001e009000cd
:10fd6000e10f50000f003600c5c2bf000080fb004d
:10fd70004400de000080fb00610060000000a20083
:10fd8000614060004401dd00512c2000914078006a
:10fd9000f0ceb30000c0600002407000c5e2b700c2
:10fda000cf0037002e409000614060004401dd002c
:10fdb000512c200091407800f0ceb30000c06000cc
:10fdc00002407000c5e2b700c50037001e00900079
:10fdd000e10f50000f003600c5c2bf000080fb00dd
:10fde0004200de000080fb00610060000000a20015
:10fdf000614060004201dd00512c200091407800fc
:10fe0000b0cfb30000c0600002407000c5e2b70090
:10fe1000b30037002e409000614060004201dd00d9
:10fe2000512c200091407800b0cfb30000c060009a
:10fe300002407000c5e2b700a90037001e00900024
:10fe4000e10f50000f003600c5c2bf000080fb006c
:10fe50004500de000080fb00610060000000a200a1
:10fe6000614060004501dd00512c20009140780088
:10fe7000f0cdb30000c0600002407000c5e2b700e2
:10fe8000970037002e409000614060004501dd0082
:10fe9000512c200091407800f0cdb30000c06000ec
:10fea00002407000c5e2b7008d0037001e009000d0
:10feb000e10f50000f003600c5c2bf000080fb00fc
:10fec0004600de000080fb00610060000000a20030
:10fed000614060004601dd00512c20009140780017
:10fee000f0cbb30000c0600002407000c5e2b70074
:10fef0007b0037002e409000614060004601dd002d
:10ff0000512c200091407800f0cbb30000c060007d
:10ff100002407000c5e2b700710037001e0090007b
:10ff2000e10f50000b003600c5c2bf000080fb008f
:10ff30004700de000080fb000000a200c700dd00db
:10ff4000c5c2bf000074a10001407000c5e2b70047
:10ff5000630037002e409000c700dd00c5c2bf001f
:10ff60000074a10001407000c5e2b7005c003700da
:10ff70002e409000c700dd00c5c2bf000074a10084
:10ff800001407000c5e2b700c5c2bf000080fb00a1
:10ff90004700de000080fb00614060004601dd009c
:10ffa000512c200091407800f0cbb30000c06000dd
:10ffb00002407000c5e2b700c5c2bf000080fb0070
:10ffc0004600de000080fb006100600061406000d0
:10ffd0004501dd00512c200091407800f0cdb300a8
:10ffe00000c0600002407000c5e2b700c5c2bf009b
:10fff0000080fb004500de000080fb006100600027
:020000040001f9
:10000000614060004201dd00512c200091407800e9
:10001000b0cfb30000c0600002407000c5e2b7007e
:10002000c5c2bf000080fb004200de000080fb0074
:1000300061006000614060004401dd00512c20003f
:1000400091407800f0ceb30000c060000240700024
:10005000c5e2b700c5c2bf000080fb004400de005f
:100060000080fb0061006000614060000041d00042
:10007000512c200091407800d0cfb30000c0600028
:1000800002407000c5e2b700c5c2bf000080fb009f
:100090000000d1000080fb0061006000c700dd00af
:1000a000c4c2bf000074a10001407000c4e2b700e8
:1000b000c4c2bf000080fb004700de000080fb00e0
:1000c000614060004601dd00412c20009140780035
:1000d000f0cbb30000c0600002407000c4e2b70083
:1000e0000080fa00000006000000fa00c4c2a90067
:1000f000c4e2a900c522a900c582a900c542a90081
:10010000c5a2a900c5c2a900c5e2a9000080fa00e5
:10011000000006000200fa00000f78001000200026
:100120009e0f10000f003600d0c2bf000080fb0001
:100130004200de000080fb00610060000000a200c1
:10014000614060004201dd00012d200091407800f7
:10015000b0cfb30000c0600002407000d0e2b70032
:10016000090037009e40780061c060004201dd0058
:10017000012d200091407800b0cfb30000c0600096
:1001800002407000d0e2b7000080fa0000000600d4
:100190000200fa00000f7800100020009e0f1000ef
:1001a0000f003600d0c2bf000080fb000000d1006d
:1001b0000080fb00610060000000a2006140600060
:1001c0000041d000012d200091407800d0cfb30035
:1001d00000c0600002407000d0e2b70009003700a4
:1001e0009e40780061c060000041d000012d2000d9
:1001f00091407800d0cfb30000c060000240700092
:10020000d0e2b7000080fa00000006000000fa000b
:10021000c4c2bf000080fb004600de000080fb007f
:10022000610060000080ea00614060004601dd007e
:10023000412c200091407800f0cbb30000c060005a
:1002400002407000c4e2b700c4c2bf000080fb00df
:100250004700de000080fb000080ea00c700dd00f0
:10026000c4c2bf000074a10001407000c4e2b70026
:10027000c5c2bf000080fb000000d1000080fb0071
:10028000610060000080ea00614060000041d00031
:10029000512c200091407800d0cfb30000c0600006
:1002a00002407000c5e2b700c5c2bf000080fb007d
:1002b0004400de000080fb00610060000080ea0076
:1002c000614060004401dd00512c20009140780025
:1002d000f0ceb30000c0600002407000c5e2b7007d
:1002e000c5c2bf000080fb004200de000080fb00b2
:1002f000610060000080ea00614060004201dd00b2
:10030000512c200091407800b0cfb30000c06000b5
:1003100002407000c5e2b700c5c2bf000080fb000c
:100320004500de000080fb00610060000080ea0004
:10033000614060004501dd00512c200091407800b3
:10034000f0cdb30000c0600002407000c5e2b7000d
:10035000c5c2bf000080fb004600de000080fb003d
:10036000610060000080ea00614060004601dd003d
:10037000512c200091407800f0cbb30000c0600009
:1003800002407000c5e2b700c5c2bf000080fb009c
:100390004700de000080fb000080ea00c700dd00af
:1003a000c5c2bf000074a10001407000c5e2b700e3
:1003b0000080fa00000006000000fa00c4c2bf007e
:1003c0000080fb004600de000080fb006100600052
:1003d0000080ea00614060004601dd00412c200001
:1003e00091407800f0cbb30000c060000240700084
:1003f000c4e2b7000080fa00000006000000fa0026
:10040000c4c2bf000080fb004700de000080fb008c
:100410000080ea00c700dd00c4c2bf000074a10074
:1004200001407000c4e2b7000080fa00000006003e
:100430000000fa00c5c2bf000080fb000000d10030
:100440000080fb00610060000080ea006140600005
:100450000041d000512c200091407800d0cfb30053
:1004600000c0600002407000c5e2b7000080fa00e2
:10047000000006000000fa00c5c2bf000080fb00bb
:100480004400de000080fb00610060000080ea00a4
:10049000614060004401dd00512c20009140780053
:1004a000f0ceb30000c0600002407000c5e2b700ab
:1004b0000080fa00000006000000fa00c5c2bf007c
:1004c0000080fb004200de000080fb006100600055
:1004d0000080ea00614060004201dd00512c2000f4
:1004e00091407800b0cfb30000c0600002407000bf
:1004f000c5e2b7000080fa00000006000000fa0024
:10050000c5c2bf000080fb004500de000080fb008c
:10051000610060000080ea00614060004501dd008c
:10052000512c200091407800f0cdb30000c0600055
:1005300002407000c5e2b7000080fa00000006002b
:100540000000fa00c5c2bf000080fb004600de00cc
:100550000080fb00610060000080ea0061406000f4
:100560004601dd00512c200091407800f0cbb30013
:1005700000c0600002407000c5e2b7000080fa00d1
:10058000000006000000fa00c5c2bf000080fb00aa
:100590004700de000080fb000080ea00c700dd00ad
:1005a000c5c2bf000074a10001407000c5e2b700e1
:1005b0000080fa00000006000200fa00000f780038
:1005c0009e0078006010280088fc07000080fa0078
:1005d000000006000000fa0060102800b4fc0700cc
:1005e0000080fa00000006000200fa00000f780008
:1005f0001e00e000030035009e0078006010280017
:10060000d3fc07000080fa00000006000000fa009a
:10061000e851e2000b003a008000eb00700020007f
:1006200062fd0700e8d1bf000080fb001100200040
:100630005efd0700e8d1bf000040e800e8f1b70028
:100640001c003700801e210071c0b30090cf100045
:100650000c003a00e8d1bf000080fb000000e90078
:100660008000eb0051fd0700e8d1bf000080fb00d7
:10067000110020004dfd07000040eb00e8f1b7003d
:100680000c003700e8d1bf000080fb000000e9004b
:100690008000eb0045fd0700e8d1bf000080fb00b3
:1006a0001100200041fd0700e8d1bf000040e80034
:1006b000e8f1b7000080fa00000006000200fa002e
:1006c000e9d1bf000080fb00000f78001e00780019
:1006d000e20f50001c0032009e007800e28f5000b4
:1006e00007003c001e0078000000e0000b00320014
:1006f0009e007800e18f50000c003200230037008c
:100700001e007800e30f5000160032009e007800b3
:10071000e48f50001a0032001c0037002100200036
:100720000000eb0021fd0700180037002100200029
:10073000100020001dfd0700210020007000200097
:100740001afd0700110037002100200020002000c2
:1007500016fd0700210020006000200013fd0700a7
:100760000a00370021002000300020000ffd0700a4
:1007700021002000500020000cfd0700030037007e
:10078000210020004000200008fd0700901e2100ed
:1007900031c0b30090cf100004003e00e9d1bf008b
:1007a0000040e800e9f1b700020037000040eb002c
:1007b000e9f1b7000080fa00000006000000fa002e
:1007c000ea51e2000e003a001a52e2000c00320038
:1007d00010c0b300eaf1b7008000eb000000eb00ae
:1007e000f2fc0700ead1bf000080fb0011002000ee
:1007f000eefc07000040eb001af2b7002b003700b8
:10080000ea51e2000e003a001a52e2000c003a00ef
:1008100070c0b300eaf1b7008000eb000000eb000d
:10082000e2fc0700ead1bf000080fb0011002000bd
:10083000defc070010c0b3001af2b7001b0037003f
:10084000a01e210071c0b30090cf10000a003a0032
:100850000040eb00eaf1b7008000eb0070002000e0
:10086000d2fc0700ead1bf000080fb00110020008d
:10087000cefc07000d003700a01e210011c0b30000
:1008800090cf100009003a000040eb00eaf1b700f9
:100890008000eb0010002000c4fc0700ead1bf007c
:1008a0000080fb0011002000c0fc07000080fa005f
:1008b000000006000200fa00ebd1bf000080fb0040
:1008c000000f78001e007800e10f50001500320084
:1008d0009e007800e18f500004003c001e0078006c
:1008e0000000e000080032001a0037009e00780087
:1008f000e28f5000120032001e007800e30f50001b
:100900001300320013003700210020000000eb002c
:10091000a6fc07002100200040002000a3fc0700e7
:100920000c00370021002000100020009ffc070071
:1009300021002000300020009cfc0700050037004b
:10094000210020002000200098fc07000100370053
:10095000e5fd0700b01e210021c0b30090cf1000bc
:1009600004003e00ebd1bf000040e800ebf1b7000f
:10097000020037000040eb00ebf1b7000080fa0006
:10098000000006000200fa00ecd1bf000080fb006e
:10099000000f78001e007800e10f500015003200b3
:1009a0009e007800e18f500004003c001e0078009b
:1009b0000000e000080032001a0037009e007800b6
:1009c000e28f5000120032001e007800e30f50004a
:1009d0001300320013003700210020000000eb005c
:1009e00072fc070021002000400020006ffc07007f
:1009f0000c00370021002000700020006bfc070075
:100a0000210020005000200068fc0700050037008e
:100a1000210020006000200064fc07000100370076
:100a2000b1fd0700c01e210021c0b30090cf10000f
:100a300004003e00ecd1bf000040e800ecf1b7003c
:100a4000020037000040eb00ecf1b7000080fa0034
:100a5000000006000400fa00c411e2001c0032008d
:100a600080da2f00b811e30019003500802520003e
:100a7000b811e30016003c00d602a900d622a90056
:100a8000d642a900d662a9000000eb00208e8800a3
:100a9000c28d8000020f78001e0178000200e00085
:100aa00003003d001e0178000201ea00020f7800f9
:100ab000007122001e017800110009000200d80018
:100ac000ef005000a0522800a1fb070049003700aa
:100ad000b811e2000b003400008e80000000e80036
:100ae000008e8800e08d80000000e900e08d880025
:100af000bc11e2000e003d0030002000e08d8800b7
:100b00000b003700008e80000000e900008e880096
:100b1000e08d80000000e800e08d880030002000bb
:100b2000bc11e300020034000000eb00e08d8800ff
:100b3000e28d8000120798001e009000e10f500027
:100b4000130032001e019000e10f510004003c0030
:100b50001e0090000000e000080032001a0037007c
:100b60001e019000e20f51000e0032001e009000a6
:100b7000e30f50001000320013003700d602a90026
:100b8000d622a800d642a900d662a8000e003700df
:100b9000d602a900d622a800d642a800d662a90093
:100ba00009003700d602a800d622a900d642a80024
:100bb000d662a90004003700d602a800d622a900f8
:100bc000d642a900d662a80080da2f00b811e3004f
:100bd0000800350080252000b811e30005003c0026
:100be00010002000208e8800f1002000a052280074
:100bf00057fb07000080fa00000006000400fa001e
:100c0000c611e2001c00320080da2f00ba11e300a6
:100c10001900350080252000ba11e30016003c00c1
:100c2000d682a900d6a2a900d6c2a900d6e2a90000
:100c30000000eb00308e8800d28d8000020f78001b
:100c40001e0178000200e00003003d001e01780054
:100c50000201ea00020f7800007122001e017800f4
:100c6000110009000200d800ef005000e05f2800ea
:100c700037fb070049003700ba11e2000b003d00c6
:100c8000108e80000000e900108e8800f08d80003a
:100c90000000e900f08d8800be11e2000e003d006a
:100ca00030002000f08d88000b003700108e80008f
:100cb0000000e800108e8800f08d80000000e80041
:100cc000f08d880030002000be11e30002003400e7
:100cd0000000eb00f08d8800f28d80001207980074
:100ce0001e009000e10f5000130032001e01900022
:100cf000e10f510004003c001e0090000000e000e5
:100d0000080032001a0037001e019000e20f510067
:100d10000e0032001e009000e30f50001000320061
:100d200013003700d682a900d6a2a800d6c2a90017
:100d3000d6e2a8000e003700d682a900d6a2a800ed
:100d4000d6c2a800d6e2a90009003700d682a800c2
:100d5000d6a2a900d6c2a800d6e2a9000400370096
:100d6000d682a800d6a2a900d6c2a900d6e2a800c1
:100d700080da2f00ba11e30008003500802520003a
:100d8000ba11e30005003c0010002000308e8800fe
:100d9000f1002000e05f2800edfa07000080fa0073
:100da000000006000000fa008000eb00a0522800be
:100db0008efa07008000eb00e05f28008bfa070046
:100dc0000080fa00000006000200fa00000f780020
:100dd0001e00e0000a003a000000eb00c08d880011
:100de0008000eb00a0522800d9fa0700d602a90023
:100df000d622a900d642a900d662a9002d0037004c
:100e000080c12f009e0f10000a003d0080c12f00fe
:100e1000c08d8800008f2d00c28d80001100090058
:100e20000200d8008000fd00a0522800c8fa070088
:100e300020003700803e20009e0f10000a00340082
:100e4000803e2000c08d880000712200c28d80008d
:100e5000110009000200d8008000fd00a052280007
:100e6000bbfa0700130037001e007800c08d880011
:100e70001e00e00008003d00008f2d001e017800dc
:100e8000110009000200d8008000fd00a0522800d7
:100e9000affa070007003700007122001e0178003a
:100ea000110009000200d8008000fd00a0522800b7
:100eb000a7fa07000080fa00000006000200fa000e
:100ec000000f78001e00e0000a003a000000eb006e
:100ed000d08d88008000eb00e05f28009cfa0700be
:100ee000d682a900d6a2a900d6c2a900d6e2a9003e
:100ef0002d00370080c12f009e0f10000a003d001a
:100f000080c12f00d08d8800008f2d00d28d8000f1
:100f1000110009000200d8008000fd00e05f2800f9
:100f20008bfa070020003700803e20009e0f100043
:100f30000a003400803e2000d08d8800007122001d
:100f4000d28d8000110009000200d8008000fd0051
:100f5000e05f28007efa0700130037001e007800cb
:100f6000d08d88001e00e00008003d00008f2d009d
:100f70001e017800110009000200d8008000fd0069
:100f8000e05f280072fa07000700370000712200b6
:100f90001e017800110009000200d8008000fd0049
:100fa000e05f28006afa07000080fa0000000600ef
:100fb0000800fa00000f7800110798001e00780062
:100fc000200798002e0190000200e00003003d0081
:100fd0002e0090000000ea00200798001e019000fb
:100fe000320798003e0090000000e00003003d0042
:100ff0003e0190000201ea00320798002e009000a6
:101000003e01900082004000803e2000808f500012
:1010100006003c001e0090001e0010006aff070042
:101020001e0090001e004000a4ff07000080fa0090
:10103000000006000000fa00008e80000080fa0028
:10104000000006000200fa00000f78001e00780081
:10105000008e88000080fa00000006000000fa0000
:10106000108e80000080fa00000006000200fa00e6
:10107000000f78001e007800108e88000080fa00b3
:10108000000006000000fa00dec2a8008200a800ee
:101090008400a9008c00a8000080fa00000006006f
:1010a0003600f800809fbe00829fbe00849fbe0075
:1010b000869fbe000000fa008c00a90051012000ac
:1010c000e0872800c9f907000040eb00eff1b70006
:1010d0000040eb00eef1b7000040eb00f0f1b7008c
:1010e0000080fa004f03be004f02be004f01be0059
:1010f0004f00be003600f900004006000200fa0072
:101100000080eb000e12e3001a003a00e0c2bf00bc
:101110000080fb004600de000080fb0061006000f4
:101120000000e000070032008c00a8008400a90045
:10113000e0872800def907000080eb00709088004f
:101140005800370091002000e087280000fa0700cf
:101150000040eb00eff1b7000040eb00eef1b7000c
:101160000040eb00f0f1b7000000eb007090880049
:101170004c003700100020000e12e3000d003a0072
:10118000e0c2bf000080fb004600de000080fb00e4
:1011900061006000f0f1b70021012000e087280025
:1011a000ebf9070011002000100020007ffa070073
:1011b0003c003700100020000e12e3001200340043
:1011c000600020000e12e3000f003c00e0c2bf00f0
:1011d0000080fb004600de000080fb006100600034
:1011e000004f78009e80fb00709080006600100029
:1011f0000008dd00004f7800eed1bf001e40400027
:10120000eef1b70027003700600020000e12e30067
:1012100012003400c00020000e12e3000f003c005a
:10122000e0c2bf000080fb004600de000080fb0043
:1012300061006000004f78009e80fb00709080008d
:101240006c0010000008dd00004f7800efd1bf00f7
:101250001e404000eff1b70012003700d000200020
:101260000e12e3000f003a008000eb001000200097
:101270004efa07008c00a8008400a900e08728002f
:101280008bf907000080eb0070908800f0d1bf0060
:101290000cf2b700eed1bf00f1f1b700efd1bf0003
:1012a000f2f1b7000080eb000e12e3000300320001
:1012b000709080000000e800709088000080fa00c4
:1012c000000006000000fa000cd2bf000080fb0006
:1012d0000080fa00000006000000fa00f1d1bf0013
:1012e0000080fb000080fa00000006000000fa0009
:1012f000f2d1bf000080fb000080fa000000060071
:101300000000fa00c4c2a900c4e2a900c522a900d5
:10131000c582a900c542a900c5a2a900c5c2a900ed
:10132000c5e2a900c0c2a900c0e2a900c122a9006b
:10133000c182a900c142a900c1a2a900c1c2a900dd
:10134000c1e2a900d022a900cc22a900d042a90064
:10135000cc42a900e2e2a900e302a900e802a90048
:10136000e822a900dee2a900df02a900e402a90048
:10137000e422a900e202a900de02a900d602a90027
:10138000d622a900d642a900d662a900d682a90019
:10139000d6a2a900d6c2a900d6e2a900d202a9000d
:1013a000d222a900d242a900d262a900d282a90009
:1013b000d2a2a900d2c2a900d2e2a900d1a2a9005a
:1013c000cda2a900e842a900e862a900e442a90070
:1013d000e462a900de22a800dec2a800e4c2a800e0
:1013e000e4e2a800e502a800e522a800d302a800d4
:1013f000d322a800d342a800d362a800d382a800b9
:10140000d3a2a800d3c2a800d3e2a8000080fa00ab
:10141000000006000c22ef000e22ef000ee2a900f1
:101420000ec2a9008520a9008d20a8000de2a80009
:1014300070002000a01088008540a9008d40a80001
:1014400081e0a900c0048000f1002f00008060004e
:101450000155200000804000c00488000fe2a80071
:101460000f42a800ba30ef00bc30ef0000000600c9
:101470001622ef001822ef0018e2a90018c2a900f6
:101480008700a9008f00a80017e2a800f0108800cc
:101490008720a9008f20a80081e0a9000005800016
:1014a00001f02f0000806000510520000080400006
:1014b0000005880019e2a8001942a800fe30ef00dc
:1014c0000031ef0000000600809fbe008520a900cb
:1014d000d0858000f003b200a10721008100400008
:1014e0000000eb0012c2bf0080487800ba30ec0068
:1014f0004f00be0000400600d0858000e1858000de
:101500000100500000000600d1858000e2858000c7
:101510000208e10008003200f203b200a107210036
:10152000028140009240780001487800bc30ec0015
:1015300010002000000006000000eb000000060084
:101540008540a900809fbe00821f7800f811e2004c
:1015500015003200f411e20016003200f611e2002c
:1015600014003200a18f8000420020000f22af0043
:10157000feff3700b08f80000000e000070032005f
:101580000000e900f6b1b7003140780010e2b70082
:101590000201e900f5ff3a0002003700f431ef00e4
:1015a00001003700a18f88004f0178004f00be0076
:1015b0000040060000002000c08f88004f01780026
:1015c0004f00be0000400600f811e200feff3a00a6
:1015d0008d40a9008100e900b18f8800b0407800fb
:1015e00081108800a08f880011002000c18f880022
:1015f0008d40a80000000600c08f8000000006009b
:10160000809fbe008700a900f0878000f003b20031
:10161000e10b2100810040000000eb001cc2bf0074
:1016200080487800fe30ec004f00be00004006000d
:10163000f087800001888000010050000000060053
:10164000f1878000028880000208e1000800320073
:10165000f203b200e10b21000281400092407800c9
:10166000014878000031ec00100020000000060066
:101670000000eb00000006008720a900809fbe004c
:10168000821f7800fe11e20015003200fa11e2001c
:1016900016003200fc11e20014003200d18f8000ed
:1016a000420020001922af00feff3700e08f8000cb
:1016b0000000e000070032000000e900fcb1b700c4
:1016c000314078001ae2b7000201e900f5ff3a0064
:1016d00002003700fa31ef0001003700d18f880097
:1016e0004f0178004f00be000040060000002000bf
:1016f000f08f88004f0178004f00be0000400600c8
:10170000fe11e200feff3a008f20a9008100e900ef
:10171000e18f8800b0407800d1108800d08f880019
:1017200011002000f18f88008f20a8000000060023
:10173000f08f8000000006000600fa00000f78001d
:101740001e007800200798002e019000e10f510044
:10175000130032002e0090000000e0000400320070
:101760002e019000e20f51001900320024003700d2
:101770009e007800200320000008b8002276800038
:10178000020040000000d00062d92000820040002a
:10179000808c800011001000100798001a0037009c
:1017a0009e007800200320000008b8002276800008
:1017b000020040000000d00062d9200082004000fa
:1017c000908c800011001000100798000e00370068
:1017d0009e007800200320000008b80022768000d8
:1017e000020040000000d00062d9200082004000ca
:1017f00000918000110010001007980002003700cf
:10180000a0292000100798001e0090000080fa0018
:10181000000006000c00fa00000f78001107980085
:101820006000b800200798003107980020002000d1
:101830009e0f100031003e001e0090000000e000ee
:101840002e0032009e00900020032000808f500068
:101850002a003e000000eb0040079800217680003f
:101860001e009000008050003003b00022032000d2
:10187000110009000280d8008000fd005007980088
:10188000ce0090001e009000808f50001b003100a1
:101890009e007800200320000008b8005e01900040
:1018a000020040000000d00061d92000010040008b
:1018b000100078006101b9002e009000be00900079
:1018c00000004100818049002007980031079800fe
:1018d0004e0090000000e800400798005e00900075
:1018e0000000e80022032000110009000200d800d7
:1018f0008000fd0050079800e1ff37001e009000b7
:101900006101b8002e009000be009000ebca0700f5
:101910000080fa00000006000000fa0051002000dc
:101920000000eb00bbff070080007800808c800087
:1019300000805000a08c8800510020001000200082
:10194000b4ff070080007800908c80000080500079
:10195000b08c88005100200020002000adff07005f
:10196000800078000091800000805000c08c8800ca
:101970000080fa00000006000000fa00889fbe0008
:10198000e5ff0700a18c8000a08c80000089b900d1
:10199000b18c8000b08c80000088b900020140004a
:1019a00083814800c18c8000c08c80000088b90011
:1019b000020040008380480075c907001fd007005f
:1019c000d08c8800e18c8800a18c8000a08c8000e5
:1019d0000089b900b18c8000b08c80000088b9000b
:1019e000020040008380480069c9070013d0070047
:1019f0000004be00c08c8000cf80de0064c90700f8
:101a00000801be008dc90700c20923005326240027
:101a1000e9c907000001be0000002000412b24009e
:101a200019ca0700108d8800218d8800020020004f
:101a3000030a2400108d8000218d800099ca0700c0
:101a40000000e00004003d006000b800f08c880059
:101a5000018d880011003700b08c8000cf80de003f
:101a60004bc907000004be00a08c8000cf80de00c0
:101a700047c907000801be0070c90700c20923005a
:101a800053262400ccc90700020020004333240061
:101a9000fec90700f08c8800018d88004f04be004d
:101aa0000080fa00000006000000fa002103200078
:101ab0000000eb0057ff0700808c88002103200006
:101ac0001000200053ff0700908c880021032000a5
:101ad000200020004fff070081d12f0001004000af
:101ae000009188000080fa00000006000c00fa0057
:101af000881f7800000478009fff0700d08c8000ca
:101b0000e18c8000008fbe00f28c8000038d80008d
:101b10002207980033079800108d8000218d8000e7
:101b200040079800510798008e0078000800780060
:101b30001101be000288be0064004000e480400045
:101b40001101be000288be0064004000e480400035
:101b50001101be000288be00080078004f04780022
:101b60000080fa00000006000000fa0082ff070073
:101b7000108d8000218d80000080fa00000006009a
:101b80000000fa007cff0700f08c8000018d8000cf
:101b90000080fa00000006000000fa0076ff07004f
:101ba000d08c8000e18c80000080fa0000000600ec
:101bb0000600fa00881f78000004780056ff07002e
:101bc000a08c8000000f7800b18c80001107980075
:101bd000c08c8000200798001e00be00008cbe0054
:101be000ae00900021049800080078004f047800af
:101bf0000080fa00000006000000fa0046ff07001f
:101c0000a08c80000080fa00000006000000fa00ae
:101c100041ff0700b08c80000080fa000000060041
:101c20000000fa003cff0700c08c80000080fa0032
:101c3000000006000a00fa006000b800008fbe0035
:101c4000cfff0700008fbe00708c8000cf80de00c9
:101c5000cfc807001e01be008bc90700f0c90700ee
:101c6000200798002e0090000000e00003003d00d7
:101c7000ae0090008100ea00210798002e0190003c
:101c80006110b900c2c8070002002000030a240046
:101c900006ca07000000e000dc003400c5e2a9002d
:101ca000c5c2bf000080fb004700de000080fb00d3
:101cb000614060004601dd00512c20009140780019
:101cc000f0cbb30000c0600002407000c5e2b70076
:101cd000c5c2bf000080fb004600de000080fb00a4
:101ce00061006000614060004501dd00512c200072
:101cf00091407800f0cdb30000c060000240700059
:101d0000c5e2b700c5c2bf000080fb004500de0091
:101d10000080fb0061006000614060004201dd0066
:101d2000512c200091407800b0cfb30000c060007b
:101d300002407000c5e2b700c5c2bf000080fb00d2
:101d40004200de000080fb00610060006140600036
:101d50004401dd00512c200091407800f0ceb3000a
:101d600000c0600002407000c5e2b700c5c2bf00fd
:101d70000080fb004400de000080fb00610060008a
:101d8000614060000041d000512c2000914078005b
:101d9000d0cfb30000c0600002407000c5e2b700c1
:101da000c5c2bf000080fb000000d1000080fb0026
:101db00061006000c700dd00c4c2bf000074a10064
:101dc00001407000c4e2b700c4c2bf000080fb0045
:101dd0004700de000080fb00614060004601dd003e
:101de000412c200091407800f0cbb30000c060008f
